:020000040800F2
:1080000068F50020A1810008A981000889AB00085B
:10801000AD810008AF810008B181000800000000B8
:10802000000000000000000000000000B381000814
:10803000B581000800000000B7810008B981000880
:10804000BB810008BB810008BB810008BB81000820
:10805000BB810008BB810008199E0008299E00080A
:10806000BB810008BB810008BB810008BB81000800
:10807000BB810008BB810008AB990008B3990008D8
:10808000BB810008BB990008BB810008BB810008C8
:10809000BB810008BB810008BB810008BB810008D0
:1080A000BB810008BB810008BB810008BB810008C0
:1080B000CD5C0308BB810008BB810008BB810008C0
:1080C000BB810008BB810008BB810008BB810008A0
:1080D000BB810008236C03082B6C0308336C030876
:1080E000219E0008BB810008BB810008BB810008FD
:1080F000BB810008BB810008BB810008C399000850
:10810000BB810008BB810008BB810008BB8100085F
:10811000136C03081B6C0308BB810008BB810008BB
:10812000BB810008BB810008BB810008BB8100083F
:10813000BB810008BB810008BB810008BB8100082F
:10814000BB810008BB810008BB810008BB8100081F
:10815000BB810008CB990008D39900083B6C030849
:10816000BB810008BB810008BB810008BB810008FF
:10817000BB810008BB810008BB810008BB810008EF
:10818000BB810008BB810008DFF810D000F058FC6C
:1081900000480047818A0308AFF3008068F500209B
:1081A0000648804706480047FEE7FEE7FEE7FEE791
:1081B000FEE7FEE7FEE7FEE7FEE7FEE7655C030895
:1081C000898100082DE9F0410024061B254671F144
:1081D000000605DA01240027D0EB070067EB010158
:1081E000161E73F1000605DA0027D2EB07020125FF
:1081F00067EB030300F0C1FA86460E4617469C461D
:10820000AC4204D00025D0EB050E65EB010624B18D
:108210000020D2EB000760EB030C704631463A4673
:108220006346BDE8F081202A06DBCB17203A41FAED
:1082300002F043EAE07306E041FA02F3D040C2F1F3
:108240002002914008431946704740EA01039B070A
:1082500003D009E008C9121F08C0042AFAD203E0BB
:1082600011F8013B00F8013B521EF9D27047421E43
:1082700012F8013F002BFBD111F8013B02F8013B42
:10828000002BF9D17047421C10F8011B0029FBD1CB
:10829000801A704730B505460020034600E05B1C9D
:1082A000934205D2EC5CC85C201A01D1002CF6D1B7
:1082B00030BD2DE9FE4F804681EA0300C00F0C4619
:1082C000009021F0004123F00045B8EB0200A941E5
:1082D00005D24046214690461C460B46024623F0F6
:1082E0000040104347D0270DC7F30A00C3F30A51DB
:1082F0000290401A019040286BDAC3F3130040F457
:10830000801B0098924620B10023D2EB030A63EB56
:108310000B0B01985946C0F14002504600F05EFA3E
:1083200006460D4650465946019AFFF77CFF10EB72
:1083300008006141002487EA115284EAE7731A4376
:1083400040D0009A62B3019A012A4FEA075215DC25
:10835000001B61EB02014FF0004202EA0752CDE937
:108360000042001C41F5801132462B4600F0EAFA2B
:1083700003B0BDE8F08F40462146F9E7001B61EBF2
:108380000201001C41F5801300185B412018A2F582
:10839000001747EB030140EAD570B6196D4111E0B3
:1083A0006D084FEA360645EAC0754FEA0752001BD2
:1083B00061EB0201001C41F5801149084FEA3000D1
:1083C0000019514132462B4603B0BDE8F04F00F092
:1083D000AABA0098012240000023D0EB020263EB0E
:1083E000E073009821464FEAE074B8EB000061EBBF
:1083F0000401E9E783F000435BE781F0004158E7BF
:108400002DE9FE4F81EA030404F0004421F000410D
:1084100000944FF0000B23F0004350EA01045ED0BB
:1084200052EA03045BD0C3F30A54C1F30A552C4447
:10843000A4F2F3340194A0FB0254C1F3130141F4FC
:108440008011C3F3130343F4801301FB024400FBC8
:10845000034E840A970A44EA815447EA8357A4FBEF
:10846000076802958D0A05FB07854FEA932C04FBEC
:108470000C542705029D4FEA065847EA1637B5EB1C
:1084800008056EEB070C870E920E47EA811742EA49
:108490008312A7FB0201B6EB0B0164EB00042B0D6A
:1084A00043EA0C335E1844EB1C50DA465146E7FBB6
:1084B0000201C5F313044FEA0B3343EA14534FEAA6
:1084C0000432019C43EA0603A4F10C040294009CCC
:1084D000CDE900B400F036FA03B0BDE8F08F00201B
:1084E0000146F9E72DE9F04D81EA030404F0004B61
:1084F00021F0004514464FF0000A23F0004150EAF5
:10850000050220D054EA01021DD0C5F30A570246E5
:10851000C5F31303C1F31300C1F30A5640F48015E9
:1085200043F48013A7EB0608101BD64608F2FD386B
:1085300073EB050002D308F1010801E092185B41DA
:10854000B8F1000F03DA00200146BDE8F08D0020ED
:108550004FF48011064684460EE0171B73EB0507A7
:1085600005D3121B63EB050306434CEA010C4908D3
:108570004FEA300092185B4150EA0107EDD152EA10
:10858000030012D082EA040083EA0501084305D003
:10859000101BAB4106D20122002306E000224FF05F
:1085A000004302E06FF0010253101AEB06004CEB9F
:1085B000085110EB0A0041EB0B01BDE8F04D00F053
:1085C000B2B9F0B4CA17CB0F50405140C61841F1B0
:1085D00000054FEAC372314628004FF0960303D0DE
:1085E000B623F0BC00F071B930460021F9E70EB5B2
:1085F000C10F80EAE0700844CA07002140F233430B
:108600008DE80E000A460B4600F09CF903B000BD51
:108610000EB540F2334102910021CDE900110A4626
:108620000B4600F08FF903B000BD3EB5CA17CB0F63
:10863000002450405140C0186141DA0740F23343F2
:108640000094CDE901232246234600F07BF903B0D4
:1086500030BD10B500F0004420F00040C20DC0F362
:10866000160040F400007F2A02DA0020014610BD07
:108670000021962A03DCC2F19602D04002E0963A2D
:1086800000F0ACF8002CF2D00023D0EB030063EB39
:10869000010110BD70B5C1F30A5201F0004500247C
:1086A000C1F3130140F2FF3341F480119A4201DA21
:1086B000002070BD40F233439A42A2F2334203DC01
:1086C000524200F09AF800E090402C43F1D0404232
:1086D00070BD70B5C1F30A5201F000450024C1F32A
:1086E000130140F2FF3341F480119A4202DA002074
:1086F000014670BD40F233439A42A2F2334203DC9A
:10870000524200F07AF801E000F068F82C43F0D013
:108710000023D0EB030063EB010170BD00F00042C9
:1087200030F000400AD0C10D01F56071C0F31600B1
:1087300042EA0151C2084007114370470020014638
:10874000704701F0004330B421F0004150EA0102CB
:1087500006D00A0DA2F56072C1F31301002A02DCF3
:1087600030BC00207047440F44EAC104C100E01847
:1087700030BC00EBC25000F09FB82DE9F05F054619
:10878000002092469B4688460646814640241BE0D0
:10879000284641464746224600F02FF853465A469F
:1087A000C01A914110D311461846224600F016F81F
:1087B0002D1A67EB01084F4622460120002100F0E8
:1087C0000DF817EB00094E41201EA4F10104DFDC77
:1087D000484631462A464346BDE8F09F202A04DB3E
:1087E000203A00FA02F1002070479140C2F12003C4
:1087F00020FA03F3194390407047202A04DB203A03
:1088000021FA02F00021704721FA02F3D040C2F1B0
:108810002002914008431946704700000FB400231E
:1088200000B589B00CA900910B996FF00042CB60A4
:108830001E4B06931E4B07930423CDE901321D4ABC
:10884000089202466B46002000F0A6F909B05DF8D8
:1088500014FB70B586B006464FF0FF300091CDE9AD
:108860000101002015460C4604903246694604A8D2
:10887000FFF7D4FF02460498211825B108B1084635
:1088800000E020462860049800280DD0002A02DD70
:108890000098884208D0081B0094CDE901043246B4
:1088A000694604A8FFF7BAFF06B070BDD18D000875
:1088B000EF8D0008658A00080029A8BF7047401C9A
:1088C000490008BF20F00100704710B4B0FA80FCE6
:1088D00000FA0CF050EA010404BF10BC704749B123
:1088E000CCF1200421FA04F411FA0CF118BF012193
:1088F00021430843A3EB0C01CB1D4FEA00614FEA73
:10890000102042BF002010BC704700EBC350104441
:108910000029A4BF10BC7047401C490008BF20F0CC
:10892000010010BC704710B5141E73F1000408DA82
:10893000401C41F1000192185B411A4301D120F023
:10894000010010BD2DE9F04D92469B4611B1B1FAE0
:1089500081F202E0B0FA80F220329046FFF73EFF4B
:1089600004460F4640EA0A0041EA0B0153465A46C4
:10897000084313D0114653EA010019D0C8F1400250
:108980005046FFF73AFF05460E46504659464246C6
:10899000FFF724FF084305D0012004E020463946B4
:1089A000BDE8F08D0020054346EAE0762C433743CE
:1089B0000A986305E40AA0EB08000022FD0A44EAD5
:1089C00047540A3002D500200146E9E70105101995
:1089D0006941DDE9084500196941BDE8F04DA2E7AC
:1089E00070B521F0004303430CD0C1F30A550024B5
:1089F000D5EB040564EB0403D617AD1AB34102DBD3
:108A00000020014670BD201841EB025170BD0000EE
:108A100030B5041E71F1000404DB4FF00044404205
:108A200064EB0101141E73F1000405DB1C464FF0DA
:108A30000043524263EB0403994208BF904230BDA9
:108A4000064C074D06E0E06840F0010394E807009B
:108A500098471034AC42F6D3FFF79AFB081104088C
:108A600028110408C0B24FF4F05100F03BBA0000E6
:108A70002DE9FF4F087883B09946FF2805D0491C9F
:108A80002D2804D00024002008E000200BE0012461
:108A9000F9E700EB800003EB4000491C0B78FF2B4B
:108AA000F7D104B1404200230293147819461D46C1
:108AB0002D2C01D02B2C04D1521C2D2C13D0002492
:108AC0000294AA461478FF2C0FD00A25A3FB057840
:108AD00001FB05814FF0000C03FB0C11521CE31944
:108AE0004AEB0101EEE70124EAE7814453EA010081
:108AF00002D019F5C87F06DA03980021C0E90011F9
:108B000007B0BDE8F08F0025AE4E2F46DFF8B882E3
:108B1000184600F0FBF9CDE90001B9F1000002DAD6
:108B2000C9F1000400E004460023A74A1AEB030B36
:108B300042EB045A12E0E00707D02A463346384693
:108B40004146FFF75DFC074688462A4633461046F5
:108B50001946FFF755FC05460E466410002CEAD175
:108B6000DDE90001B9F1000F5A46534606DAFFF776
:108B7000B9FC3A464346FFF7B5FC05E0FFF740FC79
:108B80003A464346FFF73CFC029A0AB181F00041A5
:108B9000039AC2E90001B3E72DE9FF4F1F468DB0EC
:108BA000D7E901464FF0FF382E2045464FF0000927
:108BB0000B90B9696D1C0E988847396A82468847C0
:108BC0000028F6D1BAF1FF3F0AD024F4D064002E79
:108BD00011DDBAF12B0F08D0BAF12D0F0BD102E045
:108BE000404611B08DE744F48064B9696D1C0E985D
:108BF00088478246761E6946600501D52D2000E033
:108C00002B208DF8000001F1010B0DF1200809E087
:108C1000B9696D1C0E98884782460F9844F4007419
:108C2000761E0560002E02DDBAF1300FF0D00B99F0
:108C30008A453ED144F0800406E00F99681CA9F1F2
:108C4000010944F400740860B9696D1C761E0E9821
:108C5000884782463028F0D02BE00B998A4505D111
:108C6000200603D444F08004761E18E050462FF00E
:108C700021FB08B30DF11301761E44F400748B45FB
:108C800008D2AAF130000BF8010B200607D5A9F194
:108C9000010003E0200602D409F101008146A0058D
:108CA00002D50F99681C0860B9696D1C0E98884739
:108CB0008246002ED1DC53E0002E51DDBAF1650F63
:108CC00002D0BAF1450F4BD1A00549D5B9696D1C49
:108CD00024F44074761E0E9888478246002E0CDDE0
:108CE0002B2804D0BAF12D0F07D144F48074B96950
:108CF0006D1C0E9888478246761EE00501D52D2111
:108D000000E02B2108F8011BCDF82C8021E00DF1AB
:108D10002901761E44F4007488450CD2AAF1300073
:108D200010F0FF0088F8000002D10B99884509D99E
:108D300008F1010806E0E00501D5244801E042F20F
:108D40000F708146B9696D1C0E98884782460F984E
:108D50000560002E04DD50462FF0ACFA0028D6D175
:108D6000F9690E988847FF208BF8000088F800000A
:108D70000020069007904B466A4608A906A8FFF710
:108D800077FEA00502D46FF001002AE714F0240F4B
:108D90000AD0E00714D1DDE906123868031D3B60F4
:108DA0000068C0E900120BE0DDE90601FFF7C9FC2D
:108DB0000146E00704D13868021D3A60006801608E
:108DC00028460EE7000014400000F03FF1D8FFFFF6
:108DD000426842B1016811F8013B23B1521EC0E95B
:108DE0000012184670470121C160881E7047426812
:108DF0005AB1C368016843B983688B4205D0491EE4
:108E0000521CC0E90012002070474FF0FF3070473D
:108E10002DE9F04D00231A461B1A8A4103DB00207E
:108E20000146BDE8F08DC1F30A52C1F3130141F4CC
:108E300080154FF0000BD10702D100186D41521E72
:108E40000027044640F2FF11384601EB620A3E4615
:108E50008046024600204FF48011FFF7CEFCC21975
:108E60007141BB1846EB0100B4EB030C75EB000C31
:108E700004D3E41A65EB000517460E46241908F1E1
:108E800001006D4180463428E3DDF91946EB060008
:108E9000091BA84103D24FF0FF32134601E0002224
:108EA00013461BEB070046EB0A51BDE8F04DFFF7F8
:108EB0003ABD000030B5041E71F1000404DB4FF030
:108EC0000044404264EB0101141E73F1000405DB11
:108ED0001C464FF00043524263EB04038B4208BF31
:108EE000824230BD7F2801D9002208E0064A02EB09
:108EF0005002C007127800D1120902F00F020120BF
:108F00009040084070470000C81004080EB540F2B9
:108F1000334202920022CDE900221346FFF712FDF0
:108F200003B000BD70B58C1810F8015B15F0070395
:108F300001D110F8013B2A1106D110F8012B03E0F2
:108F400010F8016B01F8016B5B1EF9D12B0705D4FA
:108F50000023521E0DD401F8013BFAE710F8013B43
:108F6000CB1A921C03E013F8015B01F8015B521E5F
:108F7000F9D5A142D8D3002070BD10B502461078B3
:108F800003E012F8014B2318D8B20B1EA1F1010423
:108F9000A1B2F6D110BD000070B5ADF5287D044634
:108FA0000D460020A790A690002604EB44004549FA
:108FB00001EBC000408AA84203DC00200DF5287DAB
:108FC00070BD0020A69077E004EB44003D4B03EB1E
:108FD000C000028A04EB440003EBC00080892844EF
:108FE00081B2394800F010F90020A79011E004EB9D
:108FF0004400344901EBC0004068BDF89C12405C5D
:1090000001A9BDF89C228854BDF89C02401C80B286
:10901000A79004EB44002B4901EBC000008ABDF887
:109020009C128842E3DC04EB4400264A02EBC000B9
:10903000008A401E81B201A8FFF79FFF23490870F4
:1090400004EB44001F4901EBC000008A401E01A947
:10905000085C1E490978884226D10020A79016E0B6
:1090600004EB4400174901EBC0004068BDF89C12B6
:10907000405C04EB4401134A02EBC1018968BDF86E
:109080009C228854BDF89C02401C80B2A79004EB3F
:1090900044000C4901EBC000008A401EBDF89C1240
:1090A0008842DDDC012089E764202FF041FBBDF818
:1090B0009802401C80B2A690BDF89802062883DB77
:1090C00000207BE774E80308D0AE0020310A0020BE
:1090D0002DE9F043ADF5257D04460E460025002719
:1090E000A846A94604EB4400324901EBC000408A7F
:1090F000B04204DC00200DF5257DBDE8F08300259D
:1091000018E004EB44002B4901EBC0008068405D8F
:1091100004EB4401274A02EBC1014968485504EBBE
:109120004400114601EBC0004068405D0DF80500A9
:10913000681C85B204EB44001E4901EBC000008AA4
:10914000401EA842DDDC04EB44000A4602EBC000EE
:10915000008A401E81B26846FFF70FFF04EB44010E
:10916000144A02EBC101098A491E0DF801000027CB
:109170001BE004EB44000F4B03EBC000028A04EB3E
:10918000440003EBC0008089304481B2684600F09F
:109190004FF931462046FFF7FFFE012800D1AAE72C
:1091A00064202FF0C5FA781C87B2062FE1DB00207F
:1091B000A1E7000074E8030808B50020009029F03A
:1091C000FDFD0F49087000F09BF80D480078242839
:1091D00004D0272807D028280FD109E0002109480A
:1091E00080F8081D09E00121064880F8081D04E008
:1091F0000221044880F8081D00BF00BF08BD000020
:109200002C0A0020BC2200202DE9F04106460D4624
:109210001746002401202FF043F800202849088039
:109220000DE029F0ADFD00F0800000B10BE0012061
:109230002FF07EFA22480088401C214908802048EF
:109240000088C828EDDB00BF1D480088C82832DA36
:1092500010211C4801F08CFC08211A4801F08AFCFE
:10926000E82000F031F8C5F3871000F02DF8A906CA
:10927000080E00F029F8002000F026F8002404E091
:10928000002000F021F8601C84B2042CF8DB0024DC
:1092900005E0FF2000F018F83055601C84B2BC4295
:1092A000F7DB1021074801F065FC00202EF0F8FFE5
:1092B0000120BDE8F08100202EF0F2FF0020F8E749
:1092C0002E0A00200000024010B5044600BF022113
:1092D0000A4829F083FE0028F9D02146074829F0E2
:1092E00089FE00BF0121054829F078FE0028F9D049
:1092F000024829F07CFEC0B210BD000000300140E1
:1093000010B501202EF0CCFF00201E4908800DE092
:1093100029F036FD00F0800000B10BE001202FF0B5
:1093200007FA18480088401C16490880154800882C
:10933000C828EDDB00BF13480088C8281CDA1021BC
:10934000114801F015FC08210F4801F013FC3D20E5
:10935000FFF7BAFF2A20FFF7B7FF8020FFF7B4FF1F
:10936000A720FFF7B1FF1021074801F003FC002000
:109370002EF096FF012010BD00202EF091FF00205E
:10938000F9E700002E0A00200000024070B50546F3
:109390000E46002401202EF083FF00202249088081
:1093A0000DE029F0EDFC00F0800000B10BE00120A1
:1093B0002FF0BEF91C480088401C1B4908801A4841
:1093C0000088C828EDDB00BF17480088C82825DAC8
:1093D0001021164801F0CCFB0821144801F0CAFB0B
:1093E0008420FFF771FF0020FFF76EFF0020FFF7DA
:1093F0006BFF0020FFF768FF002404E0285DFFF703
:1094000063FF601C84B2B442F8DB1021074801F00E
:10941000B1FB00202EF044FF012070BD00202EF093
:109420003FFF0020F9E700002E0A00200000024064
:1094300070B506460C46154601202EF031FF294630
:109440003046FFF7A3FF08B9002070BD00201F4978
:1094500008800DE029F094FC00F0800000B10BE0E2
:1094600001202FF065F919480088401C1749088031
:1094700016480088C828EDDB00BF14480088C828BB
:109480001EDA1021124801F073FB0821104801F088
:1094900071FB8320FFF718FFC4F38710FFF714FF59
:1094A000A106080EFFF710FF0020FFF70DFF1021A7
:1094B000074801F05FFB00202EF0F2FE0120C4E718
:1094C00000202EF0EDFE0020BFE700002E0A002055
:1094D0000000024030B502460020002304E012F8EC
:1094E000014B60405C1CE3B28B42F8DB30BD70B5D1
:1094F00004460D46164632462946204600F001F83D
:1095000070BDF8B503460C460020002100BF06E000
:10951000C50022FA05F5EDB20DF80050401C0428F4
:10952000F6DB00201AE0064600EBD6777F100FB975
:10953000012701E04FF0FF373D4600210BE01E5CA4
:10954000012D01D10F4601E0C1F103071DF807709D
:109550007E401E54491C0429F1DB401CA042E2D38A
:10956000F8BD000010B5044639202FF023FBE0B20F
:109570002FF040FBC4F307202FF03CFBC4F307405F
:109580002FF038FB200E2FF035FB4FF480510348AD
:1095900001F0F0FA2DF094FC10BD00000004024030
:1095A0002DE9F04107460E4614463A202FF002FB03
:1095B000F0B22FF01FFB30122FF01CFB4FF4805144
:1095C0000F4801F0D7FA19E02DF07AFC05461D2D61
:1095D00011D1384600F0ACF805463B202FF0EAFAEE
:1095E0004FF48051064801F0C5FA2F4434B1208869
:1095F0002844208002E02846BDE8F081E4E700002E
:10960000000402402DE9F04107460E4614463C2076
:109610002FF0D0FAF0B22FF0EDFA30122FF0EAFA74
:109620004FF48051104801F0A5FA0CB100202080C1
:1096300019E02DF045FC05461E2D11D1384600F0ED
:109640002BF905463D202FF0B5FA4FF4805106481E
:1096500001F090FA2F4434B120882844208002E0A1
:109660002846BDE8F081E4E70004024010B529F087
:109670007FFA08B100F02EF8302000F0A9F810BDF4
:1096800010B504462146362000F08EF810BD10B506
:10969000044614B1204600F0ABF8342000F098F8EE
:1096A00010BD10B50446204600F0A2F820785C28D2
:1096B00002D020782F2803D10021642000F008F97F
:1096C000322000F085F810BD10B5682000F04CF88D
:1096D00010BD000010B522202FF06CFA2FF05FFAB9
:1096E00004464FF48051024801F044FA204610BD70
:1096F000000402402DE9F0412FF051FA04462FF00A
:109700004EFA05462FF04BFA06462FF048FA074668
:109710004FF48051054801F02DFA44EA052040EA53
:10972000064040EA0760BDE8F08100000004024006
:1097300070B5044627202FF03DFA2FF030FA064688
:10974000054646B100BF2FF02AFA2070641C701E37
:10975000C0B2061EF7D14FF48051024801F00AFA58
:10976000284670BD0004024010B504460C202FF0BE
:1097700021FA20462FF03EFAFFF7BCFF10BD000093
:1097800070B504460A202FF015FA20462FF032FA61
:109790002FF005FA05464FF48051024801F0EAF92E
:1097A000284670BD0004024070B505460C462846A8
:1097B0002FF000FA20462FF01DFA4FF48051034895
:1097C00001F0D8F92DF07CFB70BD000000040240D0
:1097D00010B5044620462FF0EDF94FF480510348B0
:1097E00001F0C8F92DF06CFB10BD00000004024030
:1097F0002DE9F041064601202FF0DCF92FF0CFF9DA
:1098000043282BDA2B20FFF7BBFF102826DA2F2066
:109810002FF0D0F900202FF0EDF93220FFF7D8FF1C
:109820000446142C1AD1CF20FFF7AAFF0446ACB18E
:109830004C20FFF799FF00EB042739464C2000F03D
:1098400047F85020FFF790FF00EB042739465020DF
:1098500000F03EF80021702000F03AF82F202FF0A1
:10986000A9F9357828462FF0C5F909E0761C357836
:109870005C2D01D02F2D00D1002528462FF0BAF9FC
:10988000002DF3D14FF48051024801F073F9BDE887
:10989000F08100000004024070B504462D202FF036
:1098A00089F92FF07CF90646054646B100BF2078BD
:1098B0002FF0A0F9641C701EC0B2061EF7D14FF441
:1098C0008051024801F056F9284670BD000402405C
:1098D00070B505460C460D202FF06CF928462FF088
:1098E00089F9E0B22FF086F9C4F307202FF082F94E
:1098F000C4F307402FF07EF9200E2FF07BF94FF4D0
:109900008051024801F036F970BD000000040240A9
:1099100070B502460C46FF25FF2309E012F8010B43
:1099200080EA05010648405C80EA03050548435C7F
:10993000201EA4F10106B4B2F0D145EA032070BDA7
:10994000DCE50308DCE603082DE9F04103460C469C
:1099500000200146024606E013F8010B411842F1CF
:109960000002601E84B2002CF6DC080C40EA024CB7
:10997000100C8DB21CEB050140F10002080C40EA0E
:10998000024041186FEA010080B2BDE8F08130B5B5
:1099900002460020002305E012F8015B2C18E0B21B
:1099A0005C1CE3B28B42F7DB30BD10B51EF038FB18
:1099B00010BD10B51EF0D2FA10BD10B51EF09EFA03
:1099C00010BD10B51EF0FAFA10BD10B520F08EFED5
:1099D00010BD10B528F006FC10BD00000246094B72
:1099E0009A4201D2084801E00648103801F00053BD
:1099F0001BB1064B0B40C36002E0044B0B4083607D
:109A00007047000010640240006002407D0F7D0F2F
:109A100021B1026842F00102026003E0026822F014
:109A20000102026070470000016821F0010101603D
:109A30000021016041608160C160016121214161BB
:109A40004A49884204D13D21484A103A91608CE04D
:109A500046491831884205D14FF47461434A103A9F
:109A6000916082E041493031884205D14FF4741150
:109A70003E4A103A916078E03C494831884205D12D
:109A80004FF07461394A103A91606EE037496031A5
:109A9000884204D13649354A103AD16065E03349ED
:109AA0007831884204D13349304A103AD1605CE0C1
:109AB0002E499031884204D12F492C4A103AD16066
:109AC00053E02A49A831884205D14FF03D51274A39
:109AD000103AD16049E02949884204D13D21274A02
:109AE000083A116041E025491831884205D14FF408
:109AF0007461224A083A116037E0204930318842C7
:109B000005D14FF474111D4A083A11602DE01B492C
:109B10004831884205D14FF07461184A083A116003
:109B200023E016496031884204D11149134A121FBB
:109B300011601AE011497831884204D10D490F4A69
:109B4000121F116011E00D499031884204D10A4979
:109B50000A4A121F116008E00849A831884204D15E
:109B60004FF03D51054A121F1160704710600240CE
:109B70003D000020400F002000003D201064024006
:109B800010B501F080034BB122B1436943F080036B
:109B9000436103E0436923F08003436180290BD0D4
:109BA0002AB1036801F01E042343036004E0036844
:109BB00001F01E04A343036010BD000010B5002295
:109BC0000268134B1A40CC680B6823434C6923434B
:109BD0008C692343CC6923430C6A23434C6A234397
:109BE0008C6A23434C6B23438C6B23431A430260E0
:109BF000426922F00702D1E90B3423431A43426140
:109C00000B6943604B6883608B68C36010BD0000C4
:109C10003F801CF01CB500240121202028F0B4FF57
:109C20003020009001208DF8040000208DF80600FF
:109C300003208DF8050000208DF8070069461748BD
:109C400000F022FF3021154800F094FF0021144855
:109C500080F8B41900201349887001204870C8703A
:109C60004FF4FA70886000F021F80F4890F80B0F5D
:109C7000592811DD24200A49F53948710820087156
:109C80003020C870142088702020487000210648B9
:109C900080F80B1F00F04EF81CBD000000140240BD
:109CA000BC320020703C0020BC2200201CB52EF0ED
:109CB00047FED0202EF010FE2EF076FE00202EF073
:109CC0000BFE2EF071FE2EF03BFED1202EF004FE96
:109CD0002EF06AFE00240EE0062C05DA01202EF09C
:109CE000CBFD0DF8040004E000202EF0C5FD0DF8BA
:109CF0000400601CC4B2072CEEDB2EF03BFE9DF886
:109D000006000A4948719DF8050008719DF8040095
:109D1000C8709DF8020088709DF8010048709DF899
:109D20000010034880F80B1F1CBD0000C731002045
:109D3000BC2200201CB500241B4890F80B0F8DF8A6
:109D400000001A4840788DF80100184880788DF896
:109D5000020001208DF803001448C0788DF804003B
:109D6000124800798DF80500104840798DF80600FA
:109D70002EF0E6FDD0202EF0AFFD2EF015FE0020D7
:109D80002EF0AAFD2EF010FE00BF07E01DF8040023
:109D90002EF0A2FD2EF008FE601CC4B2072CF5DBED
:109DA0002EF0E8FD1CBD0000BC220020C7310020C1
:109DB00070B502460C460025002309E012F8010B9D
:109DC00080EA05010648405C80EA03050548435CDB
:109DD000201EA4F10106B4B2F0D145EA032070BD03
:109DE000DCE50308DCE6030810B504460B46002159
:109DF000072A00DD072244EA042001462BB901FAB4
:109E000002F081B20912084610BD012B02D11141A6
:109E1000C8B2F9E700BFF7E710B528F0D9FC10BDCC
:109E200010B528F0D5FC10BD10B528F0D1FC10BD40
:109E30000149086070470000143C014001460020C1
:109E40000022074B1B6803EA0102054B14331B6811
:109E50000B4013B10AB1012000E000207047000060
:109E6000003C0140002123498279002A3AD00A4669
:109E7000126803689A430B461A600A1D1268036849
:109E80009A430B1D1A60027911440A6803681A4349
:109E90000A60184A0832126803689A43154B08335F
:109EA0001A601A1D126803689A43124B0C331A6029
:109EB0004279102A0ED11A1F126803681A430D4BFB
:109EC00008331A601A1D126803681A43094B0C33D1
:109ED0001A600DE00749427911440A6803681A4381
:109EE0000A6005E0027911440A6803689A430A602F
:109EF00070470000003C014010B504460B460021AD
:109F0000072A00DD072244EA0420014613B9114163
:109F1000C8B210BD012B05D101FA02F081B20912BD
:109F20000846F6E700BFF4E7F0B5ADF21C5D044665
:109F30000D460020CDF81805CDF81405002604EBD9
:109F40004400584901EBC000408AA84203DC0020CD
:109F50000DF21C5DF0BD0020CDF814059AE05148CB
:109F60000122C168504800F0A9FA4E4840680078C4
:109F70008DF800009DF8000038287DD104EB4400E6
:109F8000484B03EBC000C06804EB4403454F07EBAC
:109F9000C3031B8A03FB050104EB44003B4603EBB0
:109FA000C000028A404800F089FA0020CDF8180568
:109FB00012E004EB44003B4901EBC0004068BDF8EF
:109FC0001815405CBDF818250DF80200BDF81805FD
:109FD000401C80B2CDF8180504EB4400314901EB78
:109FE000C000008ABDF818158842E2DC04EB44008A
:109FF0002C4A02EBC000008A401E81B2684600F085
:10A0000023FB064604EB4400264901EBC000008A0E
:10A01000401E1DF80000B04233D10020CDF81805D5
:10A0200020E004EB44001F4901EBC0004068BDF88C
:10A030001815415C04EB44001A4A02EBC00080682A
:10A04000BDF81825024404EB4400164B03EBC00096
:10A05000008A401E68431154BDF81805401C80B2A8
:10A06000CDF8180504EB44000E4901EBC000008A4E
:10A07000401EBDF8181500E003E08842D1DC012045
:10A0800066E764202EF054FBBDF81405401C80B236
:10A09000CDF81405BDF814050628FFF660AF0020C2
:10A0A00056E70000C8960308208100202DE9F04102
:10A0B000ADF5A36D04460E4600250027A8460020F6
:10A0C000009004EB4400494901EBC000408AB042D3
:10A0D00004DC00200DF5A36DBDE8F0814448807BD1
:10A0E000002878D100210846FFF71EFF01287AD109
:10A0F000002520E004EB44003C4901EBC0008068EF
:10A10000411904EB4400394A02EBC000008A401EAA
:10A110007043085C04EB440102EBC10149684855F7
:10A1200004EB4400114601EBC0004068405D01A90A
:10A130004855681C85B204EB44002C4901EBC00073
:10A14000008AA842D6DC00274BE004EB4400274BF2
:10A1500003EBC000C06804EB4403DFF890C00CEBD5
:10A16000C3031B8A03FB060104EB4400634603EBB5
:10A17000C000008A401E82B21E4800F021FA04EBA3
:10A1800044001A4A02EBC000008A401E81B201A8B6
:10A1900000F05AFA009004EB4400144A02EBC000AD
:10A1A000C06804EB4402114B03EBC202128A104454
:10A1B00004EB440203EBC202128A02FB0600411EBA
:10A1C0000122684600F0FCF931462046FFF7ACFE5C
:10A1D000012801D17EE706E064202EF0A9FA781C60
:10A1E00087B2062FB1DB002074E70000C896030891
:10A1F000BC12002020810020F0B5ADF21C5D0025CE
:10A20000002400200190002600210120FFF78CFE91
:10A210004B4890F8FC6C00204A49088080E00025FB
:10A220006FE0002414E04748008800EB40004649F6
:10A2300051F83000005D4349098801EB4101424A71
:10A2400002EBC1014968085502A90855601C84B297
:10A250003C48008800EB40003B4901EBC000008A0D
:10A26000401EA042DFDC3748008800EB40000A4671
:10A2700002EBC000008A401E81B202A800F0E4F99F
:10A2800001903048008800EB40002F4B03EBC000EA
:10A29000C0682C4B1B8803EB43032B4F07EBC30316
:10A2A0001B8A03FB05012748008800EB40003B4662
:10A2B00003EBC000008A401E82B2244800F080F9FF
:10A2C0002048008800EB40003A4602EBC000C0681E
:10A2D0001C4A128802EB42023B4603EBC202128A7E
:10A2E0001044184A128802EB420203EBC202128A9F
:10A2F00002FB0500411E012201A800F061F9681C63
:10A3000085B21048008800EB40000F4901EBC00007
:10A31000408AA84285DC0B480088401C0949088017
:10A32000084800880D28FFF67AAF054880F8FC6CD5
:10A3300000210120FFF7BAFE0DF21C5DF0BD000008
:10A34000BC22002010000020C896030820810020B5
:10A350001CB50121084628F017FC01208DF80400E7
:10A3600002208DF8050000208DF8060001208DF8F0
:10A370000700182000906946144800F085FB05226C
:10A380001146124800F0C8FB052206210F4800F0D4
:10A39000C3FB052207210D4800F0BEFBA020009062
:10A3A00002208DF8040003208DF8050000208DF8B0
:10A3B00006008DF807006946044800F065FB402060
:10A3C00000906946014800F05FFB1CBD00000240A0
:10A3D0002DE9F84300240025002700200090804646
:10A3E000FFF7B6FF00F0BCF80A202EF0A1F96E4688
:10A3F00008212D4800F0BCFB10212B4800F0BAFBCF
:10A40000062000F091F80821274800F0B3FB08214E
:10A41000254800F0ADFB1021234800F0ABFB0120E4
:10A4200000F082F8002000F07FF808211E4800F0BC
:10A43000A1FB1E48D0F82C11B0F83021B0F8320141
:10A4400002FB0010B0F5003F02D900BE00BFFEE7DE
:10A450001748006808B9FFF7CFFE002015490880AB
:10A4600017E0002406E0134908782146FFF75CFD59
:10A47000601C84B20F48008800EB40000B4901EBE0
:10A48000C000408AA042EEDC0A480088401C09490E
:10A490000880084800880D28E3DB0748D0F80C0244
:10A4A0000549C873BDE8F88300000240C896030858
:10A4B0001C02434210000020BC1200202DE9F04194
:10A4C00005460C461646002701202DF0E6FE082121
:10A4D000144800F04DFB1021124800F04BFB032004
:10A4E00000F022F8C4F3074000F01EF8C4F3072080
:10A4F00000F01AF8E0B200F017F800BF06E0002004
:10A5000000F012F828706D1C781C87B2B742F6DB99
:10A510000821044800F02EFB00202DF0BEFEBDE80F
:10A52000F08100000000024010B5044600BF022187
:10A530000A4828F053FD0028F9D02146074828F0A2
:10A5400059FD00BF0121054828F048FD0028F9D039
:10A55000024828F04CFDC0B210BD000000300140A0
:10A5600000B585B00121080328F05EFB134828F0F0
:10A5700009FD0020ADF80000ADF80400ADF80600BC
:10A58000ADF808004FF40070ADF80A000820ADF8EF
:10A590000C000020ADF80E000720ADF810004FF4BD
:10A5A0008270ADF802006946044828F025FD0121BB
:10A5B000024828F0DBFC05B000BD0000003001407F
:10A5C0002DE9F04105460C461646002701202DF0E6
:10A5D00064FE08211B4800F0CBFA1021194800F056
:10A5E000C9FA0620FFF7A0FF0821164800F0C2FABA
:10A5F0000821144800F0BCFA1021124800F0BAFA01
:10A600000220FFF791FFC4F30740FFF78DFFC4F36B
:10A610000720FFF789FFE0B2FFF786FF00BF05E0E4
:10A620002878FFF781FF6D1C781C87B2B742F7DBF3
:10A630000821044800F09EFA00202DF02EFEBDE80F
:10A64000F08100000000024010B50246107803E0DF
:10A6500012F8014B2318D8B20B1EA1F10104A1B2CC
:10A66000F6D110BD2C48807F012854D100212A4802
:10A6700081772A480078C0B9012028490870284805
:10A680000068C0002749D1F8301240EA810025490E
:10A69000D1F82C1240EA41002249D1F8281208438F
:10A6A0000F2181432048017017E000201B490870EA
:10A6B0001B480068C0001B49D1F8301240EA8100F5
:10A6C0001849D1F82C1240EA41001649D1F8281255
:10A6D00008430F218143154801701348007813493E
:10A6E0000978884217D11048007811490870084647
:10A6F00000781049097888420DD00D480078064945
:10A7000008760B4800780B4908700948007810B1AA
:10A7100001200149C8757047BC120020DE0A0020E4
:10A720003402424200004242DF0A0020E00A0020D8
:10A73000E10A0020DD0A002010B5ADF57C7D002483
:10A740007DA00068FB9000200090FEF78FFF14288A
:10A750007CD17A48FEF7A5FF794908700846007851
:10A76000142874D1FEF7B0FF0021764A03C2BDF869
:10A770000000FEF7F7FE6A464FF4FA7101A8FEF7F3
:10A780000FFF71A101A82EF0B1F9714908800846A8
:10A79000008810B300BF04E000216E480155601C22
:10A7A00084B2282CF8DB01A9694A128888186AA1AA
:10A7B0002EF09CF969490880002409E0644800886B
:10A7C000C01C204401A9095C62480155601C84B288
:10A7D00062480088001FA042F0DC61A101A82EF0B1
:10A7E00085F95B4908800846008820B3002405E00D
:10A7F0000021584828300155601C84B2282CF7DB12
:10A8000001A9534A1288881853A12EF06FF95349B1
:10A81000088000240AE04E4800880830204401A93E
:10A82000095C4C4828300155601C84B24B480088B4
:10A830000938A042EFDC4DA101A82EF057F9444998
:10A8400008800846008830B3002407E06BE05BE036
:10A850000021404850300155601C84B2142CF7DBB5
:10A8600001A93B4A128888183BA12EF03FF93B49C9
:10A87000088000240AE0364800880C30204401A9F2
:10A88000095C344850300155601C84B2334800885C
:10A890000D38A042EFDC39A101A82EF027F92C4990
:10A8A00008800846008820B3002405E000202949DC
:10A8B00046390855601C84B2322CF7DB01A9244AC2
:10A8C0001288881824A12EF011F924490880002448
:10A8D0000AE01F480088801D204401A9085C1D492A
:10A8E00046390855601C84B21C480088C01FA0422D
:10A8F000EFDC00210320FFF7D9FB0120FEF7C0FEAB
:10A9000001200DF57C7D10BD0D480078422803D153
:10A910000A48FEF7BCFE0CE00120FEF7B1FE002065
:10A920000749087005E00021164880F80A1F2EF03C
:10A9300071F800BFE5E700000D0A0000480A00209A
:10A94000380A0020400A002041504E3D000000001F
:10A950005E0A0020503D00203B0000005C0A002001
:10A96000574946494E414D453D000000574946492B
:10A9700050415353574F52443D00000053455256E7
:10A9800045523D00BC22002010B5044635488442A3
:10A9900008D10121084628F007F90021012028F0FC
:10A9A00003F95EE03048844208D10121022028F0FA
:10A9B000FBF80021022028F0F7F852E02B488442EF
:10A9C00008D10121042028F0EFF80021042028F00C
:10A9D000EBF846E02648844208D10121082028F0FF
:10A9E000E3F80021082028F0DFF83AE0214884420B
:10A9F00008D10121102028F0D7F80021102028F0DC
:10AA0000D3F82EE01C48844208D10121202028F0F0
:10AA1000CBF80021202028F0C7F822E01748844214
:10AA200008D10121402028F0BFF80021402028F063
:10AA3000BBF816E01248844208D10121802028F09A
:10AA4000B3F80021802028F0AFF80AE00D488442D6
:10AA500007D10121801528F0A7F80021A01528F0C2
:10AA6000A3F810BD000002400004024000080240AC
:10AA7000000C024000100240001402400018024086
:10AA8000001C024000200240F0B50A4600210023CD
:10AA9000002400BF3DE0012505FA01F3156805EA31
:10AAA00003049C4234D105684F000326BE40B543E1
:10AAB000056015794E00B540066835430560157987
:10AAC000012D02D01579022D16D185684F0003267D
:10AAD000BE40B543856055794E00B5408668354324
:10AAE0008560456801268E40B54345604568967986
:10AAF0008E40B6B235434560C5684F000326BE4060
:10AB0000B543C560D5794E00B540C6683543C560CC
:10AB1000491C1029BFD3F0BDF0B5002300244D0718
:10AB2000ED0E02FA05F3CE1000F1200555F826507F
:10AB30004E07F70E0F26BE40B543CF1000F120069A
:10AB400046F82750CE1000F1200555F8265045EA6A
:10AB50000304CE1000F1200545F82640F0BD024662
:10AB6000002013690B400BB1012000E0002070476A
:10AB700041837047018370470249087E0021014AE2
:10AB800011767047BC1200200E48006800F00100EA
:10AB900000B100BE012080F3138800BF00BFBFF3E7
:10ABA0004F8F0848E438006800F4E0600649084325
:10ABB000001D0449E4390860BFF34F8F00BF00BF98
:10ABC000FEE70000F0ED00E00000FA054AF6AA20DA
:10ABD00001490860704700000030004030B502466F
:10ABE0000024002305E012F8015B2819C4B2581CA8
:10ABF000C3B28B42F7DB6042C0B230BD10B5002457
:10AC00002DF008FF64202DF093FD10BD2DE9F043D9
:10AC1000ADF2DC7D07460D46164698460024A14657
:10AC20008EA00068CDF8D80700200190042E7CDCAF
:10AC30008B480079302101EB101006EBC60101EBC7
:10AC40000611884A114408718548007900F00F0008
:10AC5000303006EBC60101EB061111444871804803
:10AC6000C078302101EB101006EBC60101EB061194
:10AC7000114488717A48C07800F00F00303006EB3C
:10AC8000C60101EB06111144C871FEF7EFFC142850
:10AC900071D175480078142809D006EBC60101EB84
:10ACA0000611704A8818FEF7FCFC6F4908706E4860
:10ACB0000078142872D1B5F57A7F01DD4FF47A75EA
:10ACC000FEF702FD0021694A03C268480068FEF7EA
:10ACD00049FC6348C078302101EB10108DF8080062
:10ACE0005F48C07800F00F0030308DF809005C48F4
:10ACF000807801EB10108DF80A005948807800F038
:10AD00000F0030308DF80B005548407801EB1010E3
:10AD10008DF80C005248407800F00F0030308DF86C
:10AD20000D00534890F80B0F00E093E001EB10107A
:10AD30008DF80E004E4890F80B0F00F00F003030E9
:10AD40008DF80F00B8F1020F16D13A208DF81000DF
:10AD5000002406E0395D02AA04F109001154601CC8
:10AD600084B2AC42F6DB05F1090081B201AA02A867
:10AD7000FEF748FC47E067E0B8F1000F03D154202C
:10AD80008DF8100005E0B8F1010F02D152208DF8C6
:10AD900010003A208DF81100002429E040E0204600
:10ADA00004EBD0714910795C4FEA21190A2099FB14
:10ADB000F0F0C0EBC00109F130000844C1B202AAB2
:10ADC00004F10A001154204604EBD0714910795C5B
:10ADD00001F00F090A2099FBF0F0C0EBC00109F166
:10ADE00030000844C1B204F10B001154A01C84B21D
:10ADF000B4EB450FD3DB0A2000EB450081B201AA7A
:10AE000002A8FEF7FFFB01AA02210DF5FB60FEF789
:10AE1000F9FB0120FEF734FC00201349087019E00B
:10AE200011480078422808D106EBC60101EB061153
:10AE30000C4A8818FEF72BFC0CE00120FEF720FCE2
:10AE400000200949087005E00021094880F80A1F20
:10AE50002DF0E0FD0DF2DC7DBDE8F0830D0A000071
:10AE6000C7310020600A0020380A0020400A002074
:10AE7000BC22002070B5BCB000213A9139913891C4
:10AE8000379136913591349133913291002230923D
:10AE900031922E922F922D912C912B912A912991C2
:10AEA0002891279126912591249123911591149110
:10AEB00013911291119110910F919FEDFE0A8DED5A
:10AEC0000E0AFDA006C8CDE90C12FDA006C8CDE90A
:10AED0000A12BAE0FC48807858B30020FA4988701A
:10AEE000FA48B0F8040EFA490968C1F57A71884247
:10AEF0001FD1F7480068C0F57A7081B2F348A0F816
:10AF0000FC1D0021F248001FFEF782FDF149F048C8
:10AF1000001FFEF763FD0120EF4908704FF47A71BE
:10AF2000EB488C38C0F88C100121E948001FFEF76F
:10AF30006FFDE548807B50B30021E3488173E7480B
:10AF40004088E3498C39496CC1F57A7188421ED139
:10AF5000DF488C38406CC0F57A70E0490839488089
:10AF60000021DB484C38FEF753FDDD49D8484C380A
:10AF7000FEF734FD0120DB4908704FF47A70D449A4
:10AF80008C3948640121D2484C38FEF741FDCE4847
:10AF9000807E50B30021CC488176D0488088CC494F
:10AFA0008C394969C1F57A7188421ED1C8488C38FC
:10AFB0004069C0F57A70C949083988800021C448C1
:10AFC0007C38FEF725FDC849C1487C38FEF706FDF0
:10AFD0000120C64908704FF47A71BD488C38416130
:10AFE0000121BB487C38FEF713FDB74890F82600D6
:10AFF00058B30021B44880F82610B848C088B44936
:10B000008C39C96AC1F57A7188421ED1B0488C3832
:10B01000C06AC0F57A70B1490839C8800021AC48CF
:10B020006438FEF7F5FCB249A9486438FEF7D6FC4F
:10B030000120B04908704FF47A70A5498C39C86274
:10B040000121A3486438FEF7E3FC9F488178807BA8
:10B0500001449D48807E01449B4890F826000844A6
:10B0600000287FF437AF13F0DBBF9B48007828B18E
:10B0700000209949087000212D9119E09948007825
:10B0800028B100209749087001212D9110E09748C0
:10B09000007828B100209549087002212D9107E021
:10B0A0009448007820B100209249087003212D9126
:10B0B0009DF8B41001EB4100C0EBC1108E4911F8AE
:10B0C0003000C12836D19DF8B41001EB4100C0EB2F
:10B0D000C110894901EBC000807808282AD10121DC
:10B0E0007A4880F8541E9DF8B40030B101280AD087
:10B0F00002280ED0032818D111E04FF480417F4878
:10B10000FFF736FD11E04FF400517C48FFF730FDAA
:10B110000BE04FF480517948FFF72AFD05E04FF42A
:10B1200000617648FFF724FD00BF00BF002074498E
:10B13000086098E764480C389DF8B41010F81110B6
:10B140000120B0EBD11F53F0D9856E4890F80A0F5B
:10B15000B8B1624908399DF8B40031F8101009916E
:10B160009DF8B40000EB4001C1EBC010624901EB57
:10B17000C001012308919DF8B420DDE90801FFF723
:10B1800045FD9DF8B41001EB410000EB01105E4954
:10B1900001EB001081792C919DF8B0000D2893F0FF
:10B1A0009285DFE810F0319A0D00D8177C2C993C7D
:10B1B000C93E3F43FB5154600F705E86329A6C9BD0
:10B1C0009DF8B41001EB4100C0EBC1104A4901EBFE
:10B1D000C00041780846099100211CF0ADFDC1B2C4
:10B1E0002891002136911CE09DF8B41001EB41003C
:10B1F00000EB0110444901EB00113031BDF8D800DB
:10B2000001EB001041789DF8A000814204D1BDF807
:10B21000D800C1B2289112E0BDF8D800401C81B21C
:10B2200036919DF8B41001EB410000EB0110364956
:10B2300001EB0010C179BDF8D8008142D4DC00BF19
:10B240009DF8B40000EB4001C1EBC0102A4901EBAE
:10B25000C000807800F0F000A0280DD19DF8B40067
:10B2600000EB4001C1EBC010234901EBC000807826
:10B2700000F00F0129910AE09DF8B41001EB4100A4
:10B28000C0EBC1101C4901EBC00081782991BDF8C9
:10B29000A40008B9102129919DF8B41001EB4100D8
:10B2A000C0EBC110144901EBC001BDF8A400401C63
:10B2B000095C2BE0000000000169323031303000C1
:10B2C000016932304530300058410020BC72002006
:10B2D0008C6002400088002012000020C080002006
:10B2E0000080201013000020208000101400002097
:10B2F0000088001015000020388F00200018024040
:10B3000088024242BC220020C84300202591BDF89B
:10B31000A400401C81B209919DF8B41001EB4100DA
:10B32000C0EBC111FE4800EBC1010891DDE9080145
:10B330001DF092F937909DF8B41001EB4100C0EB7D
:10B34000C110F74901EBC001BDF8A400801C095CE5
:10B35000BDF8DC00814242F0FC869DF8B41001EBA0
:10B360004100C0EBC110EE4901EBC000407800285D
:10B3700042F3EF869DF8B41001EB4100C0EBC11021
:10B38000E74901EBC001BDF8A400C01C0A5C9DF8B0
:10B39000B40040F2833110FB01F0E24901EB80017F
:10B3A00001F589619DF8A00000EB400303EB00105C
:10B3B00001EBC00080F844200021DB4A9DF8B40076
:10B3C00002EB00129DF8A0001154D84890F8280014
:10B3D000012840D19DF8B40000EB400101EB0010C2
:10B3E000D34901EB001030309DF8A01000EB0110A4
:10B3F000801C0990007820F0800080300999087046
:10B40000BDF89400B62814D0C52819D0D52802D08C
:10B41000D9281CD106E0BDF8A400032801DA0021D8
:10B42000259117E0BDF8A400032801DA0021259139
:10B4300010E0BDF8A400032801DA0021259109E0FD
:10B44000BDF8A400032801DA0021259102E00021C3
:10B45000259100BF00BFBDF89400C32801F0A78369
:10B460001EDCB32801F039840DDC112802F033858D
:10B47000122802F07885132802F01386B22842F0D1
:10B48000678601F07ABEB52801F03D84B62801F048
:10B490002A85B92801F0AF84BA28F0D101F0FCBBAD
:10B4A000D9287DD00BDCC52801F09E86CA2801F082
:10B4B000DD83CE2802F00F84D528E0D109E0E12811
:10B4C00002F01F84E52802F03284E728D7D102F089
:10B4D000E8BC9DF8B41001EB4100C0EBC1109049ED
:10B4E00001EBC000C178934880F8021D9DF8B410AC
:10B4F00040F2833011FB00F08A4901EB800101F535
:10B5000089619DF8A00000EB400202EB001011F8E9
:10B5100030109DF8B40040F2833210FB02F0814AF3
:10B5200002EB8000407981427EDA9DF8B41001EB95
:10B53000410000EB01107E4901EB001030309DF816
:10B54000A01000EB0110801C09907A4890F8020DC1
:10B550000121A1EBD0100999097860F30001099845
:10B560000170744890F8020DC0F34010F0BB9DF8D4
:10B57000B40000EB400101EB00106D4901EB00103D
:10B5800030309DF8A01000EB01108078C0F340101F
:10B5900060B39DF8B40000EB400101EB001000E047
:10B5A000ECE3634901EB001030309DF8A01000EB94
:10B5B0000110801C0990007820F00200801C09997D
:10B5C00008709DF8B41040F2833011FB00F0114672
:10B5D00001EB800000F589609DF8A01001EB4102AD
:10B5E00002EB011100EBC100183000E00BE0099004
:10B5F000007820F00200801C099908709DF8B410B2
:10B600000220FEF753FD00219DF8B40040F2833282
:10B6100010FB02F0434A02EB8000017102229DF808
:10B62000B40040F2833100E024E010FB01F03D491A
:10B6300001EB800101F589619DF8A00000EB40035A
:10B6400003EB001001F83020B6229DF8B40040F260
:10B65000833110FB01F0334901EB800000F5896074
:10B660009DF8A01001EB410303EB011100EBC100B9
:10B670004271FCE32F4890F8020DC0F3C000A8B956
:10B68000E5229DF8B40040F2833110FB01F025491A
:10B6900001EB800000F589609DF8A01001EB4103EB
:10B6A00003EB011100EBC1004271E2E79DF8B41019
:10B6B00001EB410000EB01101D4901EB001030309F
:10B6C0009DF8A01000EB0110801C0990194890F81B
:10B6D000020D0121A1EBD0120998007862F300005D
:10B6E000099908709DF8B41001EB410000EB0110BE
:10B6F0000F4901EB001030309DF8A01000EB011055
:10B70000801C09900B4890F8020D420909980078B6
:10B7100062F34100099908709DF8B4000CE0000044
:10B72000388F002088480020B8410020BC1200203B
:10B73000C8430020BC22002000EB400101EB0010B8
:10B74000FE4901EB001030309DF8A01000EB011015
:10B750008078C0F340029DF8B40040F2833110FBC2
:10B7600001F0F74901EB800000F589609DF8A01019
:10B7700001EB410303EB011100EBC100007EC0F3BC
:10B78000400082427BD09DF8B41040F2833011FB20
:10B7900000F0EB4901EB800000F589609DF8A010F6
:10B7A00001EB410202EB011100EBC10018300990DE
:10B7B0009DF8B40000EB400101EB0010DF4901EB04
:10B7C000001030309DF8A01000EB01108078420886
:10B7D0000998007862F34100099908709DF8B41047
:10B7E00001EB410000EB0110D44901EB00103030B7
:10B7F0009DF8A01000EB01108078C0F34000E8B382
:10B80000D9229DF8B40040F2833110FB01F0CC49FD
:10B8100001EB800000F589609DF8A01001EB410369
:10B8200003EB011100EBC1004271C64890F8100B08
:10B8300000287CD19DF8B41040F2833011FB00F059
:10B84000BF4901EB800000F589609DF8A01001EB75
:10B85000410202EB011100EBC10090F87F000028CB
:10B8600065D011239DF8B40040F2833110FB01F044
:10B87000B34901EB800101F5896101E06EE088E1E7
:10B880009DF8A00000EB400202EB001001EBC000AD
:10B8900090F8800040F2833110FB01F0A84901EBE1
:10B8A000800101F589619DF8B40040F2833210FBFC
:10B8B00002F0A34A02EB800202F589629DF8A00023
:10B8C00000EB400404EB001002EBC00090F8810094
:10B8D00000EB400202EB001001EBC00080F87E306C
:10B8E000F3239DF8B40040F2833110FB01F094493A
:10B8F00001EB800101F589619DF8A00000EB400299
:10B9000002EB001001EBC00090F8800040F28331A0
:10B9100010FB01F08A4901EB800101F589619DF876
:10B92000B40040F2833210FB02F0854A00E096E05A
:10B9300002EB800000F589609DF8A02002EB420434
:10B9400004EB021200EBC20090F8810000EB400211
:10B9500002EB001001EBC000437115E101229DF8DC
:10B96000B40040F2833110FB01F0754901EB800116
:10B9700001F589619DF8A00000EB400303EB001086
:10B9800001EBC0004273D9229DF8B40040F283312C
:10B9900010FB01F06A4901EB800101F589619DF816
:10B9A000A00000EB400303EB001001EBC00042716C
:10B9B00001229DF8B40040F2833110FB01F0604990
:10B9C00001EB800000F589609DF8A01001EB4103B8
:10B9D00003EB011100EBC10080F84620594890F8B4
:10B9E000100BE0BB9DF8B40040F2833110FB01F076
:10B9F000534901EB800000F589609DF8A01001EB30
:10BA0000410202EB011100EBC10090F87F0030B35E
:10BA10009DF8B41040F2833011FB00F0484901EB6F
:10BA2000800101F589619DF8A00000EB400202EB66
:10BA3000001001EBC00090F8801001EB410000EB1A
:10BA400001103E4901EB001130319DF8B40040F285
:10BA5000833210FB02F03A4A02EB800200E093E0EE
:10BA600002F589629DF8A00000EB400303EB001093
:10BA700002EBC00090F8810001EB0010801C0990DF
:10BA8000007820F004020998027000239DF8B400A9
:10BA900040F2833110FB01F0294901EB800000F5F1
:10BAA00089609DF8A01001EB410202EB011100EB4F
:10BAB000C10090F8800040F2833110FB01F0204972
:10BAC00001EB800000F589609DF8B41040F28332EC
:10BAD00011FB02F11A4A02EB810202F589629DF81C
:10BAE000A01001EB410404EB011102EBC10191F83C
:10BAF000811001EB410202EB011100EBC10080F863
:10BB00007E30F3239DF8B40040F2833110FB01F046
:10BB10000B4901EB800000F589609DF8A01001EB56
:10BB2000410202EB011100EBC10090F8800040F2ED
:10BB3000833110FB01F0024906E00000C8430020F9
:10BB400088480020BC32002001EB800000F58960AD
:10BB50009DF8B41040F2833211FB02F1FE4A02EB71
:10BB6000810101F589619DF8A02002EB420404EBFC
:10BB7000021201EBC20191F8811001EB410202EBCC
:10BB8000011100EBC10043719DF8B4100220FEF7D3
:10BB90008DFA9DF8B40000EB400101EB0010EF4975
:10BBA00001EB001130319DF8A00001EB001080780E
:10BBB00000F001029DF8B40040F2833110FB01F067
:10BBC000E54901EB800000F589609DF8A01001EBCC
:10BBD000410303EB011100EBC100007E00F0010006
:10BBE000824279D09DF8B40040F2833110FB01F01D
:10BBF000D94901EB800000F589609DF8A01001EBA8
:10BC0000410202EB011100EBC100183009909DF8D0
:10BC1000B40000EB400101EB0011D04800EB011033
:10BC200030309DF8A01000EB0110807809990A7857
:10BC300060F300020A709DF8B41001EB410000EBC4
:10BC40000110C64901EB001030309DF8A01000EB48
:10BC50000110807800F00100E8BB9DF8B41001EB02
:10BC6000410000EB0110BD4901EB001030309DF8A0
:10BC7000A01000EB01108078C0F3401068B39DF86D
:10BC8000B41040F2833011FB00F0B34901EB8000A7
:10BC900000F589609DF8A01001EB410202EB011153
:10BCA00000EBC10090F84600B8B99DF8B41040F21E
:10BCB000833011FB00F0A84901EB800000F589609A
:10BCC0009DF8A01001EB410202EB011100EBC10055
:10BCD000407B10B902E06DE0A6E24EE09DF8B410A2
:10BCE00001EB410000EB01109C4901EB00103030EA
:10BCF0009DF8A01000EB01108078C0F34000E0BB7D
:10BD000001229DF8B40040F2833110FB01F092490A
:10BD100001EB800101F589619DF8A00000EB400373
:10BD200003EB001001EBC0004273D9229DF8B40070
:10BD300040F2833110FB01F0874901EB800101F5EE
:10BD400089619DF8A00000EB400303EB001001EBBC
:10BD5000C000427101229DF8B40040F2833110FB13
:10BD600001F07D4901EB800000F589609DF8A0108D
:10BD700001EB410303EB011101E004E0FEE300EB02
:10BD8000C10080F8462000229DF8B40040F28331C3
:10BD900010FB01F0704901EB800000F589609DF80F
:10BDA000A01001EB410303EB011100EBC10080F88F
:10BDB000452034E29DF8B41040F2833011FB00F0CE
:10BDC000654901EB800000F589609DF8A01001EB4A
:10BDD000410202EB011100EBC10090F84600B0B93E
:10BDE00001229DF8B40040F2833110FB01F05A4962
:10BDF00001EB800000F589609DF8A01001EB410384
:10BE000003EB011100EBC10080F845202AE000227D
:10BE10009DF8B40040F2833110FB01F04E4901EB74
:10BE2000800101F589619DF8A00000EB400303EB60
:10BE3000001001EBC00080F845209DF8B41001EB24
:10BE4000410000EB0110454901EB001130319DF834
:10BE5000A00001EB0010801C0990007820F0010286
:10BE6000099802703E4890F8100B90B100E067E22C
:10BE70009DF8B41001EB410000EB0110374901EBD4
:10BE8000001030309DF8A01000EB0110807A0228DD
:10BE90008FD1344890F8290001288AD13148D0F850
:10BEA0000C023049498D88427DD29DF8B41040F291
:10BEB000833011FB00F0284901EB800000F5896018
:10BEC0009DF8A01001EB410202EB011100EBC10053
:10BED00090F84500012847D19DF8B40040F2833125
:10BEE00010FB01F01C4901EB800000F589609DF812
:10BEF000A01001EB410202EB011100EBC10090F830
:10BF00007F0088BB9DF8B40000EB400101EB0010FE
:10BF1000124901EB001130319DF8A00001EB001037
:10BF200001789DF8B40040F2833210FB02F00A4A17
:10BF300002EB80004170C3229DF8B40040F28331CF
:10BF400010FB01F0044901EB800101F589619DF8C6
:10BF5000A00000EB400308E088480020C843002010
:10BF6000BC320020BC12002074E003EB001001EB97
:10BF7000C000427100229DF8B40000EB400101EBCB
:10BF80000010FE4901EB001130319DF8A00001EBDB
:10BF90000010426001229DF8B40000EB400101EB6B
:10BFA0000010F64900E0EAE001EB001130319DF8A5
:10BFB000A00001EB0010C2729DF8B4100220FEF741
:10BFC00075F800213A911CE000229DF8B40040F27F
:10BFD000833110FB01F0EA4901EB800101F5896131
:10BFE0009DF8A00000EB400303EB001001EBC00143
:10BFF0004731BDF8E8000A54BDF8E800401C81B2A2
:10C000003A91BDF8E8000628DEDB00213A911CE0F9
:10C0100000229DF8B40040F2833110FB01F0D849B2
:10C0200001EB800101F589619DF8A00000EB400360
:10C0300003EB001001EBC0016331BDF8E8000A54C6
:10C04000BDF8E800401C81B23A91BDF8E8000F2825
:10C05000DEDBE4E09DF8B41040F2833011FB00F029
:10C06000C74901EB800000F589609DF8A01001EB45
:10C07000410202EB011100EBC10090F845000128DC
:10C080007DD19DF8B41040F2833011FB00F0BC4923
:10C0900001EB800101F589619DF8A00000EB4002F1
:10C0A00002EB001001EBC00090F8801040F28330EA
:10C0B00011FB00F0B24901EB800101F589619DF8A7
:10C0C000B40040F2833210FB02F0AD4A02EB800074
:10C0D00000F589609DF8A02002EB420303EB0212F9
:10C0E00000EBC20090F8810000EB400202EB001070
:10C0F00001EBC00090F87E00032840D100239DF89A
:10C10000B40040F2833110FB01F09D4901EB800146
:10C1100001F589619DF8A00000EB400202EB0010E0
:10C1200001EBC00090F8800040F2833110FB01F079
:10C13000934901EB800101F589619DF8B40040F25B
:10C14000833210FB02F08E4A02EB800202F5896214
:10C150009DF8A00000EB400404EB001002EBC000CF
:10C1600090F8810000EB400202EB001001EBC000F0
:10C1700080F87E309DF8B41001EB410000E04EE005
:10C1800000EB01107D4901EB001130319DF8A0005A
:10C1900001EB001001789DF8B40040F2833210FBEF
:10C1A00002F0774A02EB80004170C3229DF8B40090
:10C1B00040F2833110FB01F0714901EB800101F580
:10C1C00089619DF8A00000EB400303EB001001EB38
:10C1D000C000427100229DF8B40000EB400101EB69
:10C1E0000010664901EB001130319DF8A00001EB11
:10C1F0000010426002229DF8B40000EB400101EB08
:10C2000000105E4901EB001130319DF8A00001EBF8
:10C210000010C2729DF8B4100220FDF747FF9DF890
:10C22000B4100220FDF742FF9DF8B41001EB41006D
:10C2300000EB0110514901EB001030309DF8A010C7
:10C2400000EB01108078C0F3400050B39DF8B410AB
:10C2500040F2833011FB00F0494901EB800000F50A
:10C2600089609DF8A01001EB410202EB011100EB87
:10C27000C1004079D52814D1D9229DF8B40040F2EC
:10C28000833110FB01F03E4901EB800000F589602D
:10C290009DF8A01001EB410303EB011100EBC1007D
:10C2A00042719DF8B41040F2833011FB00F0344924
:10C2B00001EB800000F589609DF8A01001EB4102C0
:10C2C00002EB011100EBC1008078B22838D19DF853
:10C2D000B41001EB410000EB0110284901EB001004
:10C2E00030309DF8A01000EB01108078C0F34000C2
:10C2F00030BB9DF8B40000EB400101EB00101F497A
:10C3000001EB001030309DF8A01000EB0110807898
:10C31000C0F34010A0B9E5229DF8B40040F283318B
:10C3200010FB01F0164901EB800000F589609DF8D3
:10C33000A01001EB410303EB011100EBC1004271BE
:10C340009DF8B40040F2833110FB01F00C4901EB81
:10C35000800000F589609DF8A01001EB410202EB1E
:10C36000011100EBC100807B01283AD100229DF829
:10C37000B40040F2833110FB01F003E0C843002019
:10C3800088480020FC4901EB800101F589619DF896
:10C39000A00000EB400303EB001001EBC000827330
:10C3A000B6229DF8B40040F2833110FB01F0F2494F
:10C3B00001EB800101F589619DF8A00000EB4003CD
:10C3C00003EB001001EBC000427100219DF8B400A6
:10C3D00040F2833210FB02F0E74A02EB8000017169
:10C3E0004BE09DF8B40040F2833110FB01F0E249CC
:10C3F00001EB800000F589609DF8A01001EB41027F
:10C4000002EB011100EBC100407BB0BB9DF8B40012
:10C4100040F2833110FB01F0D74901EB800000F5B9
:10C4200089609DF8A01001EB410202EB011100EBC5
:10C43000C10090F8460001281FD1B6229DF8B40033
:10C4400040F2833110FB01F0CB4901EB800101F593
:10C4500089619DF8A00000EB400303EB001001EBA5
:10C46000C000427100219DF8B40040F2833210FBFD
:10C4700002F0C14A02EB800001719DF8B40000EBAC
:10C48000400101EB0010BD4901EB001030309DF878
:10C49000A01000EB011080780121B1EBD01F6ED10C
:10C4A0009DF8B40000EB400101EB0010B34901EB33
:10C4B000001030309DF8A01000EB0110807800F0E3
:10C4C000010000285BD19DF8B40040F2833110FBDD
:10C4D00001F0A94901EB800000F589609DF8A010EA
:10C4E00001EB410202EB011100EBC10090F84600A4
:10C4F000002844D19DF8B41001EB410000EB01107D
:10C500009E4901EB001030309DF8A01000EB0110A7
:10C510008078C0F3C00090BB9DF8B41001EB4100DF
:10C5200000EB0110954901EB001030309DF8A01090
:10C5300000EB0110407A00F0010000B39DF8B41048
:10C5400040F2833011FB00F08B4901EB800000F5D5
:10C5500089609DF8A01001EB410202EB011100EB94
:10C56000C10090F8900000F0010040B99DF8B410AF
:10C5700040F2833011FB00F07F4901E0B4E04AE073
:10C5800001EB800000F589609DF8A01001EB4102ED
:10C5900002EB011100EBC10090F88200D8B300213A
:10C5A0003A912CE09DF8B41040F2833011FB00F07A
:10C5B000714901EB800101F589619DF8A00000EB54
:10C5C000400202EB001001EBC00000F18301BDF856
:10C5D000E8000A5C9DF8B40000EB400101EB00109C
:10C5E000664901EB00100E30BDF8E810405C824255
:10C5F00000D008E0BDF8E800401C81B23A91BDF8D7
:10C60000E8000628CEDB00BFBDF8E800062869D1A7
:10C6100006213A912DE065E09DF8B41040F2833098
:10C6200011FB00F0544901EB800101F589619DF88F
:10C63000A00000EB400202EB001001EBC00000F193
:10C640008301BDF8E8000A5C9DF8B40000EB4001EE
:10C6500001EB0010494901EB00100E30BDF8E81065
:10C66000405C824200D008E0BDF8E800401C81B286
:10C670003A91BDF8E8000A28CEDB00BFBDF8E8001B
:10C680000A282FD09DF8B41040F2833011FB00F03F
:10C69000394901EB800000F589609DF8A01001EB9D
:10C6A000410202EB011100EBC100903009900078CB
:10C6B00020F00100401C0999087012229DF8B40076
:10C6C00040F2833110FB01F02B4901EB800000F5B3
:10C6D00089609DF8A01001EB410303EB011100EB11
:10C6E000C100427101F034BD9DF8B40000EB40017F
:10C6F00001EB0010214901EB0010007BD0BBBDF81D
:10C70000A400082800D0EDE700203A9028E09DF82A
:10C71000B40000EB4001C1EBC010194901EBC001AE
:10C72000BDF8E800C01C085C00F00F00092800DD1F
:10C730001AE09DF8B40000EB4001C1EBC0101049B5
:10C7400001EBC001BDF8E800C01C085C00F0F0007F
:10C75000902800DD08E0BDF8E800401C81B23A9165
:10C76000BDF8E8000628D2DB00BFBDF8E8000628C7
:10C7700008DAB7E775E0000088480020C8430020C9
:10C78000388F00209DF8B40000EB4001C1EBC010D1
:10C79000FE4901EBC000C07801049DF8B40000EB35
:10C7A0004002C2EBC010F94A02EBC000007941EA36
:10C7B00000219DF8B40000EB4002C2EBC010F34A28
:10C7C00002EBC000407901439DF8B40040F283328F
:10C7D00010FB02F0EE4A02EB800202F589629DF83E
:10C7E000A00000EB400303EB001002EBC000C0F818
:10C7F0001A109DF8B40000EB4001C1EBC010E349F2
:10C8000001EBC000807901049DF8B40000EB400208
:10C81000C2EBC010DD4A02EBC000C07941EA002142
:10C820009DF8B40000EB4002C2EBC010D74A02EB07
:10C83000C000007A01439DF8B40040F2833210FB3F
:10C8400002F0D34A02EB800000F589609DF8A02039
:10C8500002EB420303EB021200EBC200C0F81E1011
:10C86000C0E0BDF8A4000A2800D03BE700213A91BF
:10C8700028E09DF8B40000EB4001C1EBC010C349B3
:10C8800001EBC001BDF8E800C01C085C00F00F001F
:10C89000092800DD1AE09DF8B40000EB4001C1EB6F
:10C8A000C010BA4901EBC001BDF8E800C01C085C2B
:10C8B00000F0F000902800DD08E0BDF8E800401C22
:10C8C00081B23A91BDF8E8000828D2DB00BFBDF87C
:10C8D000E800082800DA05E79DF8B40000EB400105
:10C8E000C1EBC010A94901EBC000C07801069DF85A
:10C8F000B40000EB4002C2EBC010A44A02EBC0003F
:10C90000007941EA00419DF8B40000EB4002C2EB1F
:10C91000C0109E4A02EBC000407941EA00219DF818
:10C92000B40000EB4002C2EBC010984A02EBC0001A
:10C93000807901439DF8B40040F2833210FB02F08D
:10C94000934A02EB800202F589629DF8A00000EB99
:10C95000400303EB001002EBC000C0F81A109DF872
:10C96000B41001EB4100C0EBC110884901EBC000DD
:10C97000C07901069DF8B40000EB4002C2EBC01084
:10C98000824A02EBC000007A41EA00419DF8B400FF
:10C9900000EB4002C2EBC0107C4A02EBC000407AC0
:10C9A00041EA00219DF8B40000EB4002C2EBC01048
:10C9B000764A02EBC000807A01439DF8B40040F251
:10C9C000833210FB02F0724A02EB800000F58960AE
:10C9D0009DF8A02002EB420303EB021200EBC20021
:10C9E000C0F81E109DF8B41040F2833011FB00F027
:10C9F000674901EB800101F589619DF8A00000EB1A
:10CA0000400202EB001011F830109DF8B40040F223
:10CA1000833210FB02F05E4A02EB800040798142D3
:10CA200034DA00219DF8B40040F2833210FB02F0AA
:10CA3000574A02EB8000017104229DF8B40040F2D5
:10CA4000833110FB01F0524901EB800101F589614E
:10CA50009DF8A00000EB400303EB001001F830202C
:10CA6000C5229DF8B40040F2833110FB01F0484923
:10CA700001EB800000F589609DF8A01001EB4103F7
:10CA800003EB011100EBC10042718FE09DF8B4107F
:10CA900001EB410000EB01103E4901EB001030308A
:10CAA0009DF8A01000EB01108078C0F3400058B34F
:10CAB0009DF8B41040F2833011FB00F0344901EBD3
:10CAC000800000F589609DF8A01001EB410202EBA7
:10CAD000011100EBC1004079D92815D1D5229DF86C
:10CAE000B40040F2833110FB01F0294901EB8000D2
:10CAF00000F589609DF8A01001EB410303EB0111E3
:10CB000000EBC100427151E09DF8B41040F2833057
:10CB100011FB00F01E4901EB800000F589609DF8D3
:10CB2000A01001EB410202EB011100EBC100807B80
:10CB300001283BD100229DF8B40040F2833110FB64
:10CB400001F0134901EB800101F589619DF8A00016
:10CB500000EB400303EB001001EBC0008273B62230
:10CB60009DF8B40040F2833110FB01F0084901EB5D
:10CB7000800101F589619DF8A00000EB400303EB03
:10CB8000001001EBC0004271002105E0388F002049
:10CB900088480020C84300209DF8B40040F283324A
:10CBA00010FB02F0FE4A02EB800001719AE5D522EB
:10CBB0009DF8B40040F2833110FB01F0F84901EB1D
:10CBC000800101F589619DF8A00000EB400303EBB3
:10CBD000001001EBC000427101219DF8B40040F249
:10CBE000833210FB02F0EE4A02EB800001719DF8E7
:10CBF000B41001EB4100C0EBC110EA4901EBC000E9
:10CC0000C078592817D19DF8B41001EB410000EB12
:10CC10000110A2F5986101EB001030309DF8A010D2
:10CC200000EB0110801C0990007820F020002030DB
:10CC30000999087014E09DF8B41001EB410000EB75
:10CC40000110D94901EB001030309DF8A01000EB25
:10CC50000110801C0990007820F0200209980270D1
:10CC60009DF8B4100220FDF721FA3BE5D5229DF88E
:10CC7000B40040F2833110FB01F0C94901EB8000A0
:10CC800000F589609DF8A01001EB410303EB011151
:10CC900000EBC100427125E5D5229DF8B40040F2B9
:10CCA000833110FB01F0BE4901EB800101F5896180
:10CCB0009DF8A00000EB400303EB001001EBC00067
:10CCC000427101219DF8B40040F2833210FB02F062
:10CCD000B34A02EB8000017104E5D5229DF8B4004F
:10CCE00040F2833110FB01F0AD4901EB800000F50B
:10CCF00089609DF8A01001EB410303EB011100EBEB
:10CD0000C1004271EEE49DF8B41040F2833011FB93
:10CD100000F0A34901EB800000F58960BDF8D81050
:10CD200001EB410202EB011100EBC1008079012807
:10CD300040D100229DF8B40040F2833110FB01F095
:10CD4000974901EB800101F58961BDF8D80000EB3E
:10CD5000400303EB001001EBC0008271D5229DF867
:10CD6000B40040F2833110FB01F08D4901EB8001EA
:10CD700001F589619DF8A00000EB400303EB001072
:10CD800001EBC00042719DF8B41001EB410000EBD3
:10CD90000110854901EB001130319DF8A00001EB35
:10CDA0000010801C0990007820F00400001D0999F3
:10CDB00008701FE0C3229DF8B40040F2833110FBDD
:10CDC00001F0774901EB800101F589619DF8A00030
:10CDD00000EB400303EB001001EBC00042710021A7
:10CDE0009DF8B40040F2833210FB02F06C4A02EB73
:10CDF0008000017176E49DF8B41040F2833011FB9D
:10CE000000F0674901EB800000F58960BDF8D8109B
:10CE100001EB410202EB011100EBC1008079012816
:10CE200040D100229DF8B40040F2833110FB01F0A4
:10CE30005B4901EB800101F58961BDF8D80000EB89
:10CE4000400303EB001001EBC0008271D5229DF876
:10CE5000B40040F2833110FB01F0514901EB800135
:10CE600001F589619DF8A00000EB400303EB001081
:10CE700001EBC00042719DF8B41001EB410000EBE2
:10CE80000110494901EB001130319DF8A00001EB80
:10CE90000010801C0990007820F00400001D099902
:10CEA00008701FE0C3229DF8B40040F2833110FBEC
:10CEB00001F03B4901EB800101F589619DF8A0007B
:10CEC00000EB400303EB001001EBC00042710021B6
:10CED0009DF8B40040F2833210FB02F0304A02EBBE
:10CEE000800001710FE49DF8B41001EB410000EBEC
:10CEF00001102D4901EB0010007B50BB9DF8B400E0
:10CF000000EB4001C1EBC010264901EBC0000179E4
:10CF10009DF8B40000EB4002C2EBC010214A02EBC6
:10CF2000C000C07841EA00229DF8B40040F283318D
:10CF300010FB01F01A4901EB800000F589609DF8B3
:10CF4000A01001EB410303EB011100EBC1004263B0
:10CF50003CE09DF8B40000EB4001C1EBC01011496A
:10CF600001EBC000C07801049DF8B40000EB400262
:10CF7000C2EBC0100B4A02EBC000007941EA00216D
:10CF80009DF8B40000EB4002C2EBC010054A02EB72
:10CF9000C000407901439DF8B40040F2833205E0BF
:10CFA00088480020388F0020C843002010FB02F082
:10CFB000FE4A02EB800000F589609DF8A02002EB9C
:10CFC000420303EB021200EBC20041639DF8B40080
:10CFD00040F2833110FB01F0F44901EB800101F5CF
:10CFE00089619DF8A00000EB400202EB001011F8EF
:10CFF00030109DF8B40040F2833210FB02F0EB4A8F
:10D0000002EB80004079814234DA00219DF8B400BF
:10D0100040F2833210FB02F0E44A02EB800001711F
:10D0200003229DF8B40040F2833110FB01F0DF4988
:10D0300001EB800101F589619DF8A00000EB400340
:10D0400003EB001001F83020D9229DF8B40040F223
:10D05000833110FB01F0D54901EB800000F58960B8
:10D060009DF8A01001EB410303EB011100EBC1009F
:10D07000427181E09DF8B40040F2833110FB01F071
:10D08000CA4901EB800000F58960BDF8D81001EBBA
:10D09000410202EB011100EBC100807901284BD164
:10D0A00000229DF8B40040F2833110FB01F0BF492B
:10D0B00001EB800101F58961BDF8D80000EB400368
:10D0C00003EB001001EBC0008271D9229DF8B4007F
:10D0D00040F2833110FB01F0B44901EB800101F50E
:10D0E00089619DF8A00000EB400303EB001001EB09
:10D0F000C00042719DF8B41001EB410000EB01103B
:10D10000AB4901EB001030309DF8A01000EB01108E
:10D11000801C0990007820F00400001D0999087017
:10D1200001209DF8B41040F2833211FB02F19F4AB6
:10D1300002EB810108711FE0C5229DF8B40040F2A6
:10D14000833110FB01F0994901EB800101F5896100
:10D150009DF8A00000EB400303EB001001EBC000C2
:10D16000427100219DF8B40040F2833210FB02F0BE
:10D170008E4A02EB8000017118E500219DF8B40091
:10D1800040F2833210FB02F0884A02EB800001710A
:10D190009DF8B41001EB410000EB0110844901EB54
:10D1A000001130319DF8A00001EB0010801C0990A7
:10D1B000007820F00400001D09990870D5229DF820
:10D1C000B40040F2833110FB01F0784901EB80009C
:10D1D00000F589609DF8A01001EB410303EB0111FC
:10D1E00000EBC1004271E1E49DF8B41001EB410095
:10D1F00000EB01106E4901EB0010007BD0BBBDF8C5
:10D20000A4000C2800D0D1E400213A9128E09DF838
:10D21000B41001EB4100C0EBC110664901EBC00145
:10D22000BDF8E800C01C085C00F00F00092800DD14
:10D230001AE09DF8B41001EB4100C0EBC1105D494C
:10D2400001EBC001BDF8E800C01C085C00F0F00074
:10D25000902800DD08E0BDF8E800401C81B23A915A
:10D26000BDF8E8000A28D2DB00BFBDF8E8000A28B4
:10D2700001DA9BE482E000202E902F9000213A9169
:10D280001EE0DDE92E10000240EA11620902CDE93C
:10D290002E129DF8B41001EB4100C0EBC1104549BE
:10D2A00001EBC001BDF8E800C01C085CDDE92E34CC
:10D2B0001843CDE92E04BDF8E800401C80B23A9036
:10D2C000BDF8E8000528DCDB9DF8B400DDE92E217F
:10D2D00040F2833310FB03F0344B03EB800303F580
:10D2E00089639DF8A00000EB400404EB001003EB01
:10D2F000C00040F8222F416000222E922F92002180
:10D300003A911EE0DDE92E10000240EA11620902A6
:10D31000CDE92E129DF8B41001EB4100C0EBC11015
:10D32000244901EBC001BDF8E8000830085CDDE9E4
:10D330002E341843CDE92E04BDF8E800401C80B21D
:10D340003A90BDF8E8000528DCDB9DF8B400DDE983
:10D350002E1240F2833310FB03F0144B03EB8000DA
:10D3600000F589609DF8A03003EB430404EB031340
:10D3700000EBC30022308160C260C3E0BDF8A400AE
:10D380000E2800D012E400213A912FE09DF8B4104D
:10D3900001EB4100C0EBC110064901EBC001BDF833
:10D3A000E800C01C085C00F00F0005E08848002081
:10D3B000C8430020388F0020092800DD1AE09DF8BE
:10D3C000B41001EB4100C0EBC110FE4901EBC001FC
:10D3D000BDF8E800C01C085C00F0F000902800DDFB
:10D3E00008E0BDF8E800401C81B23A91BDF8E800C1
:10D3F0000C28CBDB00BFBDF8E8000C2800DA34E4D1
:10D4000000202E902F9000213A911EE0DDE92E1091
:10D41000000240EA11620902CDE92E129DF8B41013
:10D4200001EB4100C0EBC110E64901EBC001BDF8C2
:10D43000E800C01C085CDDE92E341843CDE92E0459
:10D44000BDF8E800401C80B23A90BDF8E80006281C
:10D45000DCDB9DF8B400DDE92E1240F2833310FBD3
:10D4600003F0D94B03EB800303F589639DF8A0001B
:10D4700000EB400404EB001003EBC00040F8221F57
:10D48000426000222E922F9200213A911EE0DDE9A7
:10D490002E10000240EA11620902CDE92E129DF819
:10D4A000B41001EB4100C0EBC110C64901EBC00153
:10D4B000BDF8E8000930085CDDE92E341843CDE9F9
:10D4C0002E04BDF8E800401C80B23A90BDF8E80098
:10D4D0000628DCDB9DF8B400DDE92E1240F2833330
:10D4E00010FB03F0B84B03EB800000F589609DF85A
:10D4F000A03003EB430404EB031300EBC300223022
:10D500008160C2609DF8B41040F2833011FB00F0DE
:10D51000AD4901EB800101F589619DF8A00000EBA8
:10D52000400202EB001011F830109DF8B40040F2F8
:10D53000833210FB02F0A44A02EB80004079814262
:10D540007ED19DF8B4009DF8A01001EB0010C21729
:10D55000CDE92E029D4890F8100B08B39DF8B41049
:10D5600001EB410000EB0110994901EB0010303054
:10D570009DF8A01000EB0110807A022810D09DF8D1
:10D58000B41001EB410000EB0110914901EB0010D8
:10D5900030309DF8A01000EB0110C07A00287DDD2E
:10D5A00000229DF8B40000EB400101EB0010884917
:10D5B00001EB001030309DF8A01000EB0110C2729A
:10D5C0008448D0F80C020521B0FBF1F201FB1200F7
:10D5D00000EB40017F482C3000EB41100D300990EA
:10D5E0009DF8B40040F2833110FB01F0764901EB65
:10D5F000800000F589609DF8A01001EB410202EB6C
:10D60000011100EBC1002230102201460890099858
:10D61000FAF71BFE6F48D0F80C020521B0FBF1F2BF
:10D6200001FB120000EB40016A482C3000EB411274
:10D630009DF8B40040F2833110FB01F0624900E034
:10D64000DFE201EB800101F589619DF8A00000EBAC
:10D65000400303EB001001EBC00050F81A1F42F822
:10D66000011F406850605B48D0F80C020521B0FBF8
:10D67000F1F201FB120000EB400156482C3000EBA8
:10D6800041129DF8B40000EB400101EB001050493D
:10D6900001EB001130319DF8A00000E096E101EBB4
:10D6A0000010007810704B48D0F80C020521B0FB38
:10D6B000F1F201FB120000EB400146482C3000EB78
:10D6C00041114248F538026841F81D2F8088888052
:10D6D0004048D0F80C020521B0FBF1F201FB12002A
:10D6E00000EB40013B482C3000EB41129DF8B400A8
:10D6F00040F2833110FB01F0334901EB800101F569
:10D7000089619DF8A00000EB400303EB001001EBE2
:10D71000C000406BC2F809002E48D0F80C02052169
:10D72000B0FBF1F201FB120000EB400129482C3064
:10D7300000EB41129DF8B40000EB400101EB00103A
:10D74000234901EB001130319DF8A00001EB0010DE
:10D750004068C2F8230000229DF8B40000EB4001AD
:10D7600001EB00101A4901EB001130319DF8A000C7
:10D7700001EB0010426000213A9160E01548D0F8BA
:10D780000C020521B0FBF1F201FB120000EB40019D
:10D7900010482C3000EB41112731BDF8E8409DF8CE
:10D7A000B40040F2833210FB02F0074A02EB800221
:10D7B00002F589629DF8A00000EB400303EB001026
:10D7C0000AE00000388F002088480020BC3200208A
:10D7D000C8430020BC12002002EBC00090F880007B
:10D7E00040F2833210FB02F0FE4A02EB800202F5A7
:10D7F00089629DF8B40040F2833310FB03F0F94BCB
:10D8000003EB800303F589639DF8A00000EB40055E
:10D8100005EB001003EBC00090F8810000EB400323
:10D8200003EB001002EBC0024732BDF8E800001D18
:10D83000105C0855BDF8E800401C81B23A91BDF873
:10D84000E80006289ADB00213A9142E000239DF887
:10D85000B40040F2833110FB01F0E24901EB80019A
:10D8600001F589619DF8A00000EB400202EB001079
:10D8700001EBC00090F8800040F2833110FB01F012
:10D88000D84901EB800101F589619DF8B40040F2AF
:10D89000833210FB02F0D34A02EB800202F5896268
:10D8A0009DF8A00000EB400404EB001002EBC00068
:10D8B00090F8810000EB400202EB001001EBC00188
:10D8C0004731BDF8E8000B54BDF8E800401C81B2B8
:10D8D0003A91BDF8E8000A28B8DBC348D0F80C023A
:10D8E0000521B0FBF1F080B2014609900220FBF760
:10D8F000EFFB00210620FCF7D9FBBB48D0F80C0257
:10D90000B949498D884206D2B748D0F80C02401C6C
:10D91000B549C1F80C0200210520FCF7C7FB9DF8B2
:10D92000B40000EB400101EB0010B04901EB001026
:10D9300030309DF8A01000EB0110801C0990007899
:10D9400020F00400001D09990870A748D0F80C02C7
:10D950000521B0FBF1F201FB120000EB4001A248EF
:10D960002C3000EB4110D0F823202E9800EB400122
:10D970009F4800EB4110C0F8232000203A9020E09F
:10D980009948D0F80C020521B0FBF1F201FB12001E
:10D9900000EB400194482C3000EB41102730BDF8DB
:10D9A000E810425C2E9800EB4001914800EB4111D9
:10D9B0002731BDF8E8000A54BDF8E800401C81B2E8
:10D9C0003A91BDF8E8000628DADB59E09DF8B4008A
:10D9D00000EB400101EB0010844901EB00103030F6
:10D9E0009DF8A01000EB0110801C0990007820F039
:10D9F00008000830099908709DF8B40000EB400158
:10DA000001EB0010794901EB001030309DF8A010B7
:10DA100000EB011042682E9800EB4001744800EBC7
:10DA20004110C0F8232000203A9025E09DF8B40072
:10DA300040F2833110FB01F06A4901EB800101F5EE
:10DA400089619DF8A00000EB400202EB001001EBA1
:10DA5000C0014731BDF8E8000A5C2E9800EB400198
:10DA6000634800EB41112731BDF8E8000A54BDF8C6
:10DA7000E800401C81B23A91BDF8E8000628D5DBE9
:10DA80009DF8B40000EB400101EB0010574901EB99
:10DA9000001030309DF8A01000EB0110801C0990A0
:10DAA000007820F02002099802709DF8B41002203E
:10DAB000FCF7FCFA9DF8B40040F2833110FB01F052
:10DAC000484901EB800000F589609DF8A01001EB4A
:10DAD000410202EB011100EBC100223009902E98A7
:10DAE00000EB4001424800EB41100D30102208903D
:10DAF0000999FAF7AAFB9DF8B40040F2833110FBB4
:10DB000001F0384901EB800101F589619DF8A00021
:10DB100000EB400202EB001001EBC0012E9800EB7D
:10DB20004002334800EB421051F81A2F40F8012F01
:10DB3000496841609DF8B40000EB400101EB001022
:10DB40002A4901EB001130319DF8A00001EB0010D3
:10DB500001782E9800EB4002254800EB421001703E
:10DB60002E9800EB4001224800EB41112148026849
:10DB700041F81D2F808888809DF8B41040F28330D2
:10DB800011FB00F0174901EB800101F589619DF857
:10DB9000A00000EB400202EB001001EBC000416B63
:10DBA0002E9800EB4002124800EB4210C0F809101A
:10DBB0002E9881B208200991FCF778FA00229DF88E
:10DBC000B40040F2833110FB01F0064901EB800004
:10DBD00000F589609DF8A01001EB410303EB0111F2
:10DBE0000AE0000088480020BC120020C843002042
:10DBF000D8140020C731002000EBC10080F8462077
:10DC000053E09DF8B41001EB410000EB0110FE4918
:10DC100001EB001030309DF8A01000EB0110801CCB
:10DC20000990007820F00400001D099908709DF803
:10DC3000B41001EB410000EB0110F34901EB0010BF
:10DC400030309DF8A01000EB0110801C0990007886
:10DC500020F0800080300999087001209DF8B410F0
:10DC600040F2833211FB02F1E84A02EB81010871B4
:10DC70009DF8B41040F2833011FB00F0114601EB27
:10DC8000800042799DF8B40040F2833110FB01F02E
:10DC9000DE4901EB800000F589609DF8A01001EBE2
:10DCA000410303EB011100F83120D5229DF8B400A7
:10DCB00040F2833110FB01F0D44901EB800000F504
:10DCC00089609DF8A01001EB410303EB011100EB0B
:10DCD000C10042713CE2D5229DF8B40040F283318C
:10DCE00010FB01F0C94901EB800000F589609DF847
:10DCF000A01001EB410303EB011100EBC1004271E5
:10DD000026E2D5229DF8B40040F2833110FB01F0E9
:10DD1000BE4901EB800000F589609DF8A01001EB81
:10DD2000410303EB011100EBC100427110E201213C
:10DD3000B74880F8341A9DF8B41040F2833011FBD4
:10DD400000F0B24901EB800101F589619DF8A00066
:10DD500000EB400202EB001011F830109DF8B40007
:10DD600040F2833210FB02F0A84A02EB80004079B7
:10DD7000814234DA00219DF8B40040F2833210FB76
:10DD800002F0A24A02EB8000017101229DF8B4006A
:10DD900040F2833110FB01F09C4901EB800101F559
:10DDA00089619DF8A00000EB400303EB001001F82F
:10DDB000302011229DF8B40040F2833110FB01F0B5
:10DDC000924901EB800000F589609DF8A01001EBFD
:10DDD000410303EB011100EBC100427160E09DF8CB
:10DDE000B41040F2833011FB00F0884901EB800051
:10DDF00000F589609DF8A01001EB410202EB0111D2
:10DE000000EBC1008078B22835D100219DF8B40024
:10DE100040F2833210FB02F07C4A02EB8000017179
:10DE2000B2229DF8B40040F2833110FB01F0774933
:10DE300001EB800101F589619DF8A00000EB400332
:10DE400003EB001001EBC000427100229DF8B4000A
:10DE500040F2833110FB01F06C4901EB800000F5CA
:10DE600089609DF8A01001EB410303EB011100EB69
:10DE7000C100827014E0D5229DF8B40040F28331D5
:10DE800010FB01F0614901EB800000F589609DF80D
:10DE9000A01001EB410303EB011100EBC100427143
:10DEA00056E100215A4880F8341AD5229DF8B40072
:10DEB00040F2833110FB01F0544901EB800000F582
:10DEC00089609DF8A01001EB410303EB011100EB09
:10DED000C10042713CE101229DF8B40040F283315F
:10DEE00010FB01F0494901EB800101F589619DF8C2
:10DEF000A00000EB400303EB001001EBC00080F832
:10DF0000822000213A9129E09DF8B41001EB4100F4
:10DF1000C0EBC1103F4901EBC001BDF8E800C01CD7
:10DF20000A5C9DF8B40040F2833110FB01F03749E0
:10DF300001EB800101F589619DF8A00000EB400331
:10DF400003EB001001EBC00000F18301BDF8E80015
:10DF50000A54BDF8E800401C81B23A91BDF8E800CF
:10DF60000A28D1DBF4E09DF8B40000EB4001C1EBDE
:10DF7000C010284901EBC000C07801049DF8B4002E
:10DF800000EB4002C2EBC010224A02EBC000007955
:10DF900041EA00209DF8B41001EB4102C2EBC1112F
:10DFA0001C4A02EBC10149790843B0F5E13F77D142
:10DFB0009DF8B40000EB400101EB0010124901EBA9
:10DFC000001030309DF8A01000EB0110801C09906B
:10DFD000007820F004020998027000229DF8B40035
:10DFE00040F2833110FB01F0084901EB800000F59D
:10DFF00089609DF8A01001EB410303EB011100EBD8
:10E00000C100A0F88E2007E0C84300208848002007
:10E01000BC320020388F002013229DF8B40040F25B
:10E02000833110FB01F0FE4901EB800000F58960AF
:10E030009DF8A01001EB410303EB011100EBC100BF
:10E0400042719DF8B40000EB400101EB0010F5496E
:10E0500001EB0010407903464FF480524FF4E13158
:10E0600009909DF8B4001AF009FB9DF8B40040F245
:10E07000833110FB01F0EA4901EB800101F5896170
:10E080009DF8A00000EB400202EB001001EBC00085
:10E0900090300990007820F0080008300999087045
:10E0A00056E09DF8B40000EB4001C1EBC010DE4922
:10E0B00001EBC00001799DF8B40000EB4002C2EB17
:10E0C000C010D94A02EBC000C07841EA00229DF896
:10E0D000B40040F2833110FB01F0D14901EB800123
:10E0E00001F589619DF8A00000EB400303EB0010EF
:10E0F00001EBC000A0F88E209DF8B40040F28331FF
:10E1000010FB01F0C64901EB800101F589619DF822
:10E11000A00000EB400202EB001001EBC000B0F8E1
:10E120008E109DF8B40000EB400202EB0010BD4AD7
:10E1300002EB0010408B814209DB0621A2F504723C
:10E140009DF8B40002EB00129DF8A000115400BF2E
:10E1500000BF10F0B8BD9DF8B40000EB4001C1EB6A
:10E16000C010B14911F83000042801D125900BE00E
:10E170009DF8B40000EB4001C1EBC010AA4911F8B2
:10E180003000152800D125909DF8B40000EB400127
:10E19000C1EBC010A44901EBC00041789DF8B40068
:10E1A00000EB4002C2EBC0109F4A12F8300041EA77
:10E1B000002041F23001884202D1A62025903DE0A6
:10E1C0009DF8B40000EB4001C1EBC010964901EB93
:10E1D000C00041789DF8B40000EB4002C2EBC010D3
:10E1E000914A12F8300041EA002041F231018842A0
:10E1F00002D1A720259021E09DF8B40000EB40015A
:10E20000C1EBC010884911F83000022816D19DF8E2
:10E21000B40000EB4001C1EBC010834901EBC0002A
:10E2200001799DF8B40000EB4002C2EBC0107E4AB9
:10E2300002EBC000C07841EA002125919DF8B400AE
:10E2400040F2833110FB01F0754901EB80008178C9
:10E2500028910021754A9DF8B40002EB00129DF848
:10E26000A0001154724890F82800012815D19DF89B
:10E27000B40000EB400101EB00106A4901EB001013
:10E2800030309DF8A01000EB0110801C0990007840
:10E2900020F08000803009990870BDF8941043F296
:10E2A0003002881A91427CD009DC04297AD01529E1
:10E2B00079D0A62910D0A72942F0EE8367E1B0F506
:10E2C000C06F71D0A0F2016000286ED001286DD01F
:10E2D0000428F1D101F04DBF00219DF8B40040F2B7
:10E2E000833210FB02F04E4A02EB800001719DF870
:10E2F000B40040F2833110FB01F0114601EB8000C5
:10E3000000F589609DF8A01001EB410202EB0111BC
:10E3100010F83100052829DC06229DF8B40040F2EF
:10E32000833110FB01F03E4901EB800101F5896169
:10E330009DF8A00000EB400303EB001001F8302033
:10E34000A8229DF8B40040F2833110FB01F034495B
:10E3500001EB800000F589609DF8A01001EB4103FE
:10E3600003EB011100EBC10042710EE19DF8B41006
:10E3700040F2833011FB00F0294901EB800000F5E9
:10E3800089609DF8A01001EB410202EB011110F829
:10E3900031000A2830DC0B229DF8B40040F28331B2
:10E3A00005E0BAE139E2F6E3F6E3F6E3F6E310FB63
:10E3B00001F01B4901EB800101F589619DF8A00086
:10E3C00000EB400303EB001001F83020A9229DF878
:10E3D000B40040F2833110FB01F0114901EB8000E1
:10E3E00000F589609DF8A01001EB410303EB0111DA
:10E3F00000EBC1004271C8E09DF8B41040F28330D8
:10E4000011FB00F0064901EB800000F589609DF8E2
:10E41000A01001EB410202EB011110F8310009E0FC
:10E4200088480020C8430020388F0020B8410020D1
:10E43000BC1200200F2829DC10229DF8B40040F205
:10E44000833110FB01F0FE4901EB800101F5896188
:10E450009DF8A00000EB400303EB001001F8302012
:10E46000A2229DF8B40040F2833110FB01F0F44980
:10E4700001EB800000F589609DF8A01001EB4103DD
:10E4800003EB011100EBC10042717EE09DF8B41076
:10E4900040F2833011FB00F0E94901EB800000F508
:10E4A00089609DF8A01001EB410202EB011100EB25
:10E4B000C1004079A52815D19DF8B41001EB4100A9
:10E4C00000EB0110DF4901EB001030309DF8A01087
:10E4D00000EB0110801C0990007820F00400001D62
:10E4E000099908709DF8B40040F2833110FB01F0E7
:10E4F000D34901EB800000F589609DF8A01001EB85
:10E50000410202EB011100EBC1008078A1283CD050
:10E510009DF8B40040F2833110FB01F0C84901EBD3
:10E52000800101F589619DF8A00000EB400202EB3B
:10E53000001001EBC00082789DF8B40040F28331F6
:10E5400010FB01F0BE4901EB800101F589619DF8E6
:10E55000A00000EB400303EB001001EBC000427190
:10E56000A1229DF8B40040F2833110FB01F0B449C0
:10E5700001EB800000F589609DF8A01001EB4103DC
:10E5800003EB011100EBC100827002F085BA00219B
:10E590009DF8B40040F2833210FB02F0A84A02EB6F
:10E5A000800001719DF8B40040F2833110FB01F04E
:10E5B000114601EB800000F589609DF8A01001EB89
:10E5C000410202EB011110F8310008281FDC002184
:10E5D0009DF8B40040F2833210FB02F0984A02EB3F
:10E5E0008000017108229DF8B40040F2833110FBD5
:10E5F00001F0934901EB800000F589609DF8A010BF
:10E6000001EB410303EB011100F8312028E09DF8F4
:10E61000B40040F2833110FB01F0894901EB800026
:10E6200000F589609DF8A01001EB410202EB011199
:10E6300010F831000B2813DC0C229DF8B40040F2D6
:10E64000833110FB01F07E4901EB800000F5896009
:10E650009DF8A01001EB410303EB011100F83120FC
:10E660009DF8B40040F2833110FB01F0744901EBD6
:10E67000800000F589609DF8A01001EB410202EBDB
:10E68000011100EBC1004079A42830D19DF8B400FD
:10E6900000EB400101EB00106A4901EB0010303043
:10E6A0009DF8A01000EB0110801C0990007820F06C
:10E6B000200020300999087000229DF8B40040F233
:10E6C000833110FB01F05E4901EB800000F58960A9
:10E6D0009DF8A01001EB410303EB011100EBC10019
:10E6E00080F845209DF8B4100220FBF7DFFCA12242
:10E6F0009DF8B40040F2833110FB01F0504901EB6A
:10E70000800000F589609DF8A01001EB410303EB48
:10E71000011100EBC100427137E700213A9115E089
:10E720009DF8B40000EB4001C1EBC010464901EB7D
:10E73000C001BDF8E800C01C095C16AABDF8E800DD
:10E740001154BDF8E800401C81B23A91BDF8E800D0
:10E750000628E5DB062116A82AF02EF80021CDE9CF
:10E760003001DDE93021100A40EA0164309BE218F3
:10E7700041EB2120CDE908204FF480724FF00003D7
:10E78000DDE90801F9F71EFD9DF8B40040F2833180
:10E7900010FB01F02A4901EB800000F589609DF82B
:10E7A000A01001EB410303EB011100EBC10002716A
:10E7B00000209DF8B41040F2833211FB02F1204A90
:10E7C00002EB8101087104229DF8B40040F283310C
:10E7D00010FB01F01A4901EB800000F589609DF8FB
:10E7E000A01001EB410303EB011100F83120A72237
:10E7F0009DF8B40040F2833110FB01F0104901EBA9
:10E80000800000F589609DF8A01001EB410303EB47
:10E81000011100EBC1004271B7E69DF8B40040F26F
:10E82000833110FB01F0064901EB800000F589609F
:10E830009DF8A01001EB410202EB011106E000007F
:10E8400088480020C8430020388F002010F831008D
:10E85000042878DA00219DF8B40040F2833210FBDE
:10E8600002F0FE4A02EB80000171A1229DF8B40083
:10E8700040F2833110FB01F0F84901EB800101F512
:10E8800089619DF8A00000EB400303EB001001EB51
:10E89000C00042719DF8B40040F2833110FB01F0DA
:10E8A000EE4901EB800101F589619DF8A00000EBC4
:10E8B000400202EB001001EBC00109910878401CF6
:10E8C000C1B2099801709DF8B40040F2833110FB89
:10E8D00001F0E24901EB800000F589609DF8A0108D
:10E8E00001EB410202EB011110F83100042828D19C
:10E8F0000A229DF8B40040F2833110FB01F0D749A1
:10E9000001EB800101F589619DF8A00000EB400357
:10E9100003EB001001F83020A3229DF8B40040F270
:10E92000833110FB01F0CD4901EB800000F58960D7
:10E930009DF8A01001EB410303EB011100EBC100B6
:10E94000427132E3FFE79DF8B40040F2833110FBDF
:10E9500001F0C24901EB800000F589609DF8A0102C
:10E9600001EB410202EB011110F83100042834D10F
:10E9700000219DF8B40040F2833210FB02F0B74A48
:10E9800002EB8000017105229DF8B40040F2833152
:10E9900010FB01F0B14901EB800101F589619DF89F
:10E9A000A00000EB400303EB001001F83020A3228D
:10E9B0009DF8B40040F2833110FB01F0A74901EB50
:10E9C000800000F589609DF8A01001EB410303EB86
:10E9D000011100EBC1004271E7E29DF8B40040F282
:10E9E000833110FB01F09D4901EB800000F5896047
:10E9F0009DF8A01001EB410202EB011110F831006B
:10EA0000082834DC00219DF8B40040F2833210FB6A
:10EA100002F0924A02EB8000017109229DF8B400D5
:10EA200040F2833110FB01F08C4901EB800101F5CC
:10EA300089619DF8A00000EB400303EB001001F892
:10EA40003020A7229DF8B40040F2833110FB01F082
:10EA5000824901EB800000F589609DF8A01001EB70
:10EA6000410303EB011100EBC10042719DE29DF8EF
:10EA7000B41040F2833011FB00F0784901EB8000C4
:10EA800000F589609DF8A01001EB410202EB011135
:10EA900010F83100092834DC00219DF8B40040F260
:10EAA000833210FB02F06D4A02EB800001710A22F2
:10EAB0009DF8B40040F2833110FB01F0674901EB8F
:10EAC000800101F589619DF8A00000EB400303EB94
:10EAD000001001F83020A3229DF8B40040F28331E9
:10EAE00010FB01F05D4901EB800000F589609DF8A5
:10EAF000A01001EB410303EB011100EBC1004271D7
:10EB000053E29DF8B41040F2833011FB00F05349FA
:10EB100001EB800000F589609DF8A01001EB410237
:10EB200002EB011110F831000D2838DC00219DF8AE
:10EB3000B40040F2833210FB02F0484A02EB80003E
:10EB400001710E229DF8B40040F2833110FB01F0F8
:10EB5000424901EB800101F589619DF8A00000EBBD
:10EB6000400303EB001001F83020A1229DF8B4000F
:10EB700040F2833110FB01F0384901EB800000F5D1
:10EB800089609DF8A01001EB410303EB011100EB3C
:10EB9000C100427109E209E23DE298E276E29DF8A5
:10EBA000B41040F2833011FB00F02C4901EB8000DF
:10EBB00000F589609DF8A01001EB410202EB011104
:10EBC00010F831000E2834DC00219DF8B40040F22A
:10EBD000833210FB02F0214A02EB800001710F2208
:10EBE0009DF8B40040F2833110FB01F01B4901EBAA
:10EBF000800101F589619DF8A00000EB400303EB63
:10EC0000001001F83020A3229DF8B40040F28331B7
:10EC100010FB01F0114901EB800000F589609DF8BF
:10EC2000A01001EB410303EB011100EBC1004271A5
:10EC3000BBE19DF8B41040F2833011FB00F00749AE
:10EC400001EB800000F589609DF8A01001EB410206
:10EC500002EB011110F83100102801E08848002073
:10EC60007DDC11229DF8B40040F2833110FB01F0ED
:10EC7000FE4901EB800101F589619DF8A00000EBE0
:10EC8000400303EB001001F83020A1229DF8B400EE
:10EC900040F2833110FB01F0F44901EB800101F5F2
:10ECA00089619DF8A00000EB400303EB001001EB2D
:10ECB000C00042719DF8B40040F2833110FB01F0B6
:10ECC000EA4901EB800101F589619DF8A00000EBA4
:10ECD000400303EB001001EBC00082709DF8B410FC
:10ECE00001EB410000EB0110E14901EB0011303173
:10ECF0009DF8A00001EB0010801C0990007820F026
:10ED000080008030099908709DF8B41001EB410033
:10ED100000EB0110D64901EB001030309DF8A01037
:10ED200000EB0110801C0990007820F00400001D09
:10ED3000099908709DF8B41001EB410000EB011037
:10ED4000CB4901EB001030309DF8A01000EB011012
:10ED50008078C0F34010E8B39DF8B41000E042E0C2
:10ED600001EB410000EB0110C14901EB0010303014
:10ED70009DF8A01000EB0110801C0990007820F095
:10ED80002002099802709DF8B41001EB410000EBDD
:10ED90000110B74901EB001030309DF8A01000EBD6
:10EDA00001108078C0F34000B8B99DF8B41001EBB1
:10EDB000410000EB0110AE4901EB001030309DF82E
:10EDC000A01000EB0110801C0990007820F00800D2
:10EDD000083000E072E0099908709DF8B410022034
:10EDE000FBF764F9E1E09DF8B41040F2833011FBC9
:10EDF00000F09E4901EB800101F589619DF8A000BA
:10EE000000EB400202EB001011F830109DF8B40046
:10EE100040F2833210FB02F0944A02EB800040790A
:10EE200081424BD19DF8B41040F2833011FB00F0C9
:10EE3000114601EB800000F589609DF8A01001EB00
:10EE4000410202EB011100EBC1008078A12836D00D
:10EE5000A3229DF8B40040F2833110FB01F08349F6
:10EE600001EB800101F589619DF8A00000EB4003F2
:10EE700003EB001001EBC00042719DF8B41040F2AA
:10EE8000833011FB00F0794901EB800000F58960C7
:10EE90009DF8A01001EB410202EB011100EBC10053
:10EEA0008078A2280AD000209DF8B41040F2833266
:10EEB00011FB02F16D4A02EB8101087175E09DF8CA
:10EEC000B41040F2833011FB00F0684901EB800080
:10EED00000F589609DF8A01001EB410202EB0111E1
:10EEE00000EBC100807B01283FD100229DF8B400D7
:10EEF00040F2833110FB01F05C4901EB800101F528
:10EF000089619DF8A00000EB400303EB001001EBCA
:10EF1000C0008273A3229DF8B40040F2833110FB3D
:10EF200001F0524901EB800101F589619DF8A000D3
:10EF300000EB400303EB001001EBC0004271A9227B
:10EF40009DF8B40040F2833110FB01F0474901EB1A
:10EF5000800000F589609DF8A01001EB410303EBF0
:10EF6000011100EBC10082701FE0A1229DF8B400E6
:10EF700040F2833110FB01F03C4901EB800101F5C7
:10EF800089619DF8A00000EB400303EB001001EB4A
:10EF9000C000427101219DF8B40040F2833210FBA1
:10EFA00002F0324A02EB8000017135E4A1229DF8A3
:10EFB000B40040F2833110FB01F02C4901EB8001D9
:10EFC00001F589619DF8A00000EB400303EB001000
:10EFD00001EBC00082709DF8B40040F2833110FB59
:10EFE00001F0224901EB800101F589619DF8A00043
:10EFF00000EB400303EB001001EBC0004271002165
:10F000009DF8B40040F2833210FB02F0174A02EB85
:10F0100080000171C9E700219DF8B40040F28332FD
:10F0200010FB02F0114A02EB8000017109229DF8E9
:10F03000B40040F2833110FB01F00C4901EB800178
:10F0400001F589619DF8A00000EB400303EB00107F
:10F0500001F83020A7229DF8B40040F2833110FB64
:10F0600001F0024901EB800004E000008848002024
:10F07000C843002000F589609DF8A01001EB410312
:10F0800003EB011100EBC10042718EE700219DF8F6
:10F09000B40040F2833210FB02F0FE4A02EB800023
:10F0A0000171A7229DF8B40040F2833110FB01F0FA
:10F0B000F84901EB800000F589609DF8A01001EB94
:10F0C000410303EB011100EBC10042716DE7002128
:10F0D0009DF8B40040F2833210FB02F0ED4A02EBDF
:10F0E00080000171A7229DF8B40040F2833110FB2B
:10F0F00001F0E84901EB800101F589619DF8A0006C
:10F1000000EB400303EB001001EBC00042719DF8DF
:10F11000B40000EB4001C1EBC010DF4901EBC000BF
:10F12000407930287ED19DF8B40040F2833110FB45
:10F1300001F0D84901EB800101F589619DF8A0003B
:10F1400000EB400202EB001011F830109DF8B40003
:10F1500040F2833210FB02F0CE4A02EB800040798D
:10F1600081425FD19DF8B40040F2833110FB01F081
:10F17000114601EB800000F589609DF8A01001EBBD
:10F18000410202EB011100EBC100C078312830D1FF
:10F190009DF8B40000EB400101EB0010BF4901EB0A
:10F1A000001030309DF8A01000EB0110801C099079
:10F1B000007820F020020998027000229DF8B40027
:10F1C00040F2833110FB01F0B24901EB800000F501
:10F1D00089609DF8A01001EB410303EB011100EBE6
:10F1E000C10080F845209DF8B4100220FAF75EFFB8
:10F1F00081E09DF8B40040F2833110FB01F0A54995
:10F2000001EB800000F589609DF8A01001EB410240
:10F2100002EB011100EBC100C07833286BD19DF8DF
:10F22000B40000E092E000EB400101EB00109B49CC
:10F2300001EB001030309DF8A01000EB0110801C95
:10F240000990007820F020020998027001229DF8B0
:10F25000B40040F2833110FB01F08E4901EB8000D5
:10F2600000F589609DF8A01001EB410303EB01114B
:10F2700000EBC10080F846209DF8B40040F28331D5
:10F2800010FB01F0834901EB800000F589609DF8D7
:10F29000A01001EB410303EB011100EBC10042732D
:10F2A00041F288329DF8B40040F2833110FB01F046
:10F2B000784901EB800000F589609DF8A01001EB12
:10F2C000410303EB011100EBC1004261A9229DF84B
:10F2D000B40040F2833110FB01F06E4901EB800075
:10F2E00000F589609DF8A01001EB410303EB0111CB
:10F2F00000EBC10082709DF8B41001EB410000EBFF
:10F300000110664901EB001030309DF8A01000EBB1
:10F310000110801C0990007820F001020998027009
:10F320009DF8B41001EB410000EB01105B4901EBCB
:10F33000001030309DF8A01000EB0110801C0990E7
:10F34000007820F002020998027017E19DF8B410CD
:10F3500001EB4100C0EBC1104F4901EBC000407907
:10F3600031287CD19DF8B41040F2833011FB00F0BD
:10F37000484901EB800101F589619DF8A00000EB8F
:10F38000400202EB001011F830109DF8B40040F27A
:10F39000833210FB02F03F4A02EB80004079814249
:10F3A0005DD19DF8B41040F2833011FB00F011469E
:10F3B00001EB800000F589609DF8A01001EB41028F
:10F3C00002EB011100EBC10090F8460058BB01228E
:10F3D0009DF8B40040F2833110FB01F02D4901EBA0
:10F3E000800101F589619DF8A00000EB400303EB6B
:10F3F000001001EBC00080F845209DF8B40000EB40
:10F40000400101EB0010254901EB001130319DF85E
:10F41000A00001EB0010801C0990007820F0010092
:10F42000401C099908709DF8B40000EB400101EB05
:10F4300000101A4901EB001030309DF8A01000EBCD
:10F440000110801C0990007820F0020209980270D7
:10F45000134890F8100B90B19DF8B40000E007E25B
:10F4600000EB400101EB00100C4901EB00103030C3
:10F470009DF8A01000EB0110807A02287ED1094887
:10F4800090F829000128F9D10648D0F80C02054966
:10F49000498D09E088480020388F0020C8430020AB
:10F4A000BC320020BC120020884267D29DF8B40014
:10F4B00040F2833110FB01F0FE4901EB800000F5C2
:10F4C00089609DF8A01001EB410202EB011100EBF5
:10F4D000C10090F84500012851D19DF8B40040F2D8
:10F4E000833110FB01F0F34901EB800000F58960E6
:10F4F0009DF8A01001EB410202EB011100EBC100ED
:10F5000090F87F00D8BB01229DF8B40000EB4001C9
:10F5100001EB0010E84901EB001130319DF8A0002B
:10F5200001EB0010C27200229DF8B40000EB400114
:10F5300001EB0010E04901EB001130319DF8A00013
:10F5400001EB001042604FF010429DF8B40040F211
:10F55000833110FB01F0D74901EB800101F589618E
:10F560009DF8A00000EB400303EB001001EBC0008E
:10F5700082609DF8B40000EB400101E073E073E0AD
:10F5800001EB0010CC4901EB001130319DF8A000D7
:10F5900001EB001001789DF8B40040F2833210FBBB
:10F5A00002F0C44A02EB800041709DF8B40040F2C2
:10F5B000833110FB01F0114601EB800101F58961F7
:10F5C0009DF8A00000EB400202EB001011F8301093
:10F5D0009DF8B40040F2833210FB02F0B54A02EB12
:10F5E0008000407981423ED100229DF8B40040F273
:10F5F000833110FB01F0AF4901EB800101F5896116
:10F600009DF8A00000EB400303EB001001EBC000ED
:10F61000C271A4229DF8B40040F2833110FB01F0C6
:10F62000A44901EB800101F589619DF8A00000EB80
:10F63000400303EB001001EBC0008270A3229DF891
:10F64000B40040F2833110FB01F09A4901EB8000D5
:10F6500000F589609DF8A01001EB410303EB011157
:10F6600000EBC100427179E29DF8B40040F28331B1
:10F6700010FB01F08F4901EB800000F589609DF8D7
:10F68000A01001EB410202EB011100EBC10090F868
:10F69000450001287ED19DF8B40040F2833110FB73
:10F6A00001F0844901EB800101F589619DF8A0001A
:10F6B00000EB400202EB001001EBC00090F880006C
:10F6C00040F2833110FB01F07A4901EB800101F532
:10F6D00089619DF8B40040F2833210FB02F0754A54
:10F6E00002EB800000F589609DF8A02002EB420348
:10F6F00003EB021200EBC20090F8810000EB400225
:10F7000002EB001001EBC00090F87E00032841D10D
:10F7100002229DF8B40000EB400101EB00106649A5
:10F7200001EB001130319DF8A00001EB0010C27216
:10F730004FF010429DF8B40040F2833110FB01F00D
:10F740005C4901EB800101F589619DF8A00000EBA7
:10F75000400303EB001001EBC00082609DF8B40091
:10F7600000EB400101EB0010534901EB0011303177
:10F770009DF8A00001EB001001789DF8B40040F264
:10F78000833210FB02F04B4A02EB800041709DF87F
:10F79000B40000E0ABE140F2833110FB01F0114610
:10F7A00001EB800101F589619DF8A00000EB4002AA
:10F7B00002EB001011F830109DF8B40040F28332D3
:10F7C00010FB02F03B4A02EB8000407981423ED1BF
:10F7D00000229DF8B40040F2833110FB01F035495E
:10F7E00001EB800101F589619DF8A00000EB400369
:10F7F00003EB001001EBC000C271A4229DF8B4001D
:10F8000040F2833110FB01F02A4901EB800101F540
:10F8100089619DF8A00000EB400303EB001001EBB1
:10F82000C0008270A3229DF8B40040F2833110FB27
:10F8300001F0204901EB800000F589609DF8A010DF
:10F8400001EB410303EB011100EBC1004271002207
:10F850009DF8B40000EB400101EB0010164901EBEC
:10F86000001030309DF8A01000EB0110426075E1EF
:10F870009DF8B40000EB4001C1EBC0100F4901EB53
:10F88000C000407933287DD19DF8B40000EB4001E1
:10F8900001EB0010084901EB001030309DF8A0107A
:10F8A00000EB0110801C0990007820F00100401C42
:10F8B000099905E088480020C8430020388F0020BF
:10F8C00008709DF8B40000EB400101EB0010FE4908
:10F8D00001EB001030309DF8A01000EB0110801CEF
:10F8E0000990007820F02002099802709DF8B40079
:10F8F00000EB400101EB0010F34901EB0010303048
:10F900009DF8A01000EB0110801C0990007820F0F9
:10F910000200801C099908709DF8B40040F2833100
:10F9200010FB01F0E94901EB800042799DF8B40039
:10F9300040F2833110FB01F0E44901EB800000F557
:10F9400089609DF8A01001EB410303EB011100F861
:10F9500031209DF8B40000EB400101EB0010DA49C2
:10F9600001EB001030309DF8A01000EB0110801C5E
:10F970000990007820F080008030099908709DF887
:10F98000B40000E02AE000EB400101EB0010CE499A
:10F9900001EB001030309DF8A01000EB01108078D2
:10F9A000C0F3400020B99DF8B4100220FAF77EFBA6
:10F9B000A2229DF8B40040F2833110FB01F0C3494C
:10F9C00001EB800000F589609DF8A01001EB410378
:10F9D00003EB011100EBC1008270BFE09DF8B400A1
:10F9E00000EB4001C1EBC010B94901EBC000407908
:10F9F00034287CD19DF8B40000EB400101EB0010ED
:10FA0000B14901EB001030309DF8A01000EB01105F
:10FA1000801C0990007820F02002099802709DF85F
:10FA2000B40000EB400101EB0010A74901EB00100E
:10FA300030309DF8A01000EB0110801C0990007878
:10FA400020F002020998027001229DF8B40040F2F1
:10FA5000833110FB01F09D4901EB800000F58960C6
:10FA60009DF8A01001EB410303EB011100EBC10075
:10FA700080F846209DF8B40040F2833110FB01F07D
:10FA8000924901EB800000F589609DF8A01001EB20
:10FA9000410303EB011100EBC100427341F28832D4
:10FAA0009DF8B40040F2833110FB01F0874901EB6F
:10FAB000800000F589609DF8A01001EB410303EB85
:10FAC000011100EBC1004261A9229DF8B40040F28F
:10FAD000833110FB01F07D4901EB800000F5896066
:10FAE0009DF8A01001EB410303EB011100E035E0AC
:10FAF00000EBC10082709DF8B40040F2833110FB2E
:10FB000001F0724901EB800042799DF8B40040F2A7
:10FB1000833110FB01F06D4901EB800000F5896035
:10FB20009DF8A01001EB410303EB011100F8312017
:10FB30009DF8B40000EB400101EB0010624901EBBD
:10FB4000001030309DF8A01000EB0110801C0990CF
:10FB5000007820F0800080300999087000202E90F5
:10FB60002F9000213A9122E0DDE92E10000140EAB9
:10FB700011720901CDE92E129DF8B41001EB41007C
:10FB8000C0EBC110524901EBC001BDF8E800801D77
:10FB9000085C3038C117DDE92E34184341EA04020D
:10FBA000CDE92E02BDF8E800401C80B23A90BDF8C5
:10FBB000E8000628D8DB9DF8B4002E9940F2833285
:10FBC00010FB02F0414A02EB800202F589629DF8C7
:10FBD000A00000EB400303EB001002EBC000C0F8F4
:10FBE0001A1000212E912F913A9122E0DDE92E107A
:10FBF000000140EA11720901CDE92E129DF8B410FE
:10FC000001EB4100C0EBC110314901EBC001BDF86F
:10FC1000E8000D30085C3038C117DDE92E3440EAC9
:10FC200003022143CDE92E21BDF8E800401C81B23A
:10FC30003A91BDF8E8000428D8DB9DF8B4002E996D
:10FC400040F2833210FB02F0204A02EB800202F500
:10FC500089629DF8A00000EB400303EB001002EB6B
:10FC6000C000416300222E922F9200213A9122E09F
:10FC7000DDE92E10000140EA11720901CDE92E12D2
:10FC80009DF8B41001EB4100C0EBC110104901EB2D
:10FC9000C001BDF8E8001130085C3038C117DDE95B
:10FCA0002E34184341EA0402CDE92E02BDF8E800E3
:10FCB000401C80B23A90BDF8E8000628D8DB9DF8D9
:10FCC000B4002E9906E00000C843002088480020B8
:10FCD000388F002040F2833210FB02F0FE4A02EB24
:10FCE000800202F589629DF8A00000EB400303EB5F
:10FCF000001002EBC000C0F81E109DF8B41001EB1C
:10FD00004100C0EBC110F54901EBC00042799DF8FC
:10FD1000B40040F2833110FB01F0EF4901EB8001A8
:10FD200001F589619DF8A00000EB400303EB001092
:10FD300001EBC000C2709DF8B41001EB410000EB74
:10FD40000110E74901EB001130319DF8A00001EBF3
:10FD5000001082789DF8B40040F2833110FB01F06E
:10FD6000DD4901EB800101F589619DF8A00000EB00
:10FD7000400303EB001001EBC00002769DF8B410C5
:10FD800040F2833011FB00F0D34901EB800101F513
:10FD900089619DF8A00000EB400202EB001011F811
:10FDA00030109DF8B40040F2833210FB02F0CA4AD2
:10FDB00002EB8000407981427EDA9DF8B41040F277
:10FDC000833011FB00F0114601EB800000F58960E3
:10FDD0009DF8A01001EB410202EB011110F8310077
:10FDE0000F2869DD00219DF8B40040F2833210FB3A
:10FDF00002F0B94A02EB80000171A7229DF8B4001D
:10FE000040F2833110FB01F0B34901EB800101F5B1
:10FE100089619DF8A00000EB400303EB001001EBAB
:10FE2000C000427101219DF8B40040F2833210FB02
:10FE300002F0A94A02EB800001719DF8B41040F273
:10FE4000833011FB00F0114601EB800042799DF8F0
:10FE5000B40040F2833110FB01F09F4901EB8001B7
:10FE600001F589619DF8A00000EB400303EB001051
:10FE700001F83020A1229DF8B40040F2833110FB3C
:10FE800001F0954901EB800101F589619DF8A00021
:10FE900000EB400303EB001001EBC00042719DF842
:10FEA000B41001EB410000EB01108D4901EB001192
:10FEB00030319DF8A00000E0A2E001EB0010801CB2
:10FEC0000990007820F080008030099908709DF832
:10FED000B41001EB410000EB0110814901EB00106F
:10FEE00030309DF8A01000EB0110801C09900078C4
:10FEF00020F00400001D099908709DF8B41001EB72
:10FF00004100C0EBC110754901EBC00040793028B9
:10FF100014D19DF8B41001EB410000EB01107049C1
:10FF200001EB001030309DF8A01000EB0110801C98
:10FF30000990007820F00102099802709DF8B41031
:10FF400001EB410000EB0110654901EB001030307E
:10FF50009DF8A01000EB01108078C0F3401088B924
:10FF60009DF8B41001EB410000EB01105C4901EB7E
:10FF7000001030309DF8A01000EB01108078C0F325
:10FF80004000E8B39DF8B40000EB400101EB001025
:10FF9000534901EB001030309DF8A01000EB011028
:10FFA000801C0990007820F02002099802709DF8CA
:10FFB000B40000EB400101EB0010494901EB0010D7
:10FFC00030309DF8A01000EB0110801C09900078E3
:10FFD00020F00202099802709DF8B40000EB400185
:10FFE00001EB00103E4901EB001030309DF8A010ED
:10FFF00000EB0110801C0990007820F0080000E060
:020000040801F1
:10000000B6E00830099908709DF8B4009DF8A0107A
:1000100001EB0010C217CDE92E029DF8B40040F2AA
:10002000833110FB01F02C4901EB800000F5896061
:100030009DF8A01001EB410202EB011100EBC100A1
:10004000223009902E9800EB4001264800EB411029
:100050000D30102208900999F8F7F7F89DF8B400D0
:1000600040F2833110FB01F01B4901EB800101F5E7
:1000700089619DF8A00000EB400202EB001001EB4B
:10008000C0012E9800EB4002164800EB421051F8D8
:100090001A2F40F8012F496841609DF8B40000EB29
:1000A000400101EB00100E4901EB001130319DF8C9
:1000B000A00001EB001001782E9800EB40020948E7
:1000C00000EB421001702E9800EB4001054800EB58
:1000D00041110548026809E088480020388F002057
:1000E000C8430020D8140020C731002041F81D2F3C
:1000F000808888809DF8B40040F2833110FB01F0C5
:10010000FE4901EB800101F589619DF8A00000EB3B
:10011000400202EB001001EBC000416B2E9800EB97
:100120004002F74800EB4210C0F809109DF8B400F7
:1001300000EB400101EB0010F24901EB00113031FE
:100140009DF8A00001EB001041682E9800EB4002E2
:10015000EB4800EB4210C0F823102E9881B2082023
:100160000991F9F7A3FF9DF8B4100220F9F79EFF5B
:10017000FEE300202E902F9000213A9122E0DDE94D
:100180002E10000140EA11720901CDE92E129DF8EE
:10019000B40000EB4001C1EBC010DB4901EBC00132
:1001A000BDF8E8000B30085C3038C117DDE92E34AB
:1001B000184341EA0402CDE92E02BDF8E800401CD4
:1001C00080B23A90BDF8E8000A28D8DB9DF8B40068
:1001D000DDE92E2140F2833310FB03F0C74B03EB24
:1001E000800303F589639DF8A00000EB400404EB55
:1001F000001003EBC00040F8222F416000222E9235
:100200002F9200213A9122E0DDE92E10000140EA10
:1002100011720901CDE92E129DF8B40000EB4001E6
:10022000C1EBC010B84901EBC001BDF8E8001530C2
:10023000085C3038C117DDE92E34184341EA040266
:10024000CDE92E02BDF8E800401C80B23A90BDF81E
:10025000E8000A28D8DB9DF8B400DDE92E1240F250
:10026000833310FB03F0A54B03EB800303F5896395
:100270009DF8A00000EB400404EB001003EBC0006D
:1002800022308160C26000219DF8B40040F28332C8
:1002900010FB02F0994A02EB800001719DF8B40056
:1002A00040F2833110FB01F0114601EB800101F5B2
:1002B00089619DF8A00000EB400202EB001011F8EC
:1002C00030109DF8B40040F2833210FB02F08B4AEC
:1002D00002EB8000407981427ED19DF8B4009DF808
:1002E000A01001EB0010C217CDE92E02874890F84C
:1002F000100B08B39DF8B40000EB400101EB0010B7
:10030000804901EB001030309DF8A01000EB011087
:10031000807A022810D09DF8B40000EB400101EB78
:100320000010784901EB001030309DF8A01000EB70
:100330000110C07A00287DDD00229DF8B40000EB9A
:10034000400101EB00106F4901EB001030309DF8C7
:10035000A01000EB0110C2726D48D0F80C0205210C
:10036000B0FBF1F201FB120000EB400168482C30B9
:1003700000EB41100D3009909DF8B40040F283313C
:1003800010FB01F05D4901EB800000F589609DF8EC
:10039000A01001EB410202EB011100EBC100223081
:1003A0001022014608900998F7F74FFF5848D0F8F7
:1003B0000C020521B0FBF1F201FB120000EB400141
:1003C00053482C3000EB41129DF8B40040F28331C9
:1003D00010FB01F0494900E00AE301EB800101F55F
:1003E00089619DF8A00000EB400303EB001001EBD6
:1003F000C00050F81A1F42F8011F4068506044487E
:10040000D0F80C020521B0FBF1F201FB120000EB69
:1004100040013F482C3000EB41129DF8B40000EB46
:10042000400101EB0010374901EB001130319DF81C
:10043000A00000E097E101EB001000781070344854
:10044000D0F80C020521B0FBF1F201FB120000EB29
:1004500040012F482C3000EB41129DF8B40040F2CF
:10046000833110FB01F0254901EB800101F5896121
:100470009DF8A00000EB400303EB001001EBC0006F
:10048000406BC2F809002248D0F80C020521B0FBED
:10049000F1F201FB120000EB40011D482C3000EB93
:1004A00041111A48F538026841F81D2F808888806C
:1004B0001748D0F80C020521B0FBF1F201FB120045
:1004C00000EB400112482C3000EB41129DF8B400C3
:1004D00000EB400101EB00100A4901EB0011303143
:1004E0009DF8A00001EB00104068C2F82300002234
:1004F0009DF8B40000EB40010CE0000088480020AB
:10050000D8140020C8430020388F0020BC320020BF
:10051000BC12002001EB0010FE4901EB001130314C
:100520009DF8A00001EB0010426000213A9154E0D8
:10053000F948D0F80C020521B0FBF1F201FB1200E2
:1005400000EB4001F4482C3000EB41112731BDF89D
:10055000E8409DF8B40040F2833210FB02F0EF4A0D
:1005600002EB800202F589629DF8A00000EB4003D7
:1005700003EB001002EBC00090F8800040F28332E1
:1005800010FB02F0E54A02EB800202F589629DF859
:10059000B40040F2833310FB03F0E04B03EB800325
:1005A00003F589639DF8A00000EB400505EB001002
:1005B00003EBC00090F8810000EB400303EB001058
:1005C00002EBC0024732BDF8E800001D105C085580
:1005D000BDF8E800401C81B23A91BDF8E800062859
:1005E000A6DB00213A9142E000239DF8B40040F2DE
:1005F000833110FB01F0C94901EB800101F58961EC
:100600009DF8A00000EB400202EB001001EBC000DF
:1006100090F8800040F2833110FB01F0BF4901EBFC
:10062000800101F589619DF8B40040F2833210FB2E
:1006300002F0BA4A02EB800202F589629DF8A0003E
:1006400000EB400404EB001002EBC00090F88100C6
:1006500000EB400202EB001001EBC0014731BDF896
:10066000E8000B54BDF8E800401C81B23A91BDF897
:10067000E8000A28B8DBA848D0F80C020521B0FB36
:10068000F1F080B2014609900220F8F721FD002127
:100690000620F9F70BFDA048D0F80C029E49498DC1
:1006A000884206D29C48D0F80C02401C9A49C1F8F6
:1006B0000C0200210520F9F7F9FC9DF8B40000EBCD
:1006C000400101EB0010934901EB001030309DF820
:1006D000A01000EB0110801C0990007820F00802A7
:1006E000099802708C48D0F80C020521B0FBF1F299
:1006F00001FB120000EB400187482C3000EB411059
:10070000D0F823202E9800EB4001854800EB4110E3
:10071000C0F8232000203A9020E07F48D0F80C0257
:100720000521B0FBF1F201FB120000EB40017A4819
:100730002C3000EB41102730BDF8E810425C2E98B9
:1007400000EB4001764800EB41112731BDF8E8008D
:100750000A54BDF8E800401C81B23A91BDF8E800A7
:100760000628DADB59E09DF8B40000EB400101EB0C
:100770000010684901EB001030309DF8A01000EB2C
:100780000110801C0990007820F0080108310998B8
:1007900001709DF8B40000EB400101EB00105D49D1
:1007A00001EB001130319DF8A00001EB0010416811
:1007B0002E9800EB40025A4800EB4210C0F823107C
:1007C00000213A9125E09DF8B40040F2833110FBFE
:1007D00001F0524901EB800101F589619DF8A0000B
:1007E00000EB400202EB001001EBC0014731BDF805
:1007F000E8000A5C2E9800EB4001494800EB4111EB
:100800002731BDF8E8000A54BDF8E800401C81B269
:100810003A91BDF8E8000628D5DB00229DF8B40027
:1008200040F2833110FB01F03C4901EB800101F5FE
:1008300089619DF8A00000EB400303EB001001EB81
:10084000C00080F846209DF8B40040F2833110FBD0
:1008500001F0324901EB800101F589619DF8A000AA
:1008600000EB400303EB001001EBC00042739DF866
:10087000B40040F2833110FB01F0284901EB800104
:1008800001F589619DF8A00000EB400303EB001027
:1008900001EBC00002619DF8B4100220F9F706FCDC
:1008A0009DF8B40040F2833110FB01F01B4901EBCD
:1008B000800101F589619DF8A00000EB400202EB88
:1008C000001001EBC000223009902E9800EB40018F
:1008D000134800EB41100D30102208900999F7F7EA
:1008E000B4FC9DF8B40040F2833110FB01F00B49D9
:1008F00001EB800101F589619DF8A00000EB400249
:1009000002EB001001EBC0012E9800EB40020448FE
:1009100008E00000C8430020BC12002088480020E6
:10092000D814002000EB421051F81A2F40F8012F84
:10093000496841609DF8B40000EB400101EB0010F4
:10094000FE4901EB001130319DF8A00001EB0010D1
:1009500001782E9800EB4002F94800EB421001703C
:100960002E9800EB4001F64800EB4111F54800E0FD
:1009700092E0026841F81D2F808888809DF8B400BD
:1009800040F2833110FB01F0EF4901EB800101F5EA
:1009900089619DF8A00000EB400202EB001001EB22
:1009A000C000416B2E9800EB4002E54800EB42107E
:1009B000C0F809109DF8B40000EB400101EB0010F5
:1009C000DE4901EB001130319DF8A00001EB001071
:1009D00041682E9800EB4002D94800EB4210C0F865
:1009E00023102E9881B208200991F9F75FFB28E0C7
:1009F0009DF8B40040F2833110FB01F0D24901EBC5
:100A0000800000F589609DF8A01001EB410202EB27
:100A1000011110F831000C2813DC0D229DF8B400F0
:100A200040F2833110FB01F0C74901EB800000F573
:100A300089609DF8A01001EB410303EB011100F860
:100A40003120A7229DF8B40040F2833110FB01F061
:100A5000BD4901EB800101F589619DF8A00000EB23
:100A6000400303EB001001EBC0004271A2229DF88D
:100A7000B40040F2833110FB01F0B34901EB800078
:100A800000F589609DF8A01001EB410303EB011113
:100A900000EBC100827000BF00BF0EF014B99DF8DA
:100AA000B40000EB4001C1EBC010A84911F83000C0
:100AB000042802D1042125910CE09DF8B40000EB3C
:100AC0004001C1EBC010A14911F83000152801D137
:100AD000152125919DF8B40000EB4001C1EBC01039
:100AE0009A4901EBC00041789DF8B40000EB400248
:100AF000C2EBC010954A12F8300041EA002041F2E2
:100B00003001884202D1A62125913DE09DF8B40034
:100B100000EB4001C1EBC0108C4901EBC0004178F3
:100B20009DF8B40000EB4002C2EBC010874A12F8F7
:100B3000300041EA002041F23101884202D1A72170
:100B4000259121E09DF8B40000EB4001C1EBC010FD
:100B50007E4911F83000022816D19DF8B40000EB50
:100B60004001C1EBC010794901EBC00001799DF84B
:100B7000B40000EB4002C2EBC010744A02EBC000AC
:100B8000C07841EA002125919DF8B40040F28331FC
:100B900010FB01F06C4901EB800081782891002165
:100BA0006B4A9DF8B40002EB00129DF8A0001154AE
:100BB000684890F82800012815D19DF8B40000EB92
:100BC000400101EB00105D4901EB001030309DF851
:100BD000A01000EB0110801C0990007820F080002C
:100BE000803009990870BDF89400A7287DD007DCF3
:100BF00004287BD015287AD0A62841F06A8752E0D5
:100C0000A0F55850303820B1112871D01228F4D1F5
:100C1000FEE39DF8B40040F2833110FB01F04A4935
:100C200001EB800000F589609DF8A01001EB410206
:100C300002EB011110F8310098BB00219DF8B400BF
:100C400040F2833210FB02F03F4A02EB8000017158
:100C500001229DF8B40040F2833110FB01F03A49C3
:100C600001EB800101F589619DF8A00000EB4003D4
:100C700003EB001001F83020A7229DF8B40040F2E9
:100C8000833110FB01F0304901EB800000F58960F1
:100C90009DF8A01001EB410303EB011100EBC10033
:100CA000427101F016BF00219DF8B40040F283327A
:100CB00010FB02F0244A02EB800001719DF8B400A1
:100CC00040F2833110FB01F0114601EB800000F58A
:100CD00089609DF8A01001EB410202EB011110F8B0
:100CE000310002283EDC032203E0FAE061E1B1E2D8
:100CF000E5E29DF8B40040F2833110FB01F01249A7
:100D000001EB800101F589619DF8A00000EB400333
:100D100003EB001001F83020A9229DF8B40040F246
:100D2000833110FB01F0084901EB800000F5896078
:100D30009DF8A01001EB41030EE00000C843002025
:100D4000D8140020C731002088480020388F0020A8
:100D5000B8410020BC12002003EB011100EBC100E0
:100D60004271BDE09DF8B40040F2833110FB01F008
:100D7000FE4901EB800000F589609DF8A01001EBB1
:100D8000410202EB011110F83100052829DC06228E
:100D90009DF8B40040F2833110FB01F0F34901EB00
:100DA000800101F589619DF8A00000EB400303EB91
:100DB000001001F83020A2229DF8B40040F28331E7
:100DC00010FB01F0E94901EB800000F589609DF816
:100DD000A01001EB410303EB011100EBC1004271D4
:100DE0007EE09DF8B40040F2833110FB01F0DF4952
:100DF00001EB800000F589609DF8A01001EB410235
:100E000002EB011100EBC1004079A52815D19DF836
:100E1000B40000EB400101EB0010D54901EB0010DC
:100E200030309DF8A01000EB0110801C0990007874
:100E300020F00400001D099908709DF8B40040F2EC
:100E4000833110FB01F0C94901EB800000F5896096
:100E50009DF8A01001EB410202EB011100EBC10073
:100E60008078A1283CD09DF8B40040F2833110FB7B
:100E700001F0BE4901EB800101F589619DF8A000F8
:100E800000EB400202EB001001EBC00082789DF8FD
:100E9000B40040F2833110FB01F0B44901EB800152
:100EA00001F589619DF8A00000EB400303EB001001
:100EB00001EBC0004271A1229DF8B40040F28331E1
:100EC00010FB01F0A94901EB800000F589609DF855
:100ED000A01001EB410303EB011100EBC100827094
:100EE000DFE69DF8B40040F2833110FB01F09F492A
:100EF00001EB800000F589609DF8A01001EB410234
:100F000002EB011100EBC1004079A42830D19DF81B
:100F1000B40000EB400101EB0010954901EB00101B
:100F200030309DF8A01000EB0110801C0990007873
:100F300020F0200120310998017000229DF8B400B2
:100F400040F2833110FB01F0884901EB800101F58B
:100F500089619DF8A00000EB400303EB001001EB5A
:100F6000C00080F845209DF8B4100220F9F79EF8E3
:100F700000219DF8B40040F2833210FB02F07B4A5E
:100F800002EB80000171A1229DF8B40040F2833190
:100F900010FB01F0754901EB800000F589609DF8B8
:100FA000A01001EB410303EB011100EBC100427102
:100FB00077E69DF8B40040F2833110FB01F06B49F5
:100FC00001EB800000F589609DF8A01001EB410263
:100FD00002EB011110F83100012834DC00219DF8EA
:100FE000B40040F2833210FB02F0604A02EB800052
:100FF000017102229DF8B40040F2833110FB01F030
:101000005A4901EB800101F589619DF8A00000EBD0
:10101000400303EB001001F83020A3229DF8B40038
:1010200040F2833110FB01F0504901EB800000F5E4
:1010300089609DF8A01001EB410303EB011100EB67
:10104000C100427105E19DF8B40040F2833110FB0C
:1010500001F0464901EB800000F589609DF8A01081
:1010600001EB410202EB011110F83100042834DCDD
:1010700000219DF8B40040F2833210FB02F03B4A9D
:1010800002EB8000017105229DF8B40040F283312B
:1010900010FB01F0354901EB800101F589619DF8F4
:1010A000A00000EB400303EB001001F83020A32266
:1010B0009DF8B40040F2833110FB01F02B4901EBA5
:1010C000800000F589609DF8A01001EB410303EB5F
:1010D000011100EBC1004271BBE09DF8B40040F289
:1010E000833110FB01F0214901EB800000F589609C
:1010F0009DF8A01001EB410202EB011110F8310044
:10110000062815DCA1229DF8B40040F2833110FBC3
:1011100001F0164901EB800000F589609DF8A010F0
:1011200001EB410303EB011100EBC100427190E0C0
:101130009DF8B40040F2833110FB01F00B4901EB44
:10114000800101F589619DF8A00000EB400202EBEF
:10115000001011F830109DF8B40040F2833210FBFB
:1011600002F0024A02EB8000407903E08848002048
:10117000C843002081426CD19DF8B40040F2833115
:1011800010FB01F0114601EB800000F589609DF82D
:10119000A01001EB410202EB011100EBC1008078CD
:1011A000A12836D0A3229DF8B40040F2833110FB71
:1011B00001F0FE4901EB800101F589619DF8A00075
:1011C00000EB400303EB001001EBC00042719DF8FF
:1011D000B40040F2833110FB01F0F44901EB8000D0
:1011E00000F589609DF8A01001EB410202EB0111AE
:1011F00000EBC1008078A2282BD000209DF8B4100D
:1012000040F2833211FB02F1E84A02EB81010871DE
:101210001FE0A1229DF8B40040F2833110FB01F0E1
:10122000E24901EB800101F589619DF8A00000EB26
:10123000400303EB001001EBC000427101219DF857
:10124000B40040F2833210FB02F0D84A02EB800077
:10125000017126E5A1229DF8B40040F2833110FB14
:1012600001F0D24901EB800101F589619DF8A000F0
:1012700000EB400303EB001001EBC00042719DF84E
:10128000B40040F2833110FB01F0C84901EB80014A
:1012900001F589619DF8A00000EB400303EB00100D
:1012A00001EBC000827000219DF8B40040F283324F
:1012B00010FB02F0BD4A02EB80000171F1E4002155
:1012C0009DF8B40040F2833210FB02F0B74A02EB03
:1012D00080000171A7229DF8B40040F2833110FB19
:1012E00001F0B24901EB800101F589619DF8A00090
:1012F00000EB400303EB001001EBC00042719DF8CE
:10130000B40000EB4001C1EBC010A94901EBC000E3
:10131000407930287DD19DF8B40040F2833110FB34
:1013200001F0A24901EB800101F589619DF8A0005F
:1013300000EB400202EB001011F830109DF8B400F1
:1013400040F2833210FB02F0984A02EB80004079B1
:1013500081425ED19DF8B40000EB400101EB00102A
:10136000A2F5986101EB001030309DF8A01000EB61
:101370000110801C0990007820F001020998027089
:101380009DF8B40000EB400101EB0010894901EB2E
:10139000001030309DF8A01000EB0110801C099067
:1013A000007820F00202099802709DF8B40040F223
:1013B000833110FB01F07D4901EB800000F589606D
:1013C0009DF8A01001EB410202EB011100EBC100FE
:1013D000C078312832D19DF8B40000EB400101EB18
:1013E0000010744901EB001030309DF8A01000EBA4
:1013F0000110801C0990007820F0200209980270EA
:1014000000229DF8B40040F2833110FB01F001E0AE
:10141000FEE340E0654901EB800000F589609DF83E
:10142000A01001EB410303EB011100EBC10080F8B8
:1014300045209DF8B4100220F8F738FE9DF8B4005E
:1014400040F2833110FB01F0584901EB800000F5B8
:1014500089609DF8A01001EB410202EB011100EB45
:10146000C10090F84600012814D1A9229DF8B400CB
:1014700040F2833110FB01F04C4901EB800000F594
:1014800089609DF8A01001EB410303EB011100EB13
:10149000C1008270DCE39DF8B40000EB4001C1EBB9
:1014A000C010434901EBC000407931287CD19DF840
:1014B000B40040F2833110FB01F03C4901EB8001A4
:1014C00001F589619DF8A00000EB400202EB0010DD
:1014D00011F830109DF8B40040F2833210FB02F096
:1014E000324A02EB8000407981425DD19DF8B40020
:1014F00040F2833110FB01F0114601EB800000F552
:1015000089609DF8A01001EB410202EB011100EB94
:10151000C10090F8460058BB01229DF8B40040F28B
:10152000833110FB01F0214901EB800101F5896154
:101530009DF8A00000EB400303EB001001EBC0009E
:1015400080F845209DF8B40000EB400101EB00104D
:10155000184901EB001130319DF8A00001EB00109B
:10156000801C0990007820F00100401C0999087047
:101570009DF8B40000EB400101EB00100D4901EBB8
:10158000001030309DF8A01000EB0110801C099075
:10159000007820F0020209980270074890F8100BBA
:1015A000D8B19DF8B40009E00CE2000088480020A2
:1015B000388F0020C8430020BC32002000EB4001DF
:1015C00001EB0010FC4901EB001030309DF8A01039
:1015D00000EB0110807A022876D1F84890F82900B3
:1015E0000128F9D1F548D0F80C02F449498D884218
:1015F0006AD29DF8B40040F2833110FB01F0F0494B
:1016000001EB800000F589609DF8A01001EB41021C
:1016100002EB011100EBC10090F84500012852D106
:101620009DF8B40040F2833110FB01F0E44901EB76
:10163000800000F589609DF8A01001EB410202EBEB
:10164000011100EBC10090F87F00E0BB01229DF882
:10165000B40000EB400101EB0010D74901EB001191
:1016600030319DF8A00001EB0010C2724FF0104223
:101670009DF8B40040F2833110FB01F0D04901EB3A
:10168000800101F589619DF8A00000EB400303EBA8
:10169000001001EBC00082609DF8B40000EB400137
:1016A00001EB0010C44901EB001130319DF8A0009E
:1016B00001EB001001789DF8B40040F2833210FB7A
:1016C00002F0BF4A01E072E005E102EB80004170E8
:1016D0009DF8B40040F2833110FB01F0114601EB9C
:1016E000800101F589619DF8A00000EB400202EB4A
:1016F000001011F830109DF8B40040F2833210FB56
:1017000002F0AF4A02EB8000407981423ED10022D4
:101710009DF8B40040F2833110FB01F0A84901EBC1
:10172000800101F589619DF8A00000EB400303EB07
:10173000001001EBC000C271A4229DF8B40040F279
:10174000833110FB01F09E4901EB800101F58961B5
:101750009DF8A00000EB400303EB001001EBC0007C
:101760008270A3229DF8B40040F2833110FB01F097
:10177000934901EB800000F589609DF8A01001EB12
:10178000410303EB011100EBC100427100229DF8FF
:10179000B40000EB400101EB0010874901EB0010A1
:1017A00030309DF8A01000EB0110426050E29DF82F
:1017B000B40040F2833110FB01F0814901EB80005D
:1017C00000F589609DF8A01001EB410202EB0111C8
:1017D00000EBC10090F8450001287CD19DF8B400D1
:1017E00040F2833110FB01F0754901EB800101F5F6
:1017F00089619DF8A00000EB400202EB001001EBB4
:10180000C00090F8800040F2833110FB01F06C4979
:1018100001EB800101F589619DF8B40040F283324B
:1018200010FB02F0664A02EB800000F589609DF82B
:10183000A02002EB420303EB021200EBC20090F87F
:10184000810000EB400202EB001001EBC00090F8B9
:101850007E0003283FD102229DF8B40000EB400136
:1018600001EB0010544901EB001130319DF8A0004C
:1018700001EB0010C2724FF010429DF8B40040F22C
:10188000833110FB01F04E4901EB800101F58961C4
:101890009DF8A00000EB400303EB001001EBC0003B
:1018A00082609DF8B40000EB400101EB001042495A
:1018B00001EB001130319DF8A00001EB0010017820
:1018C0009DF8B40040F2833210FB02F03C4A02EB78
:1018D0008000417000E09CE19DF8B40040F283314B
:1018E00010FB01F0114601EB800101F589619DF8C3
:1018F000A00000EB400202EB001011F830109DF840
:10190000B40040F2833210FB02F02D4A02EB80005B
:10191000407981423ED100229DF8B40040F28331EB
:1019200010FB01F0264901EB800101F589619DF86A
:10193000A00000EB400303EB001001EBC000C271FC
:10194000A4229DF8B40040F2833110FB01F01C4941
:1019500001EB800101F589619DF8A00000EB4003D7
:1019600003EB001001EBC0008270A3229DF8B400CD
:1019700040F2833110FB01F0114901EB800000F5CA
:1019800089609DF8A01001EB410303EB011100EB0E
:10199000C100427100229DF8B40000EB400101EB50
:1019A0000010054901EB001030309DF8A01000EB4D
:1019B000011042604CE10000C8430020BC1200202E
:1019C000884800209DF8B40000EB4001C1EBC01036
:1019D000FE4901EBC000407933287DD19DF8B40069
:1019E00000EB400101EB0010F94901EB0010303031
:1019F0009DF8A01000EB0110801C0990007820F0E9
:101A00000100401C099908709DF8B40000EB4001EA
:101A100001EB0010EE4901EB001030309DF8A010F2
:101A200000EB0110801C0990007820F0200209983A
:101A300002709DF8B40000EB400101EB0010E44996
:101A400001EB001030309DF8A01000EB0110801C5D
:101A50000990007820F00200801C099908709DF818
:101A6000B40040F2833110FB01F0DA4901EB800051
:101A700042799DF8B40040F2833110FB01F0D54962
:101A800001EB800000F589609DF8A01001EB410397
:101A900003EB011100F831209DF8B40000EB400188
:101AA00001EB0010CA4901EB001030309DF8A01086
:101AB00000EB0110801C0990007820F0800080303D
:101AC000099908709DF8B40000EB400101EB00108B
:101AD000BF4901EB001000E023E030309DF8A0107A
:101AE00000EB01108078C0F3400020B99DF8B410DD
:101AF0000220F8F7DBFAA2229DF8B40040F283310D
:101B000010FB01F0B34901EB800000F589609DF8FE
:101B1000A01001EB410303EB011100EBC100827047
:101B200096E09DF8B40000EB4001C1EBC010A7495E
:101B300001EBC000407934286BD19DF8B40000EB74
:101B4000400101EB0010A24901EB001030309DF87C
:101B5000A01000EB0110801C0990007820F02002FA
:101B6000099802709DF8B40000EB400101EB0010F1
:101B7000974901EB001030309DF8A01000EB0110E8
:101B8000801C0990007820F002020998027001225E
:101B90009DF8B40040F2833110FB01F08D4901EB58
:101BA000800000F589609DF8A01001EB410303EB74
:101BB000011100EBC10080F84620A9229DF8B40075
:101BC00040F2833110FB01F0824901EB800000F507
:101BD00089609DF8A01001EB410303EB011100EBBC
:101BE000C10082709DF8B40040F2833110FB01F017
:101BF000784901EB800042799DF8B40040F28331CE
:101C000010FB01F0734901EB800000F5896001E0F1
:101C1000D4E21DE09DF8A01001EB410303EB01119C
:101C200000F831209DF8B40000EB400101EB0010FA
:101C3000674901EB001030309DF8A01000EB011057
:101C4000801C0990007820F080008030099908708D
:101C500000202E902F9000213A9121E0DDE92E10F6
:101C6000000140EA11720901CDE92E129DF8B4007D
:101C700000EB4001C1EBC010544901EBC001BDF8BD
:101C8000E800801D085C3038C117DDE92E240243CE
:101C90002143CDE92E21BDF8E800401C81B23A91E4
:101CA000BDF8E8000828D9DB9DF8B4002E9940F271
:101CB000833210FB02F0474A02EB800202F5896290
:101CC0009DF8A00000EB400303EB001002EBC00006
:101CD000C0F81A1000222E922F9200213A9122E091
:101CE000DDE92E10000140EA11720901CDE92E1242
:101CF0009DF8B40000EB4001C1EBC010334901EB8B
:101D0000C001BDF8E8000F30085C3038C117DDE9CC
:101D10002E34184341EA0402CDE92E02BDF8E80052
:101D2000401C80B23A90BDF8E8000628D8DB9DF848
:101D3000B4002E9940F2833210FB02F0254A02EBE8
:101D4000800202F589629DF8A00000EB400303EBDE
:101D5000001002EBC000416300222E922F9200215E
:101D60003A9122E0DDE92E10000140EA11720901EA
:101D7000CDE92E129DF8B40000EB4001C1EBC0107C
:101D8000124901EBC001BDF8E8001530085C30389D
:101D9000C117DDE92E34184341EA0402CDE92E02D1
:101DA000BDF8E800401C80B23A90BDF8E800082871
:101DB000D8DB9DF8B4002E9940F2833210FB02F07C
:101DC000044A02EB800202F5896205E0388F0020A8
:101DD000C8430020884800209DF8A00000EB400385
:101DE00003EB001002EBC000C0F81E109DF8B40019
:101DF00000EB4001C1EBC010FE4901EBC00042798D
:101E00009DF8B40040F2833110FB01F0FA4901EB78
:101E1000800101F589619DF8A00000EB400303EB10
:101E2000001001EBC000C2709DF8B40000EB40014F
:101E300001EB0010F14901EB001130319DF8A000D9
:101E400001EB001082789DF8B40040F2833110FB62
:101E500001F0E94901EB800101F589619DF8A000DD
:101E600000EB400303EB001001EBC00002769DF88D
:101E7000B40040F2833110FB01F0DF4901EB800137
:101E800001F589619DF8A00000EB400202EB001013
:101E900011F830109DF8B40040F2833210FB02F0CC
:101EA000D54A02EB8000407981427DDA00219DF81D
:101EB000B40040F2833210FB02F0CF4A02EB800004
:101EC0000171A7229DF8B40040F2833110FB01F0AC
:101ED000C94901EB800101F589619DF8A00000EB83
:101EE000400303EB001001EBC000427101219DF89B
:101EF000B40040F2833210FB02F0BF4A02EB8000D4
:101F000001719DF8B40040F2833110FB01F01146DD
:101F100001EB800042799DF8B40040F2833110FB60
:101F200001F0B54901EB800101F589619DF8A00040
:101F300000EB400303EB001001F83020A1229DF8D4
:101F4000B40040F2833110FB01F0AB4901EB80019A
:101F500001F589619DF8A00000EB400303EB001040
:101F600001EBC00042719DF8B40000EB400101EBB1
:101F70000010A24901EB001130319DF8A00001EBE7
:101F80000010801C0990007820F0800080300999B2
:101F900008709DF8B40000EB400101EB0010974978
:101FA00001EB0010303000E05BE09DF8A01000EB8A
:101FB0000110801C0990007820F00400001D099990
:101FC00008709DF8B40000EB400101EB00108B4954
:101FD00001EB001030309DF8A01000EB011080786C
:101FE000C0F34010E8B39DF8B40000EB400101EBF2
:101FF0000010824901EB001030309DF8A01000EB7A
:102000000110801C0990007820F0200209980270CD
:102010009DF8B40000EB400101EB0010774901EBA3
:10202000001030309DF8A01000EB01108078C0F354
:102030004000E8BB9DF8B40000EB400101EB00104C
:102040006E4901EB001030309DF8A01000EB01103C
:10205000801C0990007820F0080008300999087069
:1020600000E0AAE09DF8B4009DF8A01001EB00107C
:10207000C217CDE92E029DF8B40040F2833110FB67
:1020800001F05D4901EB800000F589609DF8A0102A
:1020900001EB410202EB011100EBC100223009907B
:1020A0002E9800EB4001564800EB41100D3000E047
:1020B0007EE0102208900999F6F7C7F89DF8B40061
:1020C00040F2833110FB01F04B4901EB800101F537
:1020D00089619DF8A00000EB400202EB001001EBCB
:1020E000C0012E9800EB4002454800EB421051F829
:1020F0001A2F40F8012F496841609DF8B40000EBA9
:10210000400101EB00103D4901EB001130319DF819
:10211000A00001EB001001782E9800EB4002384837
:1021200000EB421001702E9800EB4001344800EBA8
:1021300041113448026841F81D2F808888809DF83D
:10214000B40040F2833110FB01F02B4901EB800118
:1021500001F589619DF8A00000EB400202EB001040
:1021600001EBC000416B2E9800EB4002244800EBCD
:102170004210C0F809109DF8B40000EB400101EBDB
:1021800000101E4901EB001130319DF8A00001EB59
:10219000001041682E9800EB4002194800EB4210F5
:1021A000C0F823102E9881B208200991F7F77EFF1E
:1021B0009DF8B4100220F7F779FFFDE300202E9080
:1021C0002F9000213A912DE0DDE92E10000140EA28
:1021D00011720901CDE92E129DF8B40000EB400107
:1021E000C1EBC010034901EBC001BDF8E8000B30A2
:1021F000085C09E0388F002088480020C843002090
:10220000D8140020C73100203038C117DDE92E3442
:10221000184341EA0402CDE92E02BDF8E800401C53
:1022200080B23A90BDF8E8000C28CDDB9DF8B400F0
:10223000DDE92E1240F2833310FB03F0FE4B03EB7B
:10224000800303F589639DF8A00000EB400404EBD4
:10225000001003EBC00040F8221F426000222E92C3
:102260002F9200213A9122E0DDE92E10000140EA90
:1022700011720901CDE92E129DF8B40000EB400166
:10228000C1EBC010ED4901EBC001BDF8E80017300B
:10229000085C3038C117DDE92E34184341EA0402E6
:1022A000CDE92E02BDF8E800401C80B23A90BDF89E
:1022B000E8000C28D8DB9DF8B400DDE92E2140F2BF
:1022C000833310FB03F0DC4B03EB800303F58963DE
:1022D0009DF8A00000EB400404EB001003EBC000ED
:1022E00022308260C16000219DF8B40040F2833248
:1022F00010FB02F0D04A02EB800001719DF8B4009F
:1023000040F2833110FB01F0114601EB800000F533
:1023100089609DF8A01001EB410202EB011110F859
:102320003100032814DC04229DF8B40040F283310C
:1023300010FB01F0C04901EB800000F589609DF8B9
:10234000A01001EB410303EB011100F8312073E30E
:102350009DF8B40040F2833110FB01F0B64901EB67
:10236000800101F589619DF8A00000EB400202EBBD
:10237000001011F830109DF8B40040F2833210FBC9
:1023800002F0AD4A02EB800040798142DFD19DF836
:10239000B4009DF8A01001EB0010C217CDE92E0289
:1023A000A74890F8100B08B39DF8B41001EB41005A
:1023B00000EB0110A34901EB001030309DF8A01094
:1023C00000EB0110807A022810D09DF8B41001EBC8
:1023D000410000EB01109B4901EB001030309DF8EB
:1023E000A01000EB0110C07A00287DDD00229DF8CE
:1023F000B40000EB400101EB0010924901EB00102A
:1024000030309DF8A01000EB0110C2728E48D0F859
:102410000C020521B0FBF1F201FB120000EB4001C0
:1024200089482C3000EB41100D3009909DF8B41014
:1024300040F2833011FB00F07F4901EB800000F592
:1024400089609DF8A01001EB410202EB011100EB45
:10245000C10022301022014608900998F5F7F5FED8
:102460007948D0F80C020521B0FBF1F201FB120013
:1024700000EB400174482C3000EB41129DF8B40091
:1024800040F2833110FB01F06B4901EB800101F553
:1024900089619DF8A00000EB400303EB001001EB05
:1024A000C00050F81A1F42F8011F4068506066488B
:1024B000D0F80C020521B0FBF1F201FB120000EB99
:1024C000400161482C3000EB41129DF8B40000EB54
:1024D000400101EB00105B4901EB001130319DF828
:1024E000A00001EB001000E093E100781070564866
:1024F000D0F80C020521B0FBF1F201FB120000EB59
:10250000400151482C3000EB41129DF8B40040F2DC
:10251000833110FB01F0484901EB800101F589612D
:102520009DF8A00000EB400303EB001001EBC0009E
:10253000406BC2F809004448D0F80C020521B0FBFA
:10254000F1F201FB120000EB40013F482C3000EBA0
:1025500041113B48F538026841F81D2F808888807A
:102560003948D0F80C020521B0FBF1F201FB120052
:1025700000EB400134482C3000EB41129DF8B400D0
:1025800000EB400101EB00102E4901EB001130314E
:102590009DF8A00001EB00104068C2F82300002263
:1025A0009DF8B40000EB400101EB0010254901EB60
:1025B000001130319DF8A00001EB001042600021B5
:1025C0003A9160E02048D0F80C020521B0FBF1F20E
:1025D00001FB120000EB40011B482C3000EB4111C5
:1025E0002731BDF8E8409DF8B40040F2833210FB7B
:1025F00002F0114A02EB800202F589629DF8A00008
:1026000000EB400303EB001002EBC00090F88000E9
:1026100040F2833210FB02F0074A02EB800202F51F
:1026200089629DF8B40040F2833310FB03F0024B43
:1026300003EB80030AE0000088480020388F002068
:10264000BC320020C8430020BC12002003F589637F
:102650009DF8A00000EB400505EB001003EBC00067
:1026600090F8810000EB400303EB001002EBC00286
:102670004732BDF8E800001D105C0855BDF8E800C1
:10268000401C81B23A91BDF8E80006289ADB00218F
:102690003A9142E000239DF8B40040F2833110FBF0
:1026A00001F0FE4901EB800101F589619DF8A00070
:1026B00000EB400202EB001001EBC00090F880003C
:1026C00040F2833110FB01F0F44901EB800202F586
:1026D00089629DF8B40040F2833110FB01F0EF49AC
:1026E00001EB800101F589619DF8A00000EB400439
:1026F00004EB001001EBC00090F8810000EB4001FA
:1027000001EB001002EBC0014731BDF8E8000B54AB
:10271000BDF8E800401C81B23A91BDF8E8000A28F3
:10272000B8DBDF48D0F80C020521B0FBF1F080B235
:10273000014609900220F6F7CBFC00210620F7F7AE
:10274000B5FCD748D0F80C02D549498D884206D24D
:10275000D348D0F80C02401CD149C1F80C0200212A
:102760000520F7F7A3FC9DF8B41001EB410000EB46
:102770000110CC4901EB001030309DF8A01000EBA7
:102780000110801C0990007820F00802099802705E
:10279000C348D0F80C020521B0FBF1F201FB120096
:1027A00000EB4001BE482C3000EB4110D0F8232054
:1027B0002E9800EB4001BC4800EB4110C0F82320EC
:1027C00000203A9020E0B648D0F80C020521B0FB7A
:1027D000F1F201FB120000EB4001B1482C3000EB9C
:1027E00041102730BDF8E810425C2E9800EB400104
:1027F000AD4800EB41112731BDF8E8000A54BDF89F
:10280000E800401C81B23A91BDF8E8000628DADB06
:1028100059E09DF8B41001EB410000EB0110A14913
:1028200001EB001030309DF8A01000EB0110801C6F
:102830000990007820F008000830099908709DF888
:10284000B41001EB410000EB0110964901EB0010C0
:1028500030309DF8A01000EB011042682E9800EB7C
:102860004001914800EB4110C0F8232000203A902D
:1028700025E09DF8B41040F2833011FB00F0874949
:1028800001EB800101F589619DF8A00000EB400299
:1028900002EB001001EBC0014731BDF8E8000A5C13
:1028A0002E9800EB4001804800EB41112731BDF824
:1028B000E8000A54BDF8E800401C81B23A91BDF826
:1028C000E8000628D5DB00229DF8B40040F28331F1
:1028D00010FB01F0714901EB800101F589619DF860
:1028E000A00000EB400303EB001001EBC00080F8F8
:1028F00046209DF8B4100220F7F7D8FB9DF8B410DD
:1029000040F2833011FB00F1644800EB810101F5D6
:1029100089619DF8A00000EB400202EB001001EB82
:10292000C000223009902E9800EB40015E4800EB79
:1029300041110D3110220891DDE90801F5F785FC00
:102940009DF8B41040F2833011FB00F0534901EBC5
:10295000800101F589619DF8A00000EB400202EBC7
:10296000001001EBC0012E9800EB40024E4800EB36
:10297000421051F81A2F40F8012F496841609DF824
:10298000B41001EB410000EB0110464901EB0011CE
:1029900030319DF8A00001EB001001782E9800EB7B
:1029A0004002414800EB421001702E9800EB4001BC
:1029B0003D4800EB411100E08BE03C48026841F8E3
:1029C0001D2F808888809DF8B41040F2833011FB61
:1029D00000F0324901EB800101F589619DF8A0000A
:1029E00000EB400202EB001001EBC000416B2E989F
:1029F00000EB40022C4800EB4210C0F809109DF893
:102A0000B41001EB410000EB0110264901EB00116D
:102A100030319DF8A00001EB001041682E9800EBCA
:102A20004002214800EB4210C0F823102E9881B2DA
:102A300008200991F7F73AFB00229DF8B40040F214
:102A4000833110FB01F0154901EB800101F589612B
:102A50009DF8A00000EB400303EB001001EBC00069
:102A600080F84620A7229DF8B40040F2833110FB85
:102A700001F00A4901EB800101F589619DF8A00090
:102A800000EB400303EB001001EBC0004271A222F7
:102A90009DF8B40040F283310AE00000884800202D
:102AA000BC120020C8430020D8140020C7310020E9
:102AB00010FB01F0FE4901EB800000F589609DF8F4
:102AC000A01001EB410303EB011100EBC100827088
:102AD00000BF00BF0CF0F7B80021F64A9DF8B40023
:102AE00002EB00129DF8A00011549DF8B41001EB08
:102AF0004100C0EBC110F04901EBC00040787028E4
:102B00000ED19DF8B41001EB4100C0EBC110EA49B1
:102B100001EBC0008078FA2802D1B121259142E072
:102B20009DF8B41001EB4100C0EBC110E24901EB8C
:102B3000C000407800F0F000C0280ED19DF8B4101D
:102B400001EB4100C0EBC110DB4901EBC000807814
:102B5000FA2802D1B621259125E09DF8B41001EBA9
:102B60004100C0EBC110D44911F8300000F0F00072
:102B7000502818D19DF8B41001EB4100C0EBC110F2
:102B8000CD4901EBC000407800F0F00030280AD1B8
:102B90009DF8B41001EB4100C0EBC110C64901EB38
:102BA000C000817825919DF8B41040F2833011FB6C
:102BB00000F0BF4901EB8000817828910021BD4AD7
:102BC0009DF8B40002EB00129DF8A0001154BB4820
:102BD00090F82800012815D19DF8B41001EB4100B0
:102BE00000EB0110B64901EB001030309DF8A01049
:102BF00000EB0110801C0990007820F080008030EC
:102C000009990870BDF89400652876D004DC012885
:102C100009D0032805D17FE0B12802D0B62800D121
:102C200000E087E186E19DF8B41001EB4100C0EBC4
:102C3000C110A14901EBC0000079012806D002288B
:102C400005D0032804D0052864D102E062E061E0E9
:102C500060E09DF8B41040F2833011FB00F094491D
:102C600001EB800000F589609DF8A01001EB4102A6
:102C700002EB011110F83100F0BB00219DF8B40007
:102C800040F2833210FB02F0894A02EB80000171AE
:102C900001229DF8B40040F2833110FB01F0844919
:102CA00001EB800101F589619DF8A00000EB400374
:102CB00003EB001001F83020B6229DF8B40040F27A
:102CC000833110FB01F07A4901EB800101F5896144
:102CD0009DF8A00000EB400303EB001001EBC000E7
:102CE0004271B2229DF8B40040F2833110FB01F032
:102CF0006F4901EB800001E00BE035E000F58960F1
:102D00009DF8A01001EB410303EB011100EBC100A2
:102D1000827000BF00BF0DE19DF8B41001EB4100CF
:102D2000C0EBC110644901EBC000C179654880F86F
:102D3000031D9DF8B41001EB410000EB0110604948
:102D400001EB001130319DF8A00001EB0010801C58
:102D500009905C4890F8030DC2080998007862F366
:102D6000000009990870E5E09DF8B41001EB4100FE
:102D7000C0EBC110504901EBC000007900F0F00039
:102D800010B9B821259101E0B921259100213A918E
:102D900020E09DF8B41001EB410000EB0110484920
:102DA00001EB00113031BDF8E80001EB0010417873
:102DB0009DF8B40000EB4002C2EBC0103E4A12F88E
:102DC00030005038814200D112E0BDF8E800401CCC
:102DD00081B23A919DF8B41001EB410000EB011073
:102DE000374901EB0010C179BDF8E8008142D0DC21
:102DF00000BF9DF8B41040F2833011FB00F02C4965
:102E000001EB800000F589609DF8A01001EB410204
:102E100002EB011110F83100012834D100219DF896
:102E2000B40040F2833210FB02F0214A02EB800032
:102E3000017102229DF8B40040F2833110FB01F0D1
:102E40001B4901EB800101F589619DF8A00000EBB1
:102E5000400303EB001001F83020B9229DF8B400C4
:102E600040F2833110FB01F0114901EB800101F5C3
:102E700089619DF8A00000EB400303EB001001EB1B
:102E8000C000427155E09DF8B41040F2833011FB50
:102E900000F0074901EB800000F589609DF8A01063
:102EA00001EB410202EB011110F8310001280BE0A7
:102EB00088480020B8410020388F0020BC12002034
:102EC000C8430020BC22002033D100219DF8B4006B
:102ED00040F2833210FB02F0FE4A02EB80000171E7
:102EE00002229DF8B40040F2833110FB01F0F94951
:102EF00001EB800101F589619DF8A00000EB400322
:102F000003EB001001F83020B9229DF8B40040F224
:102F1000833110FB01F0EF4901EB800000F589607F
:102F20009DF8A01001EB410303EB011100EBC10080
:102F3000427100BF00BFCDE59DF8B41001EB410028
:102F400000EB0110E44901EB0010007B20B10128E7
:102F50007DD002287CD12DE3E0499DF8B40031F802
:102F60001000801F81B209919DF8B40000EB400170
:102F7000C1EBC010DA4901EBC000401C0890099970
:102F8000F6F7E2FC0022CDE930029DF8B40000EB38
:102F90004001C1EBC010D24901EBC002CF489DF8FF
:102FA000B41030F81100401F11180991042109983C
:102FB00020F096F9C217CDE92E022FA819C82E9934
:102FC0005940604001437DD1C64A9DF8B40002EBF0
:102FD000001001709DF8B40000EB4001C1EBC0107F
:102FE000BF4901EBC00001792591BDF8940031285B
:102FF00002D0452867D10CE1B8489DF8B41030F8EC
:1030000011001838412190FBF1F0C217C1B2CDE98F
:103010002E02B54880F8AC1000203A90EFE09DF801
:10302000B40000EB4001C1EBC010AD4901EBC001A1
:10303000BDF8E80000EB80101430095C9DF8B40086
:1030400000EB4000A84AAD3202EB800201E0E3E071
:10305000AFE2BDF8E80011549DF8B40000EB400168
:10306000C1EBC0109E4901EBC001BDF8E80000EBC8
:1030700080101A30014409910821099820F0EEF8D7
:103080008DED0E0A9DF8B4000E9900EB4000964AB3
:10309000E93202EB8012BDF8E80002EB001041605B
:1030A0009DF8B40000EB4001C1EBC0108C4901EB6E
:1030B000C001BDF8E80000EB8010323001440991F6
:1030C000082101E0A7E0A5E0099820F0C7F88DED00
:1030D0000E0A9DF8B4000E9900EB4000824AE932D6
:1030E00002EB8012BDF8E80002EB001001609DF8D1
:1030F000B40000EB4001C1EBC010794901EBC00105
:10310000BDF8E80000EB80103A3001440991082135
:10311000099820F0A3F88DED0E0A9DF8B4000E99E1
:1031200000EB4000704AE93202EB8012BDF8E80083
:1031300002EB001081609DF8B40000EB4001C1EB90
:10314000C010674901EBC001BDF8E80000EB80103A
:103150004230014409910821099820F07FF88DED53
:103160000E0A9DF8B4000E9900EB40005E4AE93269
:1031700002EB8012BDF8E80002EB0010C1609DF880
:10318000B40000EB400101EB0010534901EB0011CA
:103190003031BDF8E80001EB0010801C0990007888
:1031A00020F080008030099908709DF8B40000EB91
:1031B0004001C1EBC0104A4901EBC00247489DF8ED
:1031C000B41030F81100401E125C9DF8B40040F2BB
:1031D000833110FB01F03F4901EB800000F589606D
:1031E0009DF8A01001EB410303EB011100EBC100BE
:1031F00080F84420BDF8E800401C80B23A90BDF849
:10320000E8000021DDE92E34C01AA141FFF607AF26
:1032100000E000BF00BF02E39DF8B40000EB4001F6
:10322000C1EBC0102E4901EBC000407D9DF8B410E9
:1032300001EB4102C2EBC111294A02EBC101897DB8
:1032400040EA0120C217CDE92E029DF8B40000EB40
:103250004001C1EBC010224901EBC00109911521C9
:103260000998F6F755FB0022CDE930022FA819C8BE
:103270002E995940604001437ED19DF8B40000EB87
:103280004001C1EBC011164810F83100401EC1B218
:1032900028910021134A9DF8B40002EB00129DF81A
:1032A000A00011549DF8B40000EB40000E4AAD326E
:1032B00002EB80029DF8A00011549FED0C0A10EE65
:1032C000101A9DF8B40000EB4000074AE93202EB07
:1032D00080120DE088480020C8430020B8800020FC
:1032E000388F0020B8410020BC32002000000000D0
:1032F0009DF8A00002EB001041609DF8B40000EBC7
:103300004001C1EBC010FE4901EBC00081799DF87E
:10331000B40000EB4002C2EBC010F94A02EBC0005F
:10332000407941EA002000EE100AB8EEC00A9FED95
:10333000F51AC0EE010A9DF8B40000EB4001C1EBA4
:10334000C010114601EBC00001799DF8B40000EBFC
:103350004002C2EBC010EA4A02EBC000C07841EA6A
:10336000002000EE100AB8EEC00A30EE800A10EE1F
:10337000101A9DF8B40000E01BE100EB4000E24AA7
:1033800002EB80129DF8A00002EB001001609DF896
:10339000B40000EB4001C1EBC010D94901EBC00003
:1033A000817A9DF8B40000EB4002C2EBC010D44A11
:1033B00002EBC000407A41EA002000EE100AB8EEAD
:1033C000C00A9FEDD01AC0EE010A9DF8B40000EBD0
:1033D0004001C1EBC010114601EBC000017A9DF81D
:1033E000B40000EB4002C2EBC010C54A02EBC000C3
:1033F000C07941EA002000EE100AB8EEC00A30EEB3
:10340000800A10EE101A9DF8B40000EB4000BE4A8E
:1034100002EB80129DF8A00002EB001081609DF885
:10342000B40000EB4001C1EBC010B54901EBC00096
:10343000C07A00F0800060BB9DF8B40000EB400152
:10344000C1EBC010AE4901EBC000017B9DF8B40098
:1034500000EB4002C2EBC010A94A02EBC000C07AE8
:1034600041EA002000EE100AF8EEC00AB3EE001A9E
:1034700080EE810A10EE101A9DF8B40000EB4000B7
:10348000A14A02EB80129DF8A00002EB0010C1607F
:103490004CE09DF8B40000EB4001C1EBC01098492E
:1034A00001EBC000017B9DF8B40000EB4002C2EBD1
:1034B000C010934A02EBC000C07A41EA00204042AB
:1034C00080B200EE100AB8EEC00A8DED030A039830
:1034D000F5F724F99FED8D0B53EC102BCDE904018A
:1034E0009DED040B51EC100BF4F7FCFF9FED890BE5
:1034F00053EC102BCDE906019DED060B51EC100BA2
:10350000F4F77BFFCDE908019DED080B51EC100BA2
:10351000F5F717F99DF8B41001EB41017A4A02EB77
:1035200081129DF8A01002EB0111C8609DF8B41043
:1035300001EB410000EB0110784901EB0010303045
:103540009DF8A01000EB0110801C0990007820F07D
:1035500080008030099908709DF8B41001EB41009B
:10356000C0EBC110664901EBC000C27D9DF8B400FC
:1035700040F2833110FB01F0694901EB800000F556
:1035800089609DF8A01001EB410303EB011100EBF2
:10359000C10080F844209DF8B41001EB410000EB1D
:1035A00001105E4901EB0010C1795748E93880F8F5
:1035B000AC1034E19DF8B41001EB4100C0EBC11038
:1035C0004F4901EBC000C0799DF8B41001EB4102F6
:1035D000C2EBC1114A4A02EBC101097A40EA01205B
:1035E000C217CDE92E029DF8B41001EB4100C0EBEB
:1035F000C110434901EBC001099107210998F6F771
:1036000087F90022CDE930022FA815C82E99514024
:103610006040014372D19DF8B41001EB4100C0EB52
:10362000C110374911F83000401EC1B22891002165
:103630003C4A9DF8B40002EB001001709DF8B40004
:1036400000EB4000A2F64F6202EB80029DF8A00062
:1036500011549DF8B41001EB4100C0EBC110284992
:1036600001EBC000817908460191F4F7D1FFCDE963
:1036700002019DED021B9FED2C0B23F0F9FE8DED59
:10368000060B9DF8B41001EB4100C0EBC1101C49C2
:1036900001EBC00001799DF8B40000EB4002C2EBE1
:1036A000C010174A02EBC000C07841EA002000EECB
:1036B000100AB8EEC00A8DED030A0398F5F72EF84C
:1036C000CDE904019DED060B53EC102B9DED040B91
:1036D00051EC100BF4F706FFCDE908019DED080B46
:1036E00051EC100BF5F72DF89DF8B41001EB4101EA
:1036F000054A02EB81129DF8A01019E08EE000004F
:10370000388F002000FF7F47A53300200000000015
:10371000000030400000000000000000C84300200E
:1037200088480020B841002000000000000024402C
:1037300002EB011148609FEDFC0A10EE102A9DF883
:10374000B40000EB4000F94901EB80119DF8A000A6
:1037500001EB001002609FEDF40A10EE101A9DF8C4
:10376000B40000EB4000F14A02EB80129DF8A0008B
:1037700002EB001081609FEDEC0A10EE101A9DF82C
:10378000B40000EB4000E94A02EB80129DF8A00073
:1037900002EB0010C1609DF8B41001EB410000EB9A
:1037A0000110E34901EB001130319DF8A00001EB5D
:1037B0000010801C0990007820F08000803009996A
:1037C00008709DF8B41001EB4100C0EBC111D9485D
:1037D00000EBC100427A9DF8B40040F2833110FB47
:1037E00001F0D54901EB800000F589609DF8A0103B
:1037F00001EB410303EB011100EBC10080F8442011
:103800009DF8B40000EB400101EB0010C84901EB4A
:103810000010C179C548E93880F8AC1000BF00BF7E
:103820000BF051BA9DF8B40000EB4001C1EBC010A1
:10383000C04901EBC000C1789DF8B40000EB400224
:10384000C2EBC010BB4A02EBC000807841EA002105
:1038500029919DF8B40000EB4001C1EBC010114666
:1038600001EBC001BDF8A400401C095C9DF8B40048
:1038700000EB4002C2EBC010AE4A02EBC002BDF842
:10388000A400105C41EA0020C217CDE92E029DF889
:10389000B40000EB4001C1EBC010A64901EBC00031
:1038A0000990BDF8A410F6F733F80022CDE93002F4
:1038B0002FA819C82E9959406040014341F06C86E9
:1038C0009DF8B40000EB4001C1EBC010994901EB39
:1038D000C0004178289100213A911CE09DF8B40085
:1038E00000EB400101EB0010914901EB0011303178
:1038F000BDF8E80001EB001041789DF8A00081427E
:1039000004D1BDF8E800C1B2289112E0BDF8E8008A
:10391000401C81B23A919DF8B40000EB400101EBEC
:103920000010834901EB0010C179BDF8E800814225
:10393000D4DC00BF9DF8B40000EB400101EB0010A7
:103940007B4901EB001030309DF8A01000EB011016
:10395000801C0990007820F0800080300999087060
:103960009DF8B40000EB4001C1EBC010714901EBC0
:10397000C000007925900020704A9DF8B41002EB39
:1039800001129DF8A0105054BDF89400F3287DD08A
:1039900009DC05287BD006280ED0F12878D0F22843
:1039A00041F0F985FCE3F42873D0F62872D0F728AB
:1039B00071D0F828F4D1F4E306211091002136915A
:1039C000F0E3BDF84000401C81B210919DF8B400B6
:1039D00000EB4001C1EBC010564901EBC001BDF83E
:1039E0004000095C2591BDF84000401C81B2109157
:1039F000BDF89400F12804D0F22868D0F32867D1EC
:103A0000FEE39DF8B40000EB4001C1EBC010494952
:103A100001EBC001BDF84000095C2991BDF84000F0
:103A2000401C81B210919DF8B40000EB400101EB05
:103A300000103F4901EB001130319DF8A020BDF886
:103A4000D800104401EB0010407A00F00100E8B308
:103A50009DF8B40040F2833110FB01F0364901EBD0
:103A6000800101F589619DF8A020BDF8D8001044BF
:103A700000EB400202EB001001EBC00090F8900058
:103A800000F0010010BB9DF8B40005E0FEE3FEE38A
:103A9000FEE3FEE3FEE3FEE340F2833110FB01F0C0
:103AA000254901EB800101F589619DF8A020BDF851
:103AB000D800104400EB400202EB001001EBC00004
:103AC00090F8820010B100213A913EE0A0E0FDE3C1
:103AD000FDE39DF8B40040F2833110FB01F016497C
:103AE00001EB800101F589619DF8A020BDF8D800A7
:103AF000104400EB400202EB001001EBC00000F1AB
:103B00008301BDF8E8000A5C9DF8B40000EB4001B9
:103B100001EB0010064901EB00100E30BDF8E81073
:103B2000405C82420CD014E000000000A53300206D
:103B3000C8430020388F002088480020B84100206A
:103B4000BDF8E800401C81B23A91BDF8E8000428B5
:103B5000BFDB00BFBDF8E800042859D104213A9129
:103B60002FE09DF8B40040F2833110FB01F0FE49D4
:103B700001EB800101F589619DF8A020BDF8D80016
:103B8000104400EB400202EB001001EBC00000F11A
:103B90008301BDF8E8000A5C9DF8B40000EB400129
:103BA00001EB0010F14901EB00100E30BDF8E810F8
:103BB000405C824200D008E0BDF8E800401C81B2C1
:103BC0003A91BDF8E8000A28CBDB00BFBDF8E80059
:103BD0000A281DD09DF8B40040F2833110FB01F09B
:103BE000E14901EB800000F589609DF8A020BDF857
:103BF000D810114401EB410202EB011100EBC100AE
:103C000090300990007820F00100401C099908705C
:103C1000BDF8A4000F287CD19DF8B40000EB400152
:103C200001EB0010D14901EB001030309DF8A020CD
:103C3000BDF8D810114400EB0110801C09900078E9
:103C400020F00400001D0999087000203A902DE032
:103C50009DF8B40000EB4001C1EBC010C44901EB7A
:103C6000C001BDF84020BDF8E80010440A5C9DF892
:103C7000B40040F2833110FB01F0BB4901EB80013D
:103C800001F589619DF8A030BDF8D800184400EB1B
:103C9000400303EB001001EBC0014731BDF8E80021
:103CA0000A54BDF8E800401C81B23A91BDF8E80022
:103CB0000A28CDDBBDF840000A3081B21091002106
:103CC0003A912FE09DF8B40000EB4001C1EBC01029
:103CD000A74901EBC001BDF84020BDF8E800104441
:103CE0000A5C9DF8B40040F2833110FB01F09E495C
:103CF00001EB800101F589619DF8A030BDF8D80085
:103D0000184400EB400303EB001001EBC0016031ED
:103D100000E07DE2BDF8E8000A54BDF8E800401C70
:103D200081B23A91BDF8E8000228CBDBBDF8400033
:103D3000801C81B210919DF8B40000EB4001C1EBF2
:103D4000C0108B4901EBC001BDF84000085C0104C4
:103D50009DF8B40000EB4002C2EBC010844A02EBB5
:103D6000C002BDF84000401C105C41EA00219DF8F3
:103D7000B40000EB4002C2EBC0107D4A02EBC0026F
:103D8000BDF84000801C105C01439DF8B40040F277
:103D9000833210FB02F0744A02EB800202F5896262
:103DA0009DF8A030BDF8D800184400EB400303EBA9
:103DB000001002EBC0004167BDF84000C01C81B29A
:103DC00010916C4890F8100BF0BB00213A9120E064
:103DD0009DF8B40040F2833110FB01F0624901EB21
:103DE000800101F589619DF8A020BDF8D80010443C
:103DF00000EB400202EB001001EBC0004730BDF8C1
:103E0000E810405C00B108E0BDF8E800401C81B259
:103E10003A91BDF8E8000A28DADB00BFBDF8E800F7
:103E20000A281BD140229DF8B40040F2833110FBD8
:103E300001F04D4901EB800101F589619DF8A03049
:103E4000BDF8D800184400E05FE000EB400303EB4E
:103E5000001001EBC00080F87E2069E19DF8B400FD
:103E600040F2833110FB01F03F4901EB800101F585
:103E700089619DF8A020BDF8D800104400EB4002F5
:103E800002EB001001EBC00090F87E00E8BB0021BF
:103E90002A9124E1002137912CE09DF8B40040F2F2
:103EA000833110FB01F0304901EB800101F589619C
:103EB0009DF8A020BDF8D800104400EB400202EBB2
:103EC000001001EBC0014731BDF8DC00001D095CAA
:103ED0009DF8A80000EB4002274800EB4202BDF825
:103EE000DC00105C814200D008E0BDF8DC00401C22
:103EF00081B23791BDF8DC000628CEDB00BFBDF8EB
:103F0000DC0006287ED1032200E011E19DF8B40018
:103F100040F2833110FB01F0134901EB800101F500
:103F200089619DF8A030BDF8D800184400EB40032B
:103F300003EB001001EBC00080F87E209DF8B40078
:103F400000EB400101EB0010084901EB001130319A
:103F50009DF8A020BDF8D800104401EB0010801C93
:103F6000099000780AE0000088480020C84300203B
:103F7000388F0020BC320020B837002020F0040227
:103F80000998027000203A901FE020229DF8B400AA
:103F900040F2833110FB01F0FC4901EB800101F597
:103FA00089619DF8A030BDF8D800184400EB4003AB
:103FB00003EB001001EBC0015131BDF8E8000A54D9
:103FC000BDF8E800401C81B23A91BDF8E8000F2826
:103FD000DBDB00213A9121E020229DF8B40040F281
:103FE000833110FB01F0E94901EB800101F58961A2
:103FF0009DF8A030BDF8D800184400EB400303EB57
:10400000001000E066E001EBC0016331BDF8E8009C
:104010000A54BDF8E800401C81B23A91BDF8E800AE
:104020000A28D9DB00229DF8B40040F2833110FB4E
:1040300001F0D64901EB800101F589619DF8A030BE
:10404000BDF8D800184400EB400303EB001001EB6F
:10405000C00080F8782000213A911FE000229DF8EE
:10406000B40040F2833110FB01F0C84901EB80013C
:1040700001F589619DF8A030BDF8D800184400EB27
:10408000400303EB001001EBC0017931BDF8E800FB
:104090000A54BDF8E800401C81B23A91BDF8E8002E
:1040A0000528DBDB9DF8B40040F2833110FB01F002
:1040B000B64901EB800101F589619DF8A020BDF8AA
:1040C000D800104400EB400202EB001001EBC000EE
:1040D000406F0CE09DF8A800401CC1B22A91AC488A
:1040E000B0F8FA049DF8A81088423FF7D3AE00BF9D
:1040F000A748B0F8FA049DF8A810884218D14022C9
:104100009DF8B40040F2833110FB01F09F4901EBB0
:10411000800101F589619DF8A030BDF8D8001844F0
:1041200000EB400303EB001001EBC00080F87E20A1
:104130009DF8B40040F2833110FB01F0934901EB8C
:10414000800101F589619DF8A020BDF8D8001044D8
:1041500000EB400202EB001001EBC00090F87E0083
:10416000032804D011281ED0402850D134E0F22278
:104170009DF8B40040F2833110FB01F0834901EB5C
:10418000800101F589619DF8A030BDF8D800184480
:1041900000EB400303EB001001EBC000427136E07E
:1041A000F1E3F1E317E1F3229DF8B40040F283312B
:1041B00010FB01F0754901EB800101F589619DF863
:1041C000A030BDF8D800184400EB400303EB00100A
:1041D00001EBC00042711AE0F2229DF8B40040F2F7
:1041E000833110FB01F0694901EB800101F5896120
:1041F0009DF8A030BDF8D800184400EB400300E063
:10420000CAE003EB001001EBC000427100BF6EE09A
:104210009DF8B40000EB400101EB00105D4901EB9B
:10422000001130319DF8A020BDF8D800104401EBFA
:104230000010801C0990007820F004020998027098
:104240009DF8B40040F2833110FB01F04F4901EBBF
:10425000800000F589609DF8A020BDF8D8101144B9
:1042600001EB410202EB011100EBC10090F890005C
:1042700000F0010060B300229DF8B40040F28331E9
:1042800010FB01F0414901EB800105E0FEE3FEE394
:10429000B1E0FDE3FDE3FDE301F589619DF8A030A8
:1042A000BDF8D800184400EB400303EB001001EB0D
:1042B000C000A0F88E2005229DF8B40040F28331A2
:1042C00010FB01F0314901EB800102E010E07CE0DD
:1042D0000DE001F589619DF8A030BDF8D8001844C3
:1042E00000EB400303EB001001EBC00042716CE0F7
:1042F0009DF8B40040F2833110FB01F0234901EB3B
:10430000800101F589619DF8A020BDF8D800104416
:1043100000EB400202EB001001EBC00090F87E00C1
:10432000402819D100229DF8B40040F2833110FBDF
:1043300001F0164901EB800101F589619DF8A0307B
:10434000BDF8D800184400EB400303EB001001EB6C
:10435000C00080F87E2000BF00BFF1229DF8B400AD
:1043600040F2833110FB01F0084901EB800101F5B7
:1043700089619DF8A030BDF8D800184400EB4003D7
:1043800003EB001001EBC00042711EE088480020E2
:10439000BC320020C8430020F1229DF8B40040F256
:1043A000833110FB01F0FE4901EB800101F58961C9
:1043B0009DF8A030BDF8D800184400EB400303EB93
:1043C000001001EBC000427100BF00BFBDF8D80073
:1043D000401C81B236919DF8B40000EB4001C1EB66
:1043E000C010F04901EBC0004179BDF8D80081420E
:1043F0003FF7E7AAE8E39DF8B40040F2833110FBF1
:1044000001F0E74901EB800000F589609DF8A010FC
:1044100001EB410202EB011110F8310048BB01220F
:104420009DF8B40040F2833110FB01F0DC4901EB50
:10443000800101F589619DF8A00000EB400303EBCA
:10444000001001F83020F4229DF8B40040F28331CE
:1044500010FB01F0D24901EB800000F589609DF866
:10446000A01001EB410303EB011100EBC10042710D
:10447000CCE09DF8B40000EB400101EB0010CA490C
:1044800001EB001030309DF8A01000EB0110407AD5
:1044900000F0010080B39DF8B40040F2833110FBBE
:1044A00001F0BF4901EB800000F589609DF8A01084
:1044B00001EB410202EB011100EBC10090F890000A
:1044C00000F00100C0B99DF8B40040F2833110FB48
:1044D00001F0B34901EB800000F589609DF8A01060
:1044E00001EB410202EB011100EBC10090F88200E8
:1044F00010B100203A902DE088E09DF8B40040F221
:10450000833110FB01F0A64901EB800101F58961BF
:104510009DF8A00000EB400202EB001001EBC00090
:1045200000F18301BDF8E8000A5C9DF8B40000EBDF
:10453000400101EB00109C4901EB00110E31BDF868
:10454000E800085C824200D008E0BDF8E800401CAA
:1045500081B23A91BDF8E8000428CEDB00BFBDF877
:10456000E800042852D13A902CE09DF8B40040F2C3
:10457000833110FB01F08A4901EB800101F589616B
:104580009DF8A00000EB400202EB001001EBC00020
:1045900000F18301BDF8E8000A5C9DF8B40000EB6F
:1045A000400101EB0010804901EB00110E31BDF814
:1045B000E800085C824200D008E0BDF8E800401C3A
:1045C00081B23A91BDF8E8000A28CEDB00BFBDF801
:1045D000E8000A281AD09DF8B40040F2833110FB9D
:1045E00001F06F4901EB800000F589609DF8A01093
:1045F00001EB410202EB011100EBC1009030099088
:10460000007820F00100401C09990870BDF8A40052
:10461000112877D19DF8B40000EB400101EB0010A8
:10462000614901EB001030309DF8A01000EB011043
:10463000801C0990007820F00400001D0999087082
:1046400000203A9028E09DF8B40000EB4001C1EB57
:10465000C010544901EBC001BDF8E800401D0A5CE0
:104660009DF8B40040F2833110FB01F04C4901EB9E
:10467000800101F589619DF8A00000EB400303EB88
:10468000001001EBC0014731BDF8E8000A54BDF845
:10469000E800401C81B23A91BDF8E8000A28D2DB5C
:1046A00000203A9028E09DF8B40000EB4001C1EBF7
:1046B000C0103C4901EBC001BDF8E8000F300A5CB6
:1046C0009DF8B40040F2833110FB01F0344901EB56
:1046D000800101F589619DF8A00000EB400303EB28
:1046E000001001EBC0016031BDF8E8000A54BDF8CC
:1046F000E800401C81B23A91BDF8E8000228D2DB04
:10470000B0E2FFE7BDF8A40014287DD19DF8B40005
:1047100000EB400101EB0010234901EB00103030A9
:104720009DF8A01000EB0110801C0990007820F08B
:104730000400001D0999087000203A9028E09DF8B7
:10474000B40000EB4001C1EBC010164901EBC00101
:10475000BDF8E800401D0A5C9DF8B40040F28331CA
:1047600010FB01F00E4901EB800101F589619DF814
:10477000A00000EB400303EB001001EBC001473148
:10478000BDF8E8000A54BDF8E800401C81B23A9137
:10479000BDF8E8000A28D2DB00203A902FE00000A4
:1047A00088480020388F0020C84300209DF8B400BE
:1047B00000EB4001C1EBC010FE4901EBC001BDF8A8
:1047C000E8000F300A5C9DF8B40040F2833110FB22
:1047D00001F0F94901EB800101F589619DF8A00024
:1047E00000EB400303EB001001EBC0016031BDF8AA
:1047F000E8000A54BDF8E800401C81B23A91BDF8C7
:10480000E8000228D2DB00E02DE29DF8B40000EBC6
:104810004001C1EBC010E74901EBC000407C01043E
:104820009DF8B40000EB4002C2EBC010E14A02EB7D
:10483000C000807C41EA00219DF8B40000EB4002FA
:10484000C2EBC010DB4A02EBC000C07C01439DF804
:10485000B40040F2833210FB02F0D74A02EB800032
:1048600000F589609DF8A02002EB420303EB0212E1
:1048700000EBC2004167D14890F8100BF0BB00205C
:104880003A901DE09DF8B40040F2833110FB01F036
:10489000C94901EB800101F589619DF8A00000EB99
:1048A000400202EB001001EBC0004730BDF8E810F9
:1048B000405C00B108E0BDF8E800401C81B23A91CC
:1048C000BDF8E8000A28DDDB00BFBDF8E8000A28D3
:1048D00018D140229DF8B40040F2833110FB01F062
:1048E000B54901EB800000F589609DF8A01001EB4F
:1048F000410303EB011100EBC10000E045E080F84B
:104900007E2045E19DF8B41040F2833011FB00F0A9
:10491000A94901EB800000F589609DF8A01001EB2A
:10492000410202EB011100EBC10090F87E0060BB78
:1049300000212A9106E1002137912CE09DF8B41066
:1049400040F2833011FB00F09B4901EB800101F53F
:1049500089619DF8A00000EB400202EB001001EB22
:10496000C0014731BDF8DC00001D095C9DF8A800BE
:1049700000EB4002924800EB4202BDF8DC00105C04
:10498000814203D00BE0FDE3FDE301E1BDF8DC0073
:10499000401C81B23791BDF8DC000628CEDB00BF99
:1049A000BDF8DC00062876D103229DF8B40040F261
:1049B000833110FB01F0804901EB800101F5896131
:1049C0009DF8A00000EB400303EB001001EBC000DA
:1049D00080F87E209DF8B41001EB410000EB01103F
:1049E000784901EB001130319DF8A00001EB001077
:1049F000801C0990007820F00402099802700020C1
:104A00003A901CE020229DF8B40040F2833110FB64
:104A100001F0694901EB800101F589619DF8A00071
:104A200000EB400303EB001001EBC0015131BDF876
:104A3000E8000A54BDF8E800401C81B23A91BDF884
:104A4000E8000F28DEDB00213A911CE020229DF8CF
:104A5000B40040F2833110FB01F0574901EB8001B3
:104A600001F589619DF8A00000EB400303EB001005
:104A700001EBC0016331BDF8E8000A54BDF8E8005D
:104A8000401C81B23A91BDF8E80005E0FDE3FDE38A
:104A9000FDE3FDE3EAE350E00A28D7DB00229DF8BE
:104AA000B40040F2833110FB01F0434901EB800177
:104AB00001F589619DF8A00000EB400303EB0010B5
:104AC00001EBC00080F8782000213A911CE0002220
:104AD0009DF8B40040F2833110FB01F0364901EB40
:104AE000800101F589619DF8A00000EB400303EB14
:104AF000001001EBC0017931BDF8E8000A54BDF89F
:104B0000E800401C81B23A91BDF8E8000528DEDBE0
:104B10009DF8B41040F2833011FB00F0264901EB00
:104B2000800000F589609DF8A01001EB410202EBC6
:104B3000011100EBC100406F0CE09DF8A800401C83
:104B4000C1B22A911D48B0F8FA049DF8A810884215
:104B50003FF7F1AE00BF1948B0F8FA149DF8A8006D
:104B6000814215D140229DF8B40040F2833110FB00
:104B700001F0114901EB800000F589609DF8A0105B
:104B800001EB410303EB011100EBC10080F87E2033
:104B90009DF8B41040F2833011FB00F0064901EBA0
:104BA000800000F589609DF8A01001EB410202EB46
:104BB00001110AE0388F002088480020BC32002014
:104BC000B8370020C84300204EE300EBC10090F846
:104BD0007E00032804D0112818D0402842D12BE0B1
:104BE000F2229DF8B40040F2833110FB01F0FE493F
:104BF00001EB800000F589609DF8A01001EB4103F6
:104C000003EB011100EBC10042712BE0F3229DF890
:104C1000B40040F2833110FB01F0F34901EB800056
:104C200000F589609DF8A01001EB410303EB011131
:104C300000EBC100427115E0F2229DF8B40040F291
:104C4000833110FB01F0E84901EB800000F5896039
:104C50009DF8A01001EB410303EB011100EBC10033
:104C6000427100BF00E3BDF8A40006287DD19DF885
:104C7000B41001EB4100C0EBC110DC4901EBC000F6
:104C80004079012872D10320D9490870F7229DF894
:104C9000B40040F2833110FB01F0D34901EB8001F5
:104CA00001F589619DF8A00000EB400303EB0010C3
:104CB00001EBC00042719DF8B41040F2833011FB4B
:104CC00000F0C94901EB800101F589619DF8A00060
:104CD00000EB400202EB001001EBC00090F88010E6
:104CE00001EB410000EB0110C24901EB0011303132
:104CF0009DF8B40040F2833210FB02F0BA4A02EB96
:104D0000800000F589609DF8A02002EB420303EBD0
:104D1000021200EBC20090F8810001EB00108078D5
:104D2000C0F34000F0B39DF8B41040F2833011FBA3
:104D300000F0AD4901EB800000F589609DF8A010FE
:104D400001EB410202EB011100EBC10090F8801071
:104D500001EB410000EB0110A64901EB0010807946
:104D6000012804D00A287CD13FE025E2CDE0BA2317
:104D70009DF8B40040F2833110FB01F09A4901EB39
:104D8000800101F589619DF8A00000EB400202EB73
:104D9000001001EBC00090F8800040F2833110FB5E
:104DA00001F000E01FE1904901EB800101F589610C
:104DB0009DF8B40040F2833210FB02F08A4A02EB05
:104DC000800000F589609DF8A02002EB420404EB0E
:104DD000021200EBC20090F8810000EB400202EBEF
:104DE000001001EBC00043713BE00B239DF8B400C1
:104DF00040F2833110FB01F07B4901EB800101F5AA
:104E000089619DF8A00000EB400202EB001001EB6D
:104E1000C00090F8800040F2833110FB01F072492D
:104E200001EB800101F589619DF8B40040F2833205
:104E300010FB02F06C4A02EB800000F589609DF8DF
:104E4000A02002EB420404EB021200EBC20090F837
:104E5000810000EB400202EB001001EBC000437147
:104E600000BF00BF9DF8B41040F2833011FB00F08A
:104E70005D4901EB800101F589619DF8A00000EB1F
:104E8000400202EB001001EBC00090F8801001EB33
:104E9000410000EB0110574901EB001130319DF842
:104EA000B40040F2833210FB02F04F4A02EB800262
:104EB00002F589629DF8A00000EB400303EB0010AF
:104EC00002EBC00090F8810001EB001002789DF821
:104ED000B40040F2833110FB01F0434901EB800044
:104EE00000F589609DF8A01001EB410303EB01116F
:104EF00000EBC10090F8800040F2833110FB01F01C
:104F0000394901EB80004270AEE19DF8B41001EB2D
:104F10004100C0EBC110354901EBC00040790228C7
:104F200061D1042032490870F8229DF8B40040F2A3
:104F3000833110FB01F02C4901EB800101F58961FF
:104F40009DF8A00000EB400303EB001001EBC00054
:104F500042719DF8B41040F2833011FB00F02249F9
:104F600001EB800101F589619DF8A00000EB400292
:104F700002EB001001EBC00090F8801001EB410043
:104F800000EB01101B4901EB001130319DF8B4001A
:104F900040F2833210FB02F0134A02EB800000F56E
:104FA00089609DF8A02002EB420303EB021200EBA4
:104FB000C20090F8810001EB00108078C0F340003F
:104FC00088B19DF8B41040F2833011FB00F006491F
:104FD00001EB800000F589609DF8A01001EB410213
:104FE00002EB011108E03FE188480020388F0020E3
:104FF00019020020C843002000EBC10090F8801087
:1050000001EB410000EB0110FE4901EB001080793B
:10501000012802D00A2878D13BE0B3239DF8B400E0
:1050200040F2833110FB01F0F74901EB800101F5FB
:1050300089619DF8A00000EB400202EB001001EB3B
:10504000C00090F8800040F2833110FB01F0EE497F
:1050500001EB800101F589619DF8B40040F28332D3
:1050600010FB02F0E84A02EB800000F589609DF831
:10507000A02002EB420404EB021200EBC20090F805
:10508000810000EB400202EB001001EBC000437115
:105090003BE00C239DF8B40040F2833110FB01F09B
:1050A000D94901EB800101F589619DF8A00000EB71
:1050B000400202EB001001EBC00090F8800040F2CB
:1050C000833110FB01F0D04901EB800101F58961CA
:1050D0009DF8B40040F2833210FB02F0CA4A02EBA2
:1050E000800000F589609DF8A02002EB420404EBEB
:1050F000021200EBC20090F8810000EB400202EBCC
:10510000001001EBC000437100BF00BF9DF8B40068
:1051100040F2833110FB01F0BB4901EB800101F546
:1051200089619DF8A00000EB400202EB001001EB4A
:10513000C00090F8800000EB400101EB0010B14985
:1051400001EB001130319DF8B40040F2833210FBC6
:1051500002F0AD4A02EB800202F589629DF8A000E0
:1051600000EB400303EB001002EBC00090F881005D
:1051700001EB001002789DF8B40040F2833110FB7F
:1051800001F001E08DE070E09F4901EB800000F547
:1051900089609DF8A01001EB410303EB011100EBC6
:1051A000C10090F8800040F2833110FB01F0964975
:1051B00001EB8000427057E09DF8B40000EB400125
:1051C00001EB00108F4901EB001030309DF8A0106A
:1051D00000EB0110801C0990007820F0040209986F
:1051E00002709DF8B40040F2833110FB01F0864953
:1051F00001EB800000F589609DF8A01001EB4102F1
:1052000002EB011100EBC10090F8900000F00100EA
:1052100050B300229DF8B40040F2833110FB01F03E
:10522000794901EB800101F589619DF8A00000EB4F
:10523000400303EB001001EBC000A0F88E20052214
:105240009DF8B40040F2833110FB01F06E4901EB90
:10525000800000F589609DF8A01001EB410303EB8D
:10526000011100EBC100427195E100BFF1229DF8F0
:10527000B40040F2833110FB01F0634901EB800080
:1052800000F589609DF8A01003E04FE007E18DE094
:1052900062E001EB410303EB011100EBC10042713D
:1052A00079E19DF8B40040F2833110FB01F05649DA
:1052B00001EB800000F589609DF8A01001EB410230
:1052C00002EB011100EBC10090F87E00402816D1DE
:1052D00000229DF8B40040F2833110FB01F04A49EE
:1052E00001EB800000F589609DF8A01001EB4103FF
:1052F00003EB011100EBC10080F87E2000BF00BF6E
:10530000F1229DF8B40040F2833110FB01F03E49D8
:1053100001EB800000F589609DF8A01001EB4103CE
:1053200003EB011100EBC100427134E1F1229DF861
:10533000B40040F2833110FB01F0334901EB8000EF
:1053400000F589609DF8A01001EB410303EB01110A
:1053500000EBC10042711EE103229DF8B40040F24F
:10536000833110FB01F0284901EB800101F58961CF
:105370009DF8A00000EB400303EB001001F8302083
:10538000F1229DF8B40040F2833110FB01F01E4978
:1053900001EB800000F589609DF8A01001EB41034E
:1053A00003EB011100EBC1004271F4E002229DF811
:1053B000B40040F2833110FB01F0134901EB80018E
:1053C00001F589619DF8A00000EB400303EB00109C
:1053D00001F83020F6229DF8B40040F2833110FB32
:1053E00001F0094901EB800101F589619DF8A000F8
:1053F00000EB400303EB001001EBC00042710122FF
:1054000004E00000C8430020884800209DF8B40054
:1054100040F2833110FB01F0FE4901EB800101F500
:1054200089619DF8A00000EB400303EB001001EB45
:10543000C00080F8822000213A9129E09DF8B40054
:1054400000EB4001C1EBC010F34901EBC001BDF816
:10545000E800401D0A5C9DF8B40040F2833110FB67
:1054600001F0EC4901EB800101F589619DF8A00094
:1054700000EB400303EB001001EBC00000F18301DF
:10548000BDF8E8000A54BDF8E800401C81B23A912A
:10549000BDF8E8000A28D1DBBDF8A4007BE09DF848
:1054A000B40000EB4001C1EBC010DB4901EBC000D0
:1054B00081799DF8B40000EB4002C2EBC010D64ADF
:1054C00002EBC000407941EA00229DF8B40040F2AE
:1054D000833110FB01F0CF4901EB800101F58961B7
:1054E0009DF8A00000EB400303EB001001EBC000AF
:1054F000A0F88E209DF8B40040F2833110FB01F03B
:10550000C44901EB800101F589619DF8A00000EB21
:10551000400202EB001001EBC000B0F88E109DF8C5
:10552000B40000EB400202EB0010BC4A02EB00109A
:10553000408B81422EDBF1229DF8B40040F2833192
:1055400010FB01F0B34901EB800101F589619DF881
:10555000A00000EB400303EB001001EBC000427120
:105560009DF8B40040F2833110FB01F0A94901EB32
:10557000800000F589609DF8A01001EB410202EB6C
:10558000011100EBC10090300990007820F0010279
:105590000998027000BF00BF09F095BB9DF8B400E8
:1055A00000EB4001C1EBC0109B4901EBC000017949
:1055B0002891002136911CE09DF8B40000EB4001D9
:1055C00001EB0010954901EB00113031BDF8D80016
:1055D00001EB001041789DF8A000814204D1BDF894
:1055E000D800C1B2289112E0BDF8D800401C81B2A9
:1055F00036919DF8B40000EB400101EB00108749A3
:1056000001EB0010C179BDF8D8008142D4DC00BFA5
:105610009DF8B40000EB4001C1EBC0107E4901EBE6
:10562000C000C1782591BDF89400172834D2DFE876
:1056300000F0330C0F331215181B1E333333333382
:105640003321242733332A2D30000720299023E0EB
:105650000720299020E0062029901DE006202990AF
:105660001AE00620299017E01220299014E0072064
:10567000299011E0092029900EE0062029900BE0E6
:105680000620299008E00B20299005E00B202990A6
:1056900002E02A20299000BF00BFBDF8A400001F2F
:1056A000C1B209919DF8B40000EB4001C1EBC010FC
:1056B000594901EBC000C01C08900999F3F70AFF93
:1056C00037909DF8B40000EB4001C1EBC010524987
:1056D00001EBC001BDF8A400401E095CBDF8DC0070
:1056E00081427DD19DF8B40000EB4001C1EBC010B8
:1056F000494901EBC0004078002871DD9DF8B400F5
:1057000000EB4001C1EBC010434901EBC001BDF803
:10571000A4000A5C9DF8B40040F2833110FB01F054
:105720003C4901EB800101F589619DF8A00000EB87
:10573000400303EB001001EBC00080F8442000217F
:10574000374A9DF8B40002EB00129DF8A0001154F6
:10575000344890F82800012815D19DF8B40000EBDA
:10576000400101EB00102D4901EB001030309DF895
:10577000A01000EB0110801C0990007820F0800040
:10578000803009990870BDF8940007287ED00ADCA3
:1057900007287CD2DFE810F07B006A06D1067B0088
:1057A00054061D06D40C10380728F2D2DFE810F09A
:1057B000360D200D6F006F0007000800FC0600BFCB
:1057C000BDF8940014287DD19DF8B40000EB400191
:1057D000C1EBC010104901EBC0004079010600E0A8
:1057E000FEE39DF8B40000EB4002C2EBC0100A4A91
:1057F00002EBC000807941EA00419DF8B40000EB63
:105800004002C2EBC010044A02EBC000C07941EA7A
:10581000002109E088480020388F0020C84300207C
:10582000B8410020BC1200209DF8B40000EB4002FB
:10583000C2EBC010FE4A02EBC000007A01439DF8A3
:10584000B40040F2833210FB02F0FA4A02EB80020D
:1058500002F589629DF8A00000EB400303EB001005
:1058600002EBC000C0F81A109DF8B40040F283317A
:1058700010FB01F0EF4901EB800101F589619DF812
:10588000A00000EB400202EB001001E0F0E3F0E3C7
:1058900001EBC000D0F81A1008460991002112F05F
:1058A0004BFACDE92E019DF8B40000EB400101EB6D
:1058B0000010E14901EB0010007F00F003019DF8AA
:1058C000B40000E07BE000EB400202EB0010DA4A9B
:1058D00002EB0010007FC0F3011001449DF8B400FA
:1058E00000EB400202EB0010D34A02EB0010007FF5
:1058F000C0F38100091A08460591F2F778FECDE958
:1059000006019DED061B9FEDCD0B21F0B1FD8DED48
:10591000080B9DED080B51EC100BF2F7DAFECDE908
:1059200030019DF8B40040F2833110FB01F0C14911
:1059300001EB800101F589619DF8A00000EB4002B8
:1059400002EB001001EBC000416B084607910021FB
:1059500012F0F2F9DDE92E32A0FB034501FB035101
:1059600000FB021502220023DDE93001F2F72AFCD8
:10597000231845EB0100CDE90830DDE93023DDE9EE
:105980000801F2F71FFCCDE92E01DDE92E0112F02E
:1059900087FF9DF8B41040F2833211FB02F1A54A53
:1059A00002EB810101F589619DF8A02002EB420321
:1059B00003EB021201EBC201C1F81E0046E0BDF884
:1059C0009400152842D19DF8B40000EB4001C1EBD2
:1059D000C010974901EBC000407901069DF8B40062
:1059E00000EB4002C2EBC010914A02EBC00080798C
:1059F00041EA00419DF8B40000EB4002C2EBC01048
:105A00008B4A02EBC000C07941EA00219DF8B40046
:105A100000EB4002C2EBC010854A02EBC000007AE6
:105A200001439DF8B40040F2833210FB02F0814A3A
:105A300002EB800000F589609DF8A02002EB420394
:105A400003EB021200EBC200C0F81E109DF8B40078
:105A500000EB4001C1EBC010754901EBC000427A78
:105A60009DF8B40040F2833110FB01F0714901EB65
:105A7000800101F589619DF8A00000EB400303EB74
:105A8000001001EBC00080F894209DF8B40000EBFA
:105A9000400101EB0010684901EB001030309DF827
:105AA000A01000EB0110801C09909DF8B40040F29A
:105AB000833110FB01F15F4800EB810000F5896044
:105AC0009DF8A01001EB410202EB011100EBC100B7
:105AD00090F89400C2090998017862F300010170FE
:105AE0009DF8B40040F2833110FB01F0514901EB05
:105AF000800000F589609DF8A01001EB410202EBE7
:105B0000011100EBC10090F8940000F0030001289F
:105B100018D09DF8B40040F2833110FB01F04549E4
:105B200001EB800000F589609DF8A01001EB4102B7
:105B300002EB011100EBC10090F8940000F00300AB
:105B400003282BD19DF8B40000EB400101EB0010BD
:105B5000394901EB001030309DF8A01000EB011026
:105B6000801C0990007820F00200801C09990870C0
:105B70009DF8B40000EB400101EB00102E4901EB51
:105B8000001030309DF8A01000EB0110801C09902F
:105B9000007820F020020998027014E09DF8B4000B
:105BA00000EB400101EB0010234901EB0010303005
:105BB0009DF8A01000EB0110801C0990007820F0E7
:105BC0000202099802709DF8B40000EB400101EB5D
:105BD0000010194901EB001130319DF8A00001EBD4
:105BE00000108078C0F340029DF8B40040F2833189
:105BF00010FB01F00F4901EB800000F589609DF872
:105C0000A01001EB410303EB011100EBC100007E8A
:105C1000C0F34000824277D09DF8B40040F2833157
:105C200010FB01F0034901EB800000F5896009E0F9
:105C3000388F002088480020C84300200000000062
:105C4000000024409DF8A01001EB410202EB01117D
:105C500000EBC100183009909DF8B40000EB400142
:105C600001EB0010FE4901EB001030309DF8A01050
:105C700000EB0110807842080998007862F3410037
:105C8000099908709DF8B40000EB400101EB001089
:105C9000F34901EB001030309DF8A01000EB01102B
:105CA0008078C0F3400050BB9DF8B40000EB400189
:105CB00001EB0010EA4901EB001030309DF8A01014
:105CC00000EB0110801C0990007820F02002099858
:105CD000027001229DF8B40040F2833110FB01F004
:105CE000E04901EB800000F589609DF8A01001EB10
:105CF000410303EB011100EBC10080F846209DF841
:105D0000B4100220F4F7D2F99DF8B40000EB400182
:105D100001EB0010D24901EB001130319DF8A000D9
:105D200001EB0010807800F001029DF8B40040F211
:105D3000833110FB01F0CB4901EB800000F5896055
:105D40009DF8A01001EB410303EB011100EBC10032
:105D5000007E00F00100824265D09DF8B40040F260
:105D6000833110FB01F0BF4901EB800000F5896031
:105D70009DF8A01001EB410202EB011100EBC10004
:105D8000183009909DF8B40000EB400101EB0010C1
:105D9000B34901EB001030309DF8A01000EB01106A
:105DA000807809990A7860F300020A709DF8B400BF
:105DB00000EB400101EB0010A94901EB001030306D
:105DC0009DF8A01000EB0110807800F0010058BB96
:105DD0009DF8B40000EB400101EB0010A04901EB7D
:105DE000001030309DF8A01000EB0110801C0990CD
:105DF000007820F020020998027000229DF8B4007B
:105E000040F2833110FB01F0964901EB800000F570
:105E100089609DF8A01001EB410303EB011100EB39
:105E2000C10080F8452013E29DF8B40040F28331B0
:105E300010FB01F08B4901EB800000F589609DF8B3
:105E4000A01001EB410202EB011100EBC10090F840
:105E50004600B0B901229DF8B40040F2833110FB36
:105E600001F0804901EB800000F589609DF8A010E9
:105E700001EB410303EB011100EBC10080F8452069
:105E80002AE000229DF8B40040F2833110FB01F0BB
:105E9000744901EB800101F589619DF8A00000EBD8
:105EA000400303EB001001EBC00080F845209DF893
:105EB000B40000EB400101EB0010694901EB001058
:105EC00030309DF8A01000EB0110801C0990007884
:105ED00020F0010209980270634890F8100B80B11D
:105EE0009DF8B40000EB400101EB00105C4901EBB0
:105EF000001030309DF8A01000EB0110807A0228CD
:105F00006FD15A4890F8290001286BD15748D0F832
:105F10000C025649498D884264D29DF8B40040F283
:105F2000833110FB01F04F4901EB800000F58960DF
:105F30009DF8A01001EB410202EB011100EBC10042
:105F400090F8450001284CD19DF8B40040F283310F
:105F500010FB01F0434901EB800000F589609DF8DA
:105F6000A01001EB410202EB011100EBC10090F81F
:105F70007F00B0BB01229DF8B40000EB400101EBB3
:105F80000010374901EB001130319DF8A00001EB02
:105F90000010C2729DF8B40000EB400101EB00104C
:105FA0002F4901EB001130319DF8A00001EB0010EA
:105FB00001789DF8B40040F2833210FB02F0294AC8
:105FC00002EB8000417005229DF8B40040F283315D
:105FD00010FB01F0234901EB800101F5896102E02A
:105FE000FEE307E171E09DF8A00000EB400303EB46
:105FF000001001EBC000427100229DF8B40000EBDC
:10600000400101EB0010164901EB001130319DF801
:10601000A00001EB001042609DF8B4100220F4F7DC
:1060200045F800213A9127E000229DF8B40040F2A3
:10603000833110FB01F00B4901EB800101F589610F
:106040009DF8A00000EB400303EB001001EBC00142
:106050004731BDF8E8000A54BDF8E800401C09E0EB
:10606000C843002088480020BC320020BC12002019
:1060700074E361E281B23A91BDF8E8001428D3DB01
:1060800000203A901CE000229DF8B40040F28331D9
:1060900010FB01F0FE4901EB800101F589619DF8DB
:1060A000A00000EB400303EB001001EBC0016331E3
:1060B000BDF8E8000A54BDF8E800401C81B23A91EE
:1060C000BDF8E8000A28DEDBC2E09DF8B40040F22B
:1060D000833110FB01F0EE4901EB800000F589608F
:1060E0009DF8A01001EB410202EB011100EBC10091
:1060F00090F8450001287DD19DF8B40040F283312D
:1061000010FB01F0E24901EB800101F589619DF886
:10611000A00000EB400202EB001001EBC00090F881
:10612000800040F2833110FB01F0D94901EB80017E
:1061300001F589619DF8B40040F2833210FB02F052
:10614000D34A02EB800000F589609DF8A02002EBA5
:10615000420303EB021200EBC20090F8810000EB57
:10616000400202EB001001EBC00090F87E00032813
:106170006ED102229DF8B40000EB400101EB00104B
:10618000C44901EB001130319DF8A00001EB001073
:10619000C2729DF8B40000EB400101EB0010BD4954
:1061A00001EB001130319DF8A00001EB00100178E7
:1061B0009DF8B40040F2833210FB02F0B44A02EBC7
:1061C000800041709DF8B40040F2833110FB01F073
:1061D000114601EB800101F589619DF8A00000EBFB
:1061E000400202EB001011F830109DF8B40040F2AC
:1061F000833200E02CE010FB02F0A54A02EB8000A5
:106200004079814214D105229DF8B40040F28331D7
:1062100010FB01F09E4901EB800000F589609DF8BC
:10622000A01001EB410303EB011100EBC10042712F
:1062300000229DF8B40000EB400101EB00109549ED
:1062400001EB001030309DF8A01000EB011042600F
:106250009DF8B40040F2833110FB01F08C4901EB52
:10626000800000F589609DF8A01001EB410202EB6F
:10627000011110F83100012814DC02229DF8B4004D
:1062800040F2833110FB01F0814901EB800000F501
:1062900089609DF8A01001EB410303EB011100F8A8
:1062A000312095E09DF8B40040F2833110FB01F0FD
:1062B000774901EB800000F589609DF8A01001EBA3
:1062C000410202EB011110F83100022834DC0021F8
:1062D0009DF8B40040F2833210FB02F06C4A02EBEE
:1062E0008000017103229DF8B40040F2833110FB5D
:1062F00001F0674901EB800101F589619DF8A0007B
:1063000000EB400303EB001001F8302007229DF85A
:10631000B40040F2833110FB01F05D4901EB8000D5
:1063200000F589609DF8A01001EB410303EB01111A
:1063300000EBC10042714BE09DF8B40040F28331A4
:1063400010FB01F0524901EB800101F589619DF8D4
:10635000A00000EB400202EB001011F830109DF895
:10636000B40040F2833210FB02F0494A02EB800095
:10637000407981422CD19DF8B40040F2833110FB6A
:1063800001F0114601EB800000F589609DF8A01036
:1063900001EB410202EB011100EBC10090F8940007
:1063A000C0F34010A0B116229DF8B40040F2833132
:1063B00010FB01F0364901EB800000F589609DF883
:1063C000A01001EB410303EB011100EBC10042718E
:1063D000B2E014229DF8B40040F2833110FB01F0CA
:1063E0002B4901EB800101F589619DF8A00000EBCC
:1063F000400303EB001001EBC000427101219DF846
:10640000B40040F2833210FB02F0214A02EB80001C
:1064100001719DF8B40000EB400101EB00101D4933
:1064200001EB001130319DF8A00001EB0010801C41
:106430000990007820F020002030099908707BE056
:1064400014229DF8B40040F2833110FB01F0104992
:1064500001EB800000F589609DF8A01001EB41037D
:1064600003EB011100EBC100427165E09DF8B4003F
:1064700040F2833110FB01F0054901EB800000F58B
:106480008960BDF8D81001EB410202EB011103E075
:1064900088480020C843002000EBC1008079012813
:1064A0002AD100229DF8B40040F2833110FB01F0A4
:1064B000FE4901EB800101F58961BDF8D80000EBD0
:1064C000400303EB001001EBC000827114229DF821
:1064D000B40040F2833110FB01F0F44901EB80007D
:1064E00000F589609DF8A01001EB410303EB011159
:1064F00000EBC10042711FE000219DF8B40040F2A2
:10650000833210FB02F0E94A02EB800001710522A0
:106510009DF8B40040F2833110FB01F0E34901EB38
:10652000800000F589609DF8A01001EB410303EBAA
:10653000011100EBC1004271FDE301219DF8B4009F
:1065400040F2833210FB02F0D84A02EB8000017166
:1065500014229DF8B40040F2833110FB01F0D349BE
:1065600001EB800101F589619DF8A00000EB40037B
:1065700003EB001001EBC00042719DF8B40000EB8A
:10658000400101EB0010CA4901EB001130319DF8C8
:10659000A00001EB0010801C0990007820F004009E
:1065A000001D09990870C6E300202E902F9000214D
:1065B0003A911EE0DDE92E10000240EA1162090264
:1065C000CDE92E129DF8B40000EB4001C1EBC010E4
:1065D000B84901EBC001BDF8E800401D085CDDE9E9
:1065E0002E341843CDE92E04BDF8E800401C80B2DB
:1065F0003A90BDF8E8000328DCDBDDE92E0112F05B
:106600004FF901469DF8B40040F2833210FB02F0CE
:10661000A64A02EB800202F589629DF8A00000EB19
:10662000400303EB001002EBC000C0F81E10002274
:106630002E922F9200213A911EE0DDE92E100002E9
:1066400040EA11620902CDE92E129DF8B40000EB78
:106650004001C1EBC010974901EBC001BDF8E80053
:106660000830085CDDE92E341843CDE92E04BDF86E
:10667000E800401C80B23A90BDF8E8000328DCDB5B
:10668000DDE92E0112F00CF901469DF8B40040F24C
:10669000833210FB02F0854A02EB800202F5896228
:1066A0009DF8A00000EB400303EB001002EBC000DC
:1066B000C0F81A1000222E922F9200213A911EE06B
:1066C000DDE92E10000240EA11620902CDE92E1226
:1066D0009DF8B40000EB4001C1EBC010754901EB1F
:1066E000C001BDF8E8001330085CDDE92E34184322
:1066F000CDE92E04BDF8E800401C80B23A90BDF808
:10670000E8000328DCDB9DF8B4002E9940F28332C8
:1067100010FB02F0654A02EB800202F589629DF8E7
:10672000A00000EB400303EB001002EBC00041634C
:1067300007229DF8B40040F2833110FB01F05B4961
:1067400001EB800000F589609DF8A01001EB41038A
:1067500003EB011100EBC1004271ECE200202E902E
:106760002F9000213A911EE0DDE92E10000240EA50
:1067700011620902CDE92E129DF8B40000EB400130
:10678000C1EBC0104B4901EBC001BDF8E800401D52
:10679000085CDDE92E341843CDE92E04BDF8E8008D
:1067A000401C80B23A90BDF8E8000428DCDBDDE94B
:1067B0002E0112F075F89DF8B42040F2833312FBDD
:1067C00003F23A4B03EB820303F589639DF8A020A3
:1067D00002EB420404EB021203EBC202223200E09D
:1067E000FEE39060D16000212E912F9100203A901D
:1067F0001FE0DDE92E10000240EA11620902CDE936
:106800002E129DF8B40000EB4001C1EBC0102949E5
:1068100001EBC001BDF8E8000930085CDDE92E3469
:1068200040EA0302CDE92E24BDF8E800401C81B205
:106830003A91BDF8E8000428DBDBDDE92E0112F017
:106840002FF89DF8B42040F2833312FB03F2174B6C
:1068500003EB820303F589639DF8A02002EB420459
:1068600004EB021203EBC20242F8220F51609DF8C2
:10687000B40040F2833110FB01F00C4901EB8000C1
:1068800000F589609DF8A01001EB410202EB0111B7
:1068900010F831009DF8B41040F2833211FB02F180
:1068A000024A02EB81014979884205E088480020CC
:1068B000C8430020388F00207ED19DF8B40040F2FC
:1068C000833110FB01F0114601EB800000F5896077
:1068D0009DF8A01001EB410202EB011100EBC10099
:1068E00090F89400C0F34010A8B117229DF8B400AE
:1068F00040F2833110FB01F0FE4901EB800000F50E
:1069000089609DF8A01001EB410303EB011100EB3E
:10691000C100427114E014229DF8B40040F28331AA
:1069200010FB01F0F34901EB800101F589619DF84D
:10693000A00000EB400303EB001001EBC00042712C
:106940009DF8B4009DF8A01001EB0010C217CDE92E
:106950002E02E94890F8100B08B39DF8B40000EB44
:10696000400101EB0010E54901EB001030309DF8CB
:10697000A01000EB0110807A022810D09DF8B4001E
:1069800000EB400101EB0010DC4901EB001030305E
:106990009DF8A01000EB0110C07A00287EDD0022D7
:1069A0009DF8B40040F2833110FB01F0D14901EBB6
:1069B000800101F5896100E02DE39DF8A00000EB66
:1069C000400303EB001001EBC00080F846209DF867
:1069D000B40000EB400101EB0010C84901EB0011CD
:1069E00030319DF8A00001EB0010C272C448D0F80D
:1069F0000C020521B0FBF1F201FB120000EB40019B
:106A0000BF482C3000EB41100D3009909DF8B400C8
:106A100040F2833110FB01F0B64901EB800000F534
:106A200089609DF8A01001EB410202EB011100EB1F
:106A3000C10022301022014608900998F1F705FCA8
:106A4000AF48D0F80C020521B0FBF1F201FB1200B7
:106A500000EB4001AA482C3000EB41129DF8B40035
:106A600040F2833110FB01F0A24901EB800101F5F6
:106A700089619DF8A00000EB400303EB001001EBDF
:106A8000C00050F81A1F42F8011F406850609C482F
:106A9000D0F80C020521B0FBF1F200E0A8E101FB07
:106AA000120000EB400196482C3000EB41129DF89B
:106AB000B40000EB400101EB0010904901EB001124
:106AC00030319DF8A00001EB0010007810708C4868
:106AD000D0F80C020521B0FBF1F201FB120000EB33
:106AE000400187482C3000EB41129DF8B40040F281
:106AF000833110FB01F07F4901EB800101F58961D1
:106B00009DF8A00000EB400303EB001001EBC00078
:106B1000406BC2F809007A48D0F80C020521B0FB9E
:106B2000F1F201FB120000EB400175482C3000EB44
:106B300041117148F538026841F81D2F808888801E
:106B40006F48D0F80C020521B0FBF1F201FB1200F6
:106B500000EB40016A482C3000EB41129DF8B40074
:106B600000EB400101EB0010644901EB00113031F2
:106B70009DF8A00001EB00104068C2F8230000223D
:106B80009DF8B40000EB400101EB00105B4901EB04
:106B9000001130319DF8A00001EB0010426000218F
:106BA0003A9154E05648D0F80C020521B0FBF1F2BE
:106BB00001FB120000EB400151482C3000EB411169
:106BC0002731BDF8E8409DF8B40040F2833210FB55
:106BD00002F0484A02EB800202F589629DF8A000AB
:106BE00000EB400303EB001002EBC00090F88000C4
:106BF00040F2833210FB02F03E4A02EB800202F5C3
:106C000089629DF8B40040F2833310FB03F0394BE6
:106C100003EB800303F589639DF8A00000EB4005BA
:106C200005EB001003EBC00090F8810000EB40037F
:106C300003EB001002EBC0024732BDF8E800001D74
:106C4000105C0855BDF8E800401C81B23A91BDF8CF
:106C5000E8000628A6DB00213A9142E000239DF8D7
:106C6000B40040F2833110FB01F0224901EB8001B6
:106C700001F589619DF8A00000EB400202EB0010D5
:106C800001EBC00090F8800040F2833110FB01F06E
:106C9000184901EB800101F589619DF8B40040F2CB
:106CA000833210FB02F0134A02EB800202F5896284
:106CB0009DF8A00000EB400404EB001002EBC000C4
:106CC00090F8810000EB400202EB001001EBC001E4
:106CD0004731BDF8E8000B54BDF8E800401C81B214
:106CE0003A91BDF8E8000A28B8DB0548D0F80C0254
:106CF000052107E088480020BC320020C84300205E
:106D0000BC120020B0FBF1F080B2014609900220D5
:106D1000F2F7DEF900210620F3F7C8F9FE48D0F8B3
:106D20000C02FD49498D884208D2FB48D0F80C027C
:106D3000401CF94900E002E2C1F80C0200210520E4
:106D4000F3F7B4F99DF8B40000EB400101EB00103B
:106D5000F24901EB001030309DF8A01000EB01105B
:106D6000801C0990007820F0080209980270EA4817
:106D7000D0F80C020521B0FBF1F201FB120000EB90
:106D80004001E5482C3000EB4110D0F823202E982C
:106D900000EB4001E24800EB4110C0F82320002046
:106DA0003A9020E0DC48D0F80C020521B0FBF1F26B
:106DB00001FB120000EB4001D7482C3000EB4110E2
:106DC0002730BDF8E810425C2E9800EB4001D44813
:106DD00000EB41112731BDF8E8000A54BDF8E80086
:106DE000401C81B23A91BDF8E8000628DADB6FE07A
:106DF00000229DF8B40040F2833110FB01F0C94934
:106E000001EB800101F589619DF8A00000EB4003D2
:106E100003EB001001EBC00080F846209DF8B400A1
:106E200000EB400101EB0010BC4901EB00113031D7
:106E30009DF8A00001EB0010801C0990007820F064
:106E400008000830099908709DF8B40000EB400173
:106E500001EB0010B14901EB001030309DF8A0109B
:106E600000EB011042682E9800EB4001AC4800EBAB
:106E70004110C0F8232000203A9025E09DF8B4008E
:106E800040F2833110FB01F0A64901EB800101F5CE
:106E900089619DF8A00000EB400202EB001001EBBD
:106EA000C0014731BDF8E8000A5C2E9800EB4001B4
:106EB0009B4800EB41112731BDF8E8000A54BDF8AA
:106EC000E800401C81B23A91BDF8E8000628D5DB05
:106ED0009DF8B4100220F3F7E9F89DF8B40040F2F1
:106EE000833110FB01F08F4901EB800101F58961CD
:106EF0009DF8A00000EB400202EB001001EBC00087
:106F0000223009902E9800EB4001854800EB41109B
:106F10000D30102208900999F1F797F99DF8B40007
:106F200040F2833110FB01F07E4901EB800101F555
:106F300089619DF8A00000EB400202EB001001EB1C
:106F4000C0012E9800EB4002754800EB421051F84A
:106F50001A2F40F8012F496841609DF8B40000EBFA
:106F6000400101EB00106D4901EB001130319DF83B
:106F7000A00001EB001001782E9800EB4002684859
:106F800000EB421001702E9800EB4001644800EBCA
:106F900041116548026841F81D2F808888809DF85E
:106FA000B40040F2833110FB01F05E4901EB800137
:106FB00001F589619DF8A00000EB400202EB001092
:106FC00001EBC000416B2E9800EB4002544800EBEF
:106FD0004210C0F809109DF8B40000EB400100E039
:106FE00033E101EB00104D4901EB001130319DF808
:106FF000A00001EB001041682E9800EB40024848C9
:1070000000EB4210C0F823102E9881B2082009919D
:10701000F3F74CF893E09DF8B40040F2833110FB95
:1070200001F0404901EB800101F589619DF8A00064
:1070300000EB400202EB001011F830109DF8B40094
:1070400040F2833210FB02F0364A02EB80004079B6
:10705000814274DA9DF8B40000EB400101EB0010AE
:107060002E4901EB001030309DF8A01000EB01100C
:10707000801C0990007820F00400001D0999087018
:107080009DF8B40000EB400101EB0011234800EB38
:10709000011030309DF8A01000EB0110801C099009
:1070A000007820F0800180310998017001219DF85D
:1070B000B40040F2833210FB02F01A4A02EB800067
:1070C00001719DF8B40040F2833110FB01F11046CC
:1070D00000EB810042799DF8B40040F2833110FB4F
:1070E00001F0104901EB800101F589619DF8A000D4
:1070F00000EB400303EB001001F8302014229DF850
:10710000B40040F2833110FB01F0064901EB80002E
:1071100000F589600AE012E0BC120020C84300209C
:10712000D814002088480020C73100209DF8A01006
:1071300001EB410303EB011100EBC100427183E05D
:107140000121FE4880F8341A9DF8B40040F28331E2
:1071500010FB01F0FA4901EB800101F589619DF80E
:10716000A00000EB400202EB001011F830109DF877
:10717000B40040F2833210FB02F0F14A02EB8000CF
:107180004079814233DA00219DF8B40040F2833225
:1071900010FB02F0EA4A02EB8000017101229DF827
:1071A000B40040F2833110FB01F0E54901EB8001AE
:1071B00001F589619DF8A00000EB400303EB00108E
:1071C00001F8302014229DF8B40040F2833110FB06
:1071D00001F0DB4901EB800000F589609DF8A0100B
:1071E00001EB410303EB011100EBC10042712BE005
:1071F00014229DF8B40040F2833110FB01F0D04915
:1072000001EB800000F589609DF8A01001EB4103BF
:1072100003EB011100EBC100427115E014229DF84F
:10722000B40040F2833110FB01F0C54901EB80004E
:1072300000F589609DF8A01001EB410303EB0111FB
:1072400000EBC100427100BF00BF07F03CBD9DF8DC
:10725000B40040F2833110FB01F0B94901EB80002A
:10726000817828919DF8B40000EB4001C1EBC0107B
:10727000B44911F8301029919DF8B40040F28331DF
:1072800010FB01F0AE4901EB800101F589619DF829
:10729000A00000EB400202EB001001EBC0004179BE
:1072A00025919DF8B40000EB4001C1EBC010A54949
:1072B00001EBC0010991BDF8A4100998F3F78EFC09
:1072C00037909DF8B40000EB4001C1EBC0109D4920
:1072D00001EBC001BDF8A400095CBDF8DC008142EF
:1072E00041F066879DF8B40000EB4001C1EBC0108F
:1072F000944901EBC0004078002841F359870021F0
:10730000914A9DF8B40002EB00129DF8A0001154C0
:10731000BDF8940089287DD00EDC142801F0288760
:1073200005DC082877D0102841F04187FBE31528B9
:1073300072D08028F8D1F8E38B286ED08C286DD0DD
:107340008E286CD08F28EFD1BDF8A4000D2867D10E
:107350009DF8B40000EB4001C1EBC010794901EB8E
:10736000C0004178794880F8041D9DF8B40000EB16
:107370004001C1EBC010734901EBC000C17A7348F2
:1073800080F8051D9DF8B40040F2833110FB01F038
:107390006B4901EB800000F589609DF8A01001EBBE
:1073A000410202EB011110F8310003287EDC67482E
:1073B00090F8050D00287ADD9DF8B40040F2833185
:1073C00010FB01F05E4901EB800101F589619DF838
:1073D000A00000EB400202EB001001EBC00109919C
:1073E0000878401CC1B2099801709DF8B40040F2C1
:1073F000833110FB01F0524901EB800000F58960F8
:107400009DF8A01001EB410202EB011110F83100D0
:10741000042806E0FDE3FDE3FDE3FDE3FDE3FDE31A
:10742000FDE344DB9DF8B40000EB400101EB0010EC
:10743000474901EB001030309DF8A01000EB01101F
:10744000801C0990414890F8050DC0F30010C0F170
:1074500001000999097860F30001099801703B481F
:1074600090F8040DC0F3C000F0BB9DF8B40000EB31
:10747000400101EB0010364901EB001030309DF85F
:10748000A01000EB01108078C0F3401060B39DF8AD
:10749000B40000EB400101EB00102D4901EB00109E
:1074A00030309DF8A01000EB011001E06CE009E124
:1074B000801C0990007820F00200801C0999087057
:1074C0009DF8B40040F2833110FB01F01C4901EB40
:1074D000800000F589609DF8A01001EB410202EBED
:1074E000011100EBC10000E00CE0183009900078B9
:1074F00020F00200801C099908709DF8B410022049
:10750000F2F7D4FD00219DF8B40040F2833210FB65
:1075100002F00B4A02EB8000017104229DF8B400D6
:1075200040F2833110FB01F0054901EB800101F5C8
:1075300089619DF8A00000EB40030BE0BC32002005
:1075400088480020388F0020B8410020BC2200204D
:10755000C843002003EB001001F830208C229DF876
:10756000B40040F2833110FB01F0F94901EB8001D6
:1075700001F589619DF8A00000EB400303EB0010CA
:1075800001EBC00042719DE09DF8B40040F28331F0
:1075900010FB01F0EE4901EB800101F589619DF8D6
:1075A000A00000EB400202EB001011F830109DF833
:1075B000B40040F2833210FB02F0E54A02EB800097
:1075C000407981427ED19DF8B40000EB400101EB8F
:1075D0000010A2F5986101EB001030309DF8A0106A
:1075E00000EB0110801C0990DA4890F8050DC0F3FB
:1075F0000010C0F101010998027861F300020270E5
:107600009DF8B40000EB400101EB0010D24901EB02
:10761000001130319DF8A00001EB0010801C099092
:10762000CC4890F8040DC2080998007862F3410034
:10763000099908709DF8B40000EB400101EB0010BF
:10764000C54901EB001030309DF8A01000EB01108F
:107650008078C0F340029DF8B40040F2833110FB03
:1076600001F0BB4901EB800000F589609DF8A01096
:1076700001EB410303EB011100EBC100007EC0F3FD
:10768000400082426CD09DF8B40040F2833110FB80
:1076900001F0AF4901EB800000F589609DF8A01072
:1076A00001EB410202EB011100EBC100183009901F
:1076B0009DF8B40000EB400101EB0010A64901EB7E
:1076C000001000E0C6E330309DF8A01000EB011080
:1076D000807842080998017862F3410101709DF8B1
:1076E000B40000EB400101EB00109B4901EB0010DE
:1076F00030309DF8A01000EB01108078C0F34000FE
:1077000048BB01229DF8B40040F2833110FB01F028
:107710008F4901EB800101F589619DF8A00000EB24
:10772000400303EB001001EBC00042739DF8B4006E
:1077300040F2833110FB01F0854901EB800000F538
:1077400089609DF8A01001EB410303EB011100EBF0
:10775000C10080F846209DF8B4100220F2F7A6FC84
:107760009DF8B40000EB400101EB00107A4901EBF9
:10777000001130319DF8A00001EB0010807800F07E
:1077800001029DF8B40040F2833110FB01F0704912
:1077900001EB800000F589609DF8A01001EB41032A
:1077A00003EB011100EBC100007E00F001008242FA
:1077B00079D09DF8B40040F2833110FB01F06449A8
:1077C00001EB800000F589609DF8A01001EB4102FB
:1077D00002EB011100EBC100183009909DF8B400D4
:1077E00000EB400101EB00105B4901EB001130316F
:1077F0009DF8A00001EB001082780998017862F3EF
:10780000000101709DF8B40000EB400101EB001095
:10781000514901EB001030309DF8A01000EB011031
:10782000807800F00100E8BB9DF8B40000EB400157
:1078300001EB0010484901EB001030309DF8A0101A
:1078400000EB01108078C0F3401068B39DF8B400DD
:1078500040F2833110FB01F03D4901EB800000F55F
:1078600089609DF8A01001EB410202EB011100EBD1
:10787000C10090F84600B8B99DF8B40040F28331D9
:1078800010FB01F0324901EB800000F589609DF8A2
:10789000A01001EB410202EB011100EBC100407BA3
:1078A00010B902E05AE056E23BE09DF8B40000EB6C
:1078B000400101EB0010284901EB001030309DF829
:1078C000A01000EB01108078C0F3400048BB0122FB
:1078D0009DF8B40040F2833110FB01F01C4901EB2C
:1078E000800101F589619DF8A00000EB400303EBE6
:1078F000001001EBC00042739DF8B40040F28331E8
:1079000010FB01F0124901EB800000F589609DF841
:10791000A01001EB410303EB011100EBC10080F863
:10792000462000229DF8B40040F2833110FB01F0A4
:10793000074901EB800000F589609DF8A01001EB7C
:10794000410303EB011100EBC10080F84520FDE18C
:1079500088480020BC220020C84300209DF8B400C5
:1079600040F2833110FB01F0FE4901EB800000F58D
:1079700089609DF8A01001EB410202EB011100EBC0
:10798000C10090F84600B0B901229DF8B40040F261
:10799000833110FB01F0F34901EB800000F58960B1
:1079A0009DF8A01001EB410303EB011100EBC100B6
:1079B00080F845202AE000229DF8B40040F283318F
:1079C00010FB01F0E74901EB800101F589619DF8A9
:1079D000A00000EB400303EB001001EBC00080F8B7
:1079E00045209DF8B40000EB400101EB0010DE499A
:1079F00001EB001030309DF8A01000EB0110801C4E
:107A00000990007820F0010209980270D74890F898
:107A1000100B80B19DF8B40000EB400101EB0010A9
:107A2000D14901EB001030309DF8A01000EB01109F
:107A3000807A022878D1CE4890F82900012873D1A5
:107A4000CB48D0F80C02CA49498D88426CD29DF8C7
:107A5000B40040F2833110FB01F0C24901EB800019
:107A600000F589609DF8A01001EB410202EB0111C5
:107A700000EBC10090F84500012853D19DF8B400F7
:107A800040F2833110FB01F0B64901EB800000F5B4
:107A900089609DF8A01001EB410202EB011100EB9F
:107AA000C10090F87F00E8BB01229DF8B40000EB14
:107AB000400101EB0010AC4901EB001130319DF8A1
:107AC000A00001EB0010C2729DF8B40000EB400171
:107AD00001EB0010A44901EB001130319DF8A0002A
:107AE00001EB001001789DF8B40040F2833210FBE6
:107AF00002F09C4A02EB8000417008229DF8B4001D
:107B000040F2833110FB01F0964901EB800101F551
:107B100089619DF8A00000EB400303EB001001EB2E
:107B2000C00003E061E023E3FBE0FDE342710022DB
:107B30009DF8B40000EB400101EB00108A4901EB15
:107B4000001130319DF8A00001EB001042609DF85B
:107B5000B4100220F2F7AAFA00213A911CE00022A8
:107B60009DF8B40040F2833110FB01F07D4901EB38
:107B7000800101F589619DF8A00000EB400303EB53
:107B8000001001EBC0014731BDF8E8000A54BDF810
:107B9000E800401C81B23A91BDF8E8001428DEDB11
:107BA00000203A901CE000229DF8B40040F283319E
:107BB00010FB01F06B4901EB800101F589619DF833
:107BC000A00000EB400303EB001001EBC0016331A8
:107BD000BDF8E8000A54BDF8E800401C81B23A91B3
:107BE000BDF8E8000A28DEDBB0E09DF8B40040F202
:107BF000833110FB01F05B4901EB800000F58960E7
:107C00009DF8A01001EB410202EB011100EBC10055
:107C100006E0C7E281E2FDE32AE391E3FBE37BE2D6
:107C200090F8450001287CD19DF8B40040F28331E2
:107C300010FB01F04B4901EB800101F589619DF8D2
:107C4000A00000EB400202EB001001EBC00090F836
:107C5000800040F2833110FB01F0424901EB8001CA
:107C600001F589619DF8B40040F2833210FB02F007
:107C70003C4A02EB800000F589609DF8A02002EBF1
:107C8000420303EB021200EBC20090F8810000EB0C
:107C9000400202EB001001EBC00090F87E000328C8
:107CA00054D102229DF8B40000EB400101EB00101A
:107CB0002D4901EB001130319DF8A00001EB0010BF
:107CC000C2729DF8B40000EB400101EB00102649A0
:107CD00001EB001130319DF8A00001EB001001789C
:107CE0009DF8B40040F2833210FB02F01D4A02EB13
:107CF0008000417008229DF8B40040F2833110FBEF
:107D000001F0184901EB800101F589619DF8A0009F
:107D100000EB400303EB001001EBC00042710022B6
:107D200000E013E09DF8B40000EB400101EB00100F
:107D30000D4901EB001130319DF8A00001EB00105E
:107D400042609DF8B4100220F2F7B0F99DF8B4102B
:107D50000220F2F7ABF99DF8B40040F2833110FB3A
:107D600001F007E088480020C8430020BC32002012
:107D7000BC120020FB4901EB800000F589609DF8F2
:107D8000A01001EB410202EB011100EBC100807871
:107D9000802838D19DF8B40000EB400101EB0010C1
:107DA000F14901EB001030309DF8A01000EB0110FC
:107DB0008078C0F3400030BB9DF8B40000EB400178
:107DC00001EB0010E84901EB001030309DF8A010E5
:107DD00000EB01108078C0F34010A0B915229DF887
:107DE000B40040F2833110FB01F0DE4901EB80006A
:107DF00000F589609DF8A01001EB410303EB011130
:107E000000EBC10042719DF8B40000EB400101EBB2
:107E10000010D54901EB001030309DF8A01000EBA8
:107E200001108078C0F34000A8B18F229DF8B40003
:107E300040F2833110FB01F0CA4901EB800000F5EC
:107E400089609DF8A01001EB410303EB011100EBE9
:107E5000C10042714AE09DF8B40040F2833110FB4A
:107E600001F0C04901EB800000F589609DF8A01089
:107E700001EB410202EB011100EBC100807B012804
:107E800034D100229DF8B40040F2833110FB01F0A0
:107E9000B44901EB800101F589619DF8A00000EB78
:107EA000400303EB001001EBC00082738C229DF8AD
:107EB000B40040F2833110FB01F0AA4901EB8001CC
:107EC00001F589619DF8A00000EB400303EB001071
:107ED00001EBC000427100219DF8B40040F28332F2
:107EE00010FB02F09F4A02EB800001719DF8B40084
:107EF00000EB400101EB00109B4901EB0010007BFF
:107F0000F0BB9DF8B40000EB4001C1EBC0109749F5
:107F100001EBC000807801049DF8B40000EB400242
:107F2000C2EBC010914A02EBC000C07841EA0021C8
:107F30009DF8B40000EB4002C2EBC0108B4A02EB8C
:107F4000C00000790843C117CDE9080110F0A8FC72
:107F50009DF8B41040F2833211FB02F1814A02EB2A
:107F6000810202F589629DF8A01001EB410303EB49
:107F7000011102EBC101C1F81E009DF8B40000E040
:107F80003AE000EB4001C1EBC010784901EBC000C2
:107F9000407900049DF8B41001EB4102C2EBC1111D
:107FA000724A02EBC101897940EA01209DF8B410C0
:107FB00001EB4102C2EBC1116C4A02EBC101C9796C
:107FC0000843C117CDE9080110F06AFC9DF8B41010
:107FD00040F2833211FB02F1624A02EB810101F5AA
:107FE00089619DF8A02002EB420303EB021201EB32
:107FF000C201C1F81A008FE09DF8B40000EB400107
:10800000C1EBC010594901EBC000807801069DF812
:10801000B40000EB4002C2EBC010544A02EBC000B7
:10802000C07841EA00419DF8B40000EB4002C2EB89
:10803000C0104E4A02EBC000007941EA00209DF8D2
:10804000B41001EB4102C2EBC111484A02EBC1017D
:1080500049790843C117CDE9080110F021FC9DF8CA
:10806000B41040F2833211FB02F13E4A02EB81026E
:1080700002F589629DF8A01001EB410303EB0111A9
:1080800002EBC101C1F81E009DF8B40000EB4001F5
:10809000C1EBC010354901EBC000807900069DF8A6
:1080A000B41001EB4102C2EBC111304A02EBC10135
:1080B000C97940EA01409DF8B41001EB4102C2EBDE
:1080C000C1112A4A02EBC101097A40EA01209DF858
:1080D000B41001EB4102C2EBC111244A02EBC10111
:1080E000497A0843C117CDE9080110F0D9FB9DF882
:1080F000B41040F2833211FB02F11A4A02EB810103
:1081000001F589619DF8A02002EB420303EB021206
:1081100001EBC201C1F81A0022E2BDF8A400032855
:108120001FD18F229DF8B40040F2833110FB01F083
:108130000C4901EB800101F589619DF8A00000EB7D
:10814000400303EB001001EBC000427101219DF8D8
:10815000B40040F2833210FB02F0024A02EB8000CE
:108160000171FDE188480020C8430020388F0020BD
:10817000BDF8A400032814D18F229DF8B40040F26A
:10818000833110FB01F0F74901EB800000F58960B5
:108190009DF8A01001EB410303EB011100EBC100BE
:1081A0004271DDE1BDF8A400032860D19DF8B40060
:1081B00040F2833110FB01F0EA4901EB800000F549
:1081C0008960BDF8D81001EB410202EB011100EB10
:1081D000C100807901282AD100229DF8B40040F224
:1081E000833110FB01F0DF4901EB800101F589616A
:1081F000BDF8D80000EB400303EB001001EBC0001A
:1082000082718F229DF8B40040F2833110FB01F09F
:10821000D44901EB800000F589609DF8A01001EBC6
:10822000410303EB011100EBC10042711FE0082282
:108230009DF8B40040F2833110FB01F0C94901EB15
:10824000800101F589619DF8A00000EB400303EB7C
:10825000001001EBC000427100219DF8B40040F213
:10826000833210FB02F0BF4A02EB8000017177E11C
:10827000BDF8A400032862D19DF8B40040F2833118
:1082800010FB01F0B74901EB800000F58960BDF8F3
:10829000D81001EB410202EB011100EBC100807923
:1082A00001282AD100229DF8B40040F2833110FB4E
:1082B00001F0AC4901EB800101F58961BDF8D800FE
:1082C00000EB400303EB001001EBC00082718F2232
:1082D0009DF8B40040F2833110FB01F0A14901EB9D
:1082E000800000F589609DF8A01001EB410303EBCD
:1082F000011100EBC100427121E008229DF8B40099
:1083000040F2833110FB01F0964901EB800101F549
:1083100089619DF8A00000EB400303EB001001EB26
:10832000C0004271002100E020E19DF8B40040F25D
:10833000833210FB02F08B4A02EB800001710FE1E7
:10834000BDF8A400082867D19DF8B40000EB4001F7
:10835000C1EBC010844901EBC000807801069DF894
:10836000B40000EB4002C2EBC0107F4A02EBC00039
:10837000C07841EA00419DF8B40000EB4002C2EB36
:10838000C010794A02EBC000007941EA00219DF853
:10839000B40000EB4002C2EBC010734A02EBC00015
:1083A00040790843C117CDE9080110F079FA014678
:1083B0009DF8B40040F2833210FB02F0694A02EBF0
:1083C000800202F589629DF8A00000EB400303EBF8
:1083D000001002EBC00041639DF8B40040F283310D
:1083E00010FB01F05F4901EB800101F589619DF807
:1083F000A00000EB400202EB001011F830109DF8D5
:10840000B40040F2833210FB02F0564A02EB8000C7
:10841000407902E0FEE3E3E0A2E0814234DA0021A9
:108420009DF8B40040F2833210FB02F04D4A02EB9B
:108430008000017105229DF8B40040F2833110FBE9
:1084400001F0484901EB800101F589619DF8A00028
:1084500000EB400303EB001001F830208E229DF862
:10846000B40040F2833110FB01F03E4901EB800083
:1084700000F589609DF8A01001EB410303EB0111A9
:1084800000EBC10042716BE09DF8B40040F2833113
:1084900010FB01F0334901EB800000F58960BDF865
:1084A000D81001EB410202EB011100EBC100807911
:1084B000012835D100229DF8B40040F2833110FB31
:1084C00001F0284901EB800101F58961BDF8D80070
:1084D00000EB400303EB001001EBC00082718F2220
:1084E0009DF8B40040F2833110FB01F01D4901EB0F
:1084F000800101F589619DF8A00000EB400303EBCA
:10850000001001EBC000427101219DF8B40040F25F
:10851000833210FB02F0134A02EB800001711FE06E
:108520008E229DF8B40040F2833110FB01F00D491A
:1085300001EB800101F589619DF8A00000EB40038B
:1085400003EB001001EBC000427100219DF8B40064
:1085500040F2833210FB02F0024A02EB800001710C
:10856000FEE3000088480020388F0020BDF8A400FA
:10857000032834D100219DF8B40040F2833210FB6F
:1085800002F0FE4A02EB8000017101229DF8B40066
:1085900040F2833110FB01F0F84901EB800101F555
:1085A0008961BDF8D80000EB400303EB001001EB3C
:1085B000C00082718C229DF8B40040F2833110FB20
:1085C00001F0EE4901EB800000F589609DF8A010F4
:1085D00001EB410303EB011100EBC1004271BFE36A
:1085E000BDF8A4000F287CD19DF8B40000EB400139
:1085F00001EB0010E24901EB0010007BF0BB002012
:108600002E902F9000213A9120E0DDE92E100002FB
:1086100040EA11620902CDE92E129DF8B40000EB88
:108620004001C1EBC010D74901EBC001BDF8E80023
:10863000C0F10600085CDDE92E3440EA0302CDE912
:108640002E24BDF8E800401C81B23A91BDF8E80044
:108650000528DADB9DF8B400DDE92E2140F28333F2
:1086600010FB03F0C54B03EB800303F589639DF812
:10867000A00000EB400404EB001000E049E003EB35
:10868000C00040F8222F416000222E922F9200213C
:108690003A911FE0DDE92E10000240EA1162090262
:1086A000CDE92E129DF8B40000EB4001C1EBC010E3
:1086B000B44901EBC001BDF8E800C0F10B00085C53
:1086C000DDE92E341843CDE92E04BDF8E800401C46
:1086D00080B23A90BDF8E8000528DBDB9DF8B400D5
:1086E00000E0FDE3DDE92E1240F2833310FB03F0DE
:1086F000A24B03EB800000F589609DF8A03003EBEE
:10870000430404EB031300EBC30022308160C2601A
:1087100084E000202E902F9000213A911FE0DDE9A7
:108720002E10000240EA11620902CDE92E129DF8D6
:10873000B40000EB4001C1EBC010924901EBC00155
:10874000BDF8E800C0F10700085CDDE92E341843ED
:10875000CDE92E04BDF8E800401C80B23A90BDF887
:10876000E8000628DBDB9DF8B400DDE92E1240F2BC
:10877000833310FB03F0814B03EB800303F5896324
:108780009DF8A00000EB400404EB001003EBC000D8
:1087900040F8221F426000222E922F9200213A912F
:1087A00020E0DDE92E10000240EA11620902CDE965
:1087B0002E129DF8B40000EB4001C1EBC0107149CE
:1087C00001EBC001BDF8E800C0F10D00085CDDE977
:1087D0002E3440EA0302CDE92E24BDF8E800401C07
:1087E00081B23A91BDF8E8000628DADB9DF8B400C2
:1087F000DDE92E2140F2833310FB03F05F4B03EBE6
:10880000800000F589609DF8A03003EB430404EB81
:10881000031300EBC30022308260C1609DF8B400F6
:1088200040F2833110FB01F0544901EB800101F566
:1088300089619DF8A00000EB400202EB001011F8E6
:1088400030109DF8B40040F2833210FB02F04B4A26
:1088500002EB8000407981427ED19DF8B4009DF802
:10886000A01001EB0010C217CDE92E02464890F887
:10887000100B08B39DF8B40000EB400101EB0010B1
:108880003F4901EB001030309DF8A01000EB0110C3
:10889000807A022810D09DF8B40000EB400101EB73
:1088A0000010374901EB001030309DF8A01000EBAC
:1088B0000110C07A00286BDD00229DF8B40000EBA7
:1088C000400101EB00102E4901EB001030309DF803
:1088D000A01000EB0110C2722C48D0F80C02052148
:1088E000B0FBF1F201FB120000EB400127482C30F5
:1088F00000EB41100D3009909DF8B40040F2833137
:1089000010FB01F01D4901EB800000F589609DF826
:10891000A01001EB410202EB011100EBC10022307B
:108920001022014608900998EFF78FFC1748D0F8FD
:108930000C020521B0FBF1F201FB120000EB40013B
:1089400012482C3000EB41129DF8B40040F2833104
:1089500010FB01F0094900E0F7E201EB800101F5AD
:1089600089619DF8A00000EB400303EB001001EBD0
:10897000C00050F81A1F42F8011F0AE08848002082
:10898000C8430020388F0020BC320020BC120020D9
:10899000A6E140685060FE48D0F80C020521B0FB0B
:1089A000F1F201FB120000EB4001F9482C3000EB22
:1089B00041129DF8B40000EB400101EB0010F549B5
:1089C00001EB001130319DF8A00001EB00100078A0
:1089D0001070EF48D0F80C020521B0FBF1F201FB5A
:1089E000120000EB4001EA482C3000EB4111EA484C
:1089F000026841F81D2F80888880E548D0F80C0275
:108A00000521B0FBF1F201FB120000EB4001E04850
:108A10002C3000EB41129DF8B40040F2833110FB82
:108A200001F0DE4901EB800101F589619DF8A000AC
:108A300000EB400303EB001001EBC000406BC2F8F9
:108A40000900D348D0F80C020521B0FBF1F201FB7C
:108A5000120000EB4001CE482C3000EB41129DF893
:108A6000B40000EB400101EB0010CA4901EB00111A
:108A700030319DF8A00001EB00104068C2F82300DF
:108A800000229DF8B40000EB400101EB0010C14949
:108A900001EB001130319DF8A00001EB00104260A5
:108AA00000213A9154E0BA48D0F80C020521B0FBFD
:108AB000F1F201FB120000EB4001B5482C3000EB55
:108AC00041112731BDF8E8409DF8B40040F28332EF
:108AD00010FB02F0B14A02EB800202F589629DF8B8
:108AE000A00000EB400303EB001002EBC00090F885
:108AF000800040F2833210FB02F0A84A02EB8002B1
:108B000002F589629DF8B40040F2833310FB03F054
:108B1000A24B03EB800303F589639DF8A00000EBF3
:108B2000400505EB001003EBC00090F8810000EB5E
:108B3000400303EB001002EBC0024732BDF8E8002F
:108B4000001D105C0855BDF8E800401C81B23A9148
:108B5000BDF8E8000628A6DB00203A9042E000239A
:108B60009DF8B40040F2833110FB01F08B4901EB1A
:108B7000800101F589619DF8A00000EB400202EB45
:108B8000001001EBC00090F8800040F2833110FB30
:108B900001F0824901EB800101F589619DF8B40083
:108BA00040F2833210FB02F07C4A02EB800202F5B5
:108BB00089629DF8A00000EB400404EB001002EB7A
:108BC000C00090F8810000EB400202EB001001EBC6
:108BD000C0014731BDF8E8000B54BDF8E800401C67
:108BE00081B23A91BDF8E8000A28B8DB6848D0F8AD
:108BF0000C020521B0FBF1F080B201460990022081
:108C0000F0F766FA00210620F1F750FA6048D0F834
:108C10000C0200E003E25E49498D884206D25C48BE
:108C2000D0F80C02401C5A49C1F80C020021052062
:108C3000F1F73CFA9DF8B40000EB400101EB0010A5
:108C4000544901EB001030309DF8A01000EB0110EA
:108C5000801C0990007820F00802099802704C48A6
:108C6000D0F80C020521B0FBF1F201FB120000EB81
:108C7000400147482C3000EB4110D0F823202E98BB
:108C800000EB4001464800EB4110C0F823200020D3
:108C90003A9020E03E48D0F80C020521B0FBF1F2FA
:108CA00001FB120000EB400139482C3000EB411071
:108CB0002730BDF8E810425C2E9800EB40013848A0
:108CC00000EB41112731BDF8E8000A54BDF8E80077
:108CD000401C81B23A91BDF8E8000628DADB66E074
:108CE0009DF8B40000EB400101EB0010294901EBB5
:108CF000001030309DF8A01000EB0110801C09908E
:108D0000007820F008000830099908709DF8B40038
:108D100000EB400101EB00101E4901EB0010303068
:108D20009DF8A01000EB011042682E9800EB400166
:108D30001B4800EB4110C0F8232000203A9032E09D
:108D40009DF8B40040F2833110FB01F0134901EBB0
:108D5000800101F589619DF8A00000EB400200E070
:108D600005E202EB001001EBC0014731BDF8E8005D
:108D70000A5C2E9800EB4001094800EB41112731B5
:108D8000BDF8E8000A54BDF8E800401C81B209E0D3
:108D9000BC120020C8430020C731002088480020B2
:108DA000D81400203A91BDF8E8000628C8DB9DF8E9
:108DB000B40000EB400101EB0010FE4901EB001094
:108DC00030309DF8A01000EB0110801C0990007855
:108DD00020F02002099802709DF8B4100220F1F7EB
:108DE00065F99DF8B40040F2833110FB01F0F249BF
:108DF00001EB800000F589609DF8A01001EB4102B5
:108E000002EB011100EBC100223009902E9800EB1B
:108E10004001EA4800EB41100D30102208900999FA
:108E2000EFF713FA9DF8B40040F2833110FB01F024
:108E3000E14901EB800101F589619DF8A00000EB9B
:108E4000400202EB001001EBC0012E9800EB400243
:108E5000DA4800EB421051F81A2F40F8012F496808
:108E600041609DF8B40000EB400101EB0010D149D6
:108E700001EB001130319DF8A00001EB00100178EA
:108E80002E9800EB4002CD4800EB421001702E9866
:108E900000EB4001C94800EB4111C948026841F8A4
:108EA0001D2F808888809DF8B40040F2833110FB2C
:108EB00001F0C14901EB800101F589619DF8A00035
:108EC00000EB400202EB001001EBC000416B2E985A
:108ED00000EB4002B94800EB4210C0F8091000E076
:108EE0009CE09DF8B40000EB400101EB0010B1499B
:108EF00001EB001130319DF8A00001EB001041683A
:108F00002E9800EB4002AD4800EB4210C0F8231051
:108F10002E9881B208200991F1F7C8F800229DF837
:108F2000B40040F2833110FB01F0A34901EB800053
:108F300000F589609DF8A01001EB410303EB0111DE
:108F400000EBC10080F8462053E09DF8B40000EB30
:108F5000400101EB0010974901EB001030309DF803
:108F6000A01000EB0110801C0990007820F0040094
:108F7000001D099908709DF8B40000EB400101EB59
:108F800000108C4901EB001030309DF8A01000EB70
:108F90000110801C0990007820F080008030099931
:108FA000087001229DF8B40040F2833110FB01F0FB
:108FB000814901EB800002719DF8B40040F28331D9
:108FC00010FB01F07C4901EB800042799DF8B40070
:108FD00040F2833110FB01F0774901EB800000F58E
:108FE00089609DF8A01001EB410303EB011100F82B
:108FF00031208F229DF8B40040F2833110FB01F044
:109000006D4901EB800000F589609DF8A01001EB2F
:10901000410303EB011100EBC1004271C7E0BDF851
:10902000A400032857D101216548F53080F8341A8F
:109030009DF8B40040F2833110FB01F05E4901EB72
:10904000800101F589619DF8A00000EB400202EB70
:10905000001011F830109DF8B40040F2833210FB7C
:1090600002F0554A02EB80004079814234DA002157
:109070009DF8B40040F2833210FB02F04E4A02EB3E
:109080008000017101229DF8B40040F2833110FB91
:1090900001F0494901EB800101F589619DF8A000CB
:1090A00000EB400303EB001001F830208F229DF805
:1090B000B40040F2833110FB01F03F4901EB800026
:1090C00000F589609DF8A01001EB410303EB01114D
:1090D00000EBC10042714AE09DF8B40040F28331D8
:1090E00010FB01F0344901EB800000F589609DF828
:1090F000A01001EB410202EB011100EBC1008078EE
:10910000802834D100219DF8B40040F2833210FB56
:1091100002F0294A02EB8000017180229DF8B40020
:1091200040F2833110FB01F0234901EB800101F58E
:1091300089619DF8A00000EB400303EB001001EBF8
:10914000C000427100229DF8B40040F2833110FB50
:1091500001F0194901EB800000F589609DF8A0102D
:1091600001EB410303EB011100EBC10082701EE033
:10917000BDF8A400032819D100211148F53080F86A
:10918000341A8F229DF8B40040F2833110FB01F0B5
:10919000094901EB800000F589609DF8A01001EB02
:1091A000410303EB011100EBC100427100BF00BF9E
:1091B00005F089BDC843002088480020D81400204D
:1091C000C73100209DF8B40000EB4001C1EBC01096
:1091D000FE4911F83000042801D125900BE09DF8DC
:1091E000B40000EB4001C1EBC010F84911F83000A9
:1091F000152800D125909DF8B40000EB4001C1EB8B
:10920000C010F24901EBC00041789DF8B40000EBBA
:109210004002C2EBC010ED4A12F8300041EA0020D3
:1092200041F23001884202D1A62025903DE09DF810
:10923000B40000EB4001C1EBC010E44901EBC000F9
:1092400041789DF8B40000EB4002C2EBC010DF4A49
:1092500012F8300041EA002041F23101884202D187
:10926000A720259021E09DF8B40000EB4001C1EB60
:10927000C010D64911F83000022816D19DF8B4006C
:1092800000EB4001C1EBC010D04901EBC0000179F7
:109290009DF8B40000EB4002C2EBC010CB4A02EBD9
:1092A000C000C07841EA002125919DF8B40040F249
:1092B000833110FB01F0C64901EB8000C178279192
:1092C0009DF8B40040F2833110FB01F0C04901EB7E
:1092D000800108319DF89C0000EB001001EB80003C
:1092E00082789DF8B40040F2833110FB01F0B84958
:1092F00001EB800108319DF89C0000EB001001EBB0
:109300008000C0781044C1B228910021B14A9DF874
:10931000B40002EB00129DF89C0011543A913AE01F
:109320009DF8B40040F2833110FB01F0A84901EB35
:10933000800108319DF89C0000EB001001EB8000DB
:1093400002799DF8B40040F2833110FB01F0A0498E
:1093500001EB800108319DF89C0000EB001001EB4F
:1093600080008178BDF8E800084400EB400101EB83
:1093700000119DF8B40040F2833310FB03F0944BCE
:1093800003EB800000F5896000F83120BDF8E800AB
:10939000401C81B23A919DF8B40040F2833110FB39
:1093A00001F08B4901EB800108319DF89C0000EB36
:1093B000001011F82010BDF8E8008142B0DCBDF8C3
:1093C000941043F23002881A91427DD009DC0429BE
:1093D0007BD015297AD0A62910D0A72942F03E8546
:1093E00050E1B0F5C06F72D0A0F2016000286FD0DC
:1093F00001286ED00428F1D102F030B800219DF888
:10940000B40040F2833210FB02F0714A02EB80009C
:1094100001719DF8B40040F2833110FB01F0114658
:1094200001EB800008309DF89C1001EB011100EB6E
:1094300081000079052824DC06229DF8B40040F262
:10944000833110FB01F0624901EB800108319DF886
:109450009C0000EB001001EB80000271A8229DF837
:10946000B40040F2833110FB01F0594901EB800058
:1094700008309DF89C1001EB011100EB8100427156
:10948000FEE09DF8B40040F2833110FB01F050493A
:1094900001EB800008309DF89C1001EB011100EBFE
:1094A000810000790A282BDC0B229DF8B40040F2E1
:1094B000833110FB01F0464901EB800108319DF832
:1094C0009C0000EB001005E094E111E2FEE3FEE3F6
:1094D000FEE3FEE301EB80000271A9229DF8B400D7
:1094E00040F2833110FB01F0394901EB8000083074
:1094F0009DF89C1001EB011100EB81004271BFE06F
:109500009DF8B40040F2833110FB01F0304901EBCB
:10951000800008309DF89C1001EB011100EB8100E8
:1095200000790F2824DC10229DF8B40040F283312A
:1095300010FB01F0264901EB800108319DF89C00E9
:1095400000EB001001EB80000271A2229DF8B40034
:1095500040F2833110FB01F01D4901EB800008301F
:109560009DF89C1001EB011100EB8100427187E036
:109570009DF8B40040F2833110FB01F0144901EB77
:10958000800008309DF89C1001EB011100EB810078
:109590004079A5282DD19DF8B40040F2833110FB0D
:1095A00001F00B4901EB800108319DF89C0000EBB4
:1095B000001001EB8000C1789DF8B40000EB400280
:1095C00002EB0010044A02EB001007E0388F002085
:1095D00088480020B8410020C8430020303000EB0C
:1095E0000110801C0990007820F00400001D0999EA
:1095F00008709DF8B40040F2833110FB01F0FC4983
:1096000001EB800008309DF89C1001EB011100EB8C
:1096100081008079A12833D09DF8B40040F28331D5
:1096200010FB01F0F24901EB800108319DF89C002C
:1096300000EB001001EB800082799DF8B40040F24D
:10964000833110FB01F0EA4901EB800108319DF8FC
:109650009C0000EB001001EB80004271A1229DF8FC
:10966000B40040F2833110FB01F0E14901EB8000CE
:1096700008309DF89C1001EB011100EB8100827114
:1096800002F0ECBB00219DF8B40040F2833210FBE5
:1096900002F0D74A02EB800001719DF8B40040F25D
:1096A000833110FB01F0114601EB800008309DF87A
:1096B0009C1001EB011100EB8100007908281DDCF2
:1096C00000219DF8B40040F2833210FB02F0C84A3A
:1096D00002EB8000017108229DF8B40040F2833152
:1096E00010FB01F0C24901EB800008309DF89C108E
:1096F00001EB011100EB8100027124E09DF8B40040
:1097000040F2833110FB01F0B94901EB80000830D1
:109710009DF89C1001EB011100EB810000790B28F2
:1097200011DC0C229DF8B40040F2833110FB01F0F3
:10973000AF4901EB800008309DF89C1001EB01114E
:1097400000EB810002719DF8B40040F2833110FB00
:1097500001F0A74901EB800008309DF89C1001EB57
:10976000011100EB81004079A42830D19DF8B400AC
:1097700000EB400101EB00109E4901EB001030307E
:109780009DF8A01000EB0110801C0990007820F0DB
:10979000200020300999087000229DF8B40040F2A2
:1097A000833110FB01F0924901EB800101F58961E1
:1097B0009DF8A00000EB400303EB001001EBC0009C
:1097C00080F845209DF8B4100220F0F76FFCA1222C
:1097D0009DF8B40040F2833110FB01F0844901EBA5
:1097E000800008309DF89C1001EB011100EB810016
:1097F000427145E700203A9015E09DF8B40000EB77
:109800004001C1EBC0107C4901EBC001BDF8E8008C
:10981000C01C095C16AABDF8E8001154BDF8E800A8
:10982000401C81B23A91BDF8E8000628E5DB06212C
:1098300016A81EF0C1FF0021CDE93001DDE930019D
:10984000000A40EA0160309A801841EB21214FF470
:1098500080724FF00003CDE90801EEF7B3FC9DF8EC
:10986000B40040F2833110FB01F0614901EB80014B
:1098700001F589619DF89C0000EB400303EB0010AB
:1098800001EBC000027100219DF8B40040F2833268
:1098900010FB02F0564A02EB8000017104229DF891
:1098A000B40040F2833110FB01F0514901EB80011B
:1098B00001F589619DF89C0000EB400303EB00106B
:1098C00001F83020A7229DF8B40040F2833110FB4C
:1098D00001F0474901EB800000F589609DF89C107C
:1098E00001EB410303EB011100EBC1004271C7E63C
:1098F0009DF8B40040F2833110FB01F03C4901EBCC
:10990000800008309DF89C1001EB011100EB8100F4
:109910000079042872DA00219DF8B40040F2833205
:1099200010FB02F0324A02EB80000171A1229DF887
:10993000B40040F2833110FB01F02D4901EB8001AE
:1099400008319DF89C0000EB001001EB8000427193
:109950009DF8B40040F2833110FB01F0244901EB83
:10996000800108319DF89C0000EB001001EB8000A5
:10997000001D09900078401CC2B2099802709DF841
:10998000B40040F2833110FB01F0194901EB800073
:1099900008309DF89C1001EB011100EB810000796B
:1099A000042823D10A229DF8B40040F2833110FB31
:1099B00001F00F4901EB800108319DF89C0000EB9C
:1099C000001001EB80000271A3229DF8B40040F268
:1099D000833110FB01F0064901EB800008309DF84F
:1099E0009C1001EB011100EB8100427137E305E0AF
:1099F00088480020C8430020388F00209DF8B4001C
:109A000040F2833110FB01F0FE4901EB8000083089
:109A10009DF89C1001EB011100EB810000790428F6
:109A20002FD100219DF8B40040F2833210FB02F0E8
:109A3000F44A02EB8000017105229DF8B40040F267
:109A4000833110FB01F0EF4901EB800108319DF8F3
:109A50009C0000EB001001EB80000271A3229DF836
:109A6000B40040F2833110FB01F0E64901EB8000C5
:109A700008309DF89C1001EB011100EB8100427150
:109A8000EDE29DF8B41040F2833011FB00F0DD49A7
:109A900001EB800008309DF89C1001EB011100EBF8
:109AA0008100007908282FDC00219DF8B40040F2E5
:109AB000833210FB02F0D34A02EB800001710922CD
:109AC0009DF8B40040F2833110FB01F0CD4901EB69
:109AD000800108319DF89C0000EB001001EB800034
:109AE0000271A7229DF8B40040F2833110FB01F00F
:109AF000C44901EB800008309DF89C1001EB011176
:109B000000EB81004271AAE29DF8B41040F283306C
:109B100011FB00F0BB4901EB800008309DF89C1060
:109B200001EB011100EB8100007909282FDC0021F5
:109B30009DF8B40040F2833210FB02F0B14A02EB10
:109B4000800001710A229DF8B40040F2833110FBBD
:109B500001F0AC4901EB800108319DF89C0000EB5D
:109B6000001001EB80000271A3229DF8B40040F2C6
:109B7000833110FB01F0A34901EB800008309DF810
:109B80009C1001EB011100EB8100427167E29DF82E
:109B9000B41040F2833011FB00F09A4901EB8000D1
:109BA00008309DF89C1001EB011100EB8100007959
:109BB0000D282FDC00219DF8B40040F2833210FB09
:109BC00002F0904A02EB800001710E229DF8B40071
:109BD00040F2833110FB01F08A4901EB800108312A
:109BE0009DF89C0000EB001001EB80000271A122A7
:109BF0009DF8B40040F2833110FB01F0814901EB84
